:04200000F0EF69F0A4
:0820080000C004F001C005F066
:1020100002C006F0076A03C008F000016F00D4FF99
:1020200009F06F00D8FF0AF06F00DCFF0BF03901F8
:1020300093A71EEF10F0A3B712EF2AF093AF24EF8F
:1020400010F0A3BFF4EF29F094A12AEF10F0A4B18F
:1020500025EF25F096A530EF10F0A6B5CAEF29F0D0
:1020600096AD36EF10F0A6BD00EF26F098AD3CEF30
:1020700010F0A8BD3BEF26F0600027F0F5FF6000F0
:102080002BF0F6FF60002FF0F7FF04C000F005C052
:1020900001F006C002F0078E08C003F01100F76AD5
:1020A000AE0FF66E200EF7220900F5501200280C34
:1020B0000106C00FF66E200EF7220900F55012003F
:1020C0000000C1C081C1400101C3C003800241C200
:1020D00001C6C006800741C70005C1C581C44004D0
:1020E00001CCC00C800D41CD000FC1CF81CE400E80
:1020F000000AC1CA81CB400B01C9C009800841C890
:1021000001D8C018801941D9001BC1DB81DA401AFF
:10211000001EC1DE81DF401F01DDC01D801C41DCCF
:102120000014C1D481D5401501D7C017801641D6FF
:1021300001D2C012801341D30011C1D181D040100F
:1021400001F0C030803141F10033C1F381F24032FF
:102150000036C1F681F7403701F5C035803441F4CF
:10216000003CC1FC81FD403D01FFC03F803E41FE7F
:1021700001FAC03A803B41FB0039C1F981F840388F
:102180000028C1E881E9402901EBC02B802A41EAFF
:1021900001EEC02E802F41EF002DC1ED81EC402CCF
:1021A00001E4C024802541E50027C1E781E64026FF
:1021B0000022C1E281E3402301E1C021802041E00F
:1021C00001A0C060806141A10063C1A381A24062FF
:1021D0000066C1A681A7406701A5C065806441A4CF
:1021E000006CC1AC81AD406D01AFC06F806E41AE7F
:1021F00001AAC06A806B41AB0069C1A981A840688F
:102200000078C1B881B9407901BBC07B807A41BAFE
:1022100001BEC07E807F41BF007DC1BD81BC407CCE
:1022200001B4C074807541B50077C1B781B64076FE
:102230000072C1B281B3407301B1C071807041B00E
:102240000050C190819140510193C05380524192FE
:102250000196C056805741970055C19581944054CE
:10226000019CC05C805D419D005FC19F819E405E7E
:10227000005AC19A819B405B0199C059805841988E
:102280000188C04880494189004BC18B818A404AFE
:10229000004EC18E818F404F018DC04D804C418CCE
:1022A0000044C184818540450187C04780464186FE
:1022B0000182C042804341830041C181818040400E
:1022C000583220256325632563256325632563250F
:1022D000632563202020202000005831202563251D
:1022E00063256325632563256325632563202020FB
:1022F00020200000706F736963616F2020202536F5
:102300004C640000656E747261646120202020209E
:1023100020253033750020504152414D4554524FD5
:102320005320444520200000205445535445204765
:1023300052415641444F5320000020504152412009
:10234000434F4E54494E5541522000004C4942459E
:102350005245204F5320424F544F45530000414AAD
:10236000555354452020202020202025322E306631
:102370002525000053616972202020202D20202077
:10238000202B202000002020504F52544120534148
:102390004645545920200000736169722020207343
:1023A000696D2020206E616F00002020504F525434
:1023B0004120534146455459202000002020504FD1
:1023C000525441204154495641444F20000020209E
:1023D000504F52544120534146455459202000004B
:1023E000504F525441204445534154495641444F63
:1023F00000002074696D657220667265657A657289
:102400003F2000007361697220202073696D2020D5
:10241000206E616F00002074696D65722020667205
:1024200065657A657220000020202020616A75733E
:10243000746172202020202000002074696D657274
:102440002020667265657A657220000020202020B9
:102450006D616E7469646F202020200054494D45E1
:102460005220202020253375204D696E00005361D5
:102470006972202020202D20202020202B200000E9
:1024800054494D455220202020253375204D696E3A
:1024900000002045535441204E4120454550524FA5
:1024A0004D20000020415449564152202020504FD9
:1024B000525441200000465245455A455220505240
:1024C000494D4549524F000020504F52544120463B
:1024D0005245455A45522020000073616972202000
:1024E0002073696D2020206E616F000020504F52D4
:1024F000544120465245455A455220200000205460
:10250000494D4552204154495641444F2020000036
:1025100020504F52544120465245455A45522020A2
:10252000000054494D4552204445534154495641B9
:10253000444F000020504F52544120465245455AC6
:10254000455220200000204E414F205045524D4919
:102550005449444F20200000464341204455504CEC
:102560004F20504152414441000073616972202064
:102570002073696D2020206E616F0000464341206A
:102580004455504C41205041524144410000464383
:102590004120202020202020415449564F20000077
:1025A000464341204455504C412050415241444102
:1025B00000004643412020202020494E41544956E6
:1025C0004F200000425220434F4E544147454D3F5B
:1025D0002020202000007361697220202073696D23
:1025E0002020206E616F000042522020434F4E5445
:1025F0004147454D202020200000434F4E54414785
:10260000454D20204154495641200000425220208F
:10261000434F4E544147454D202020200000434F5A
:102620004E544147454D20494E41544956410000C2
:10263000515444205245544F524E4F532025337528
:10264000000053616972202020202D2020202020AE
:102650002B200000515444205245544F524E4F53AA
:102660002025337500002045535441204E4120451C
:102670004550524F4D20000044454C4159204142A5
:102680004552545552413F20000073616972202029
:102690002073696D2020206E616F000044454C411D
:1026A0005920414245525455524120200000444592
:1026B0004C41592020202020415449564F200000F1
:1026C00044454C41592041424552545552412020E5
:1026D000000044454C4159202020494E4154495660
:1026E0004F20000054502044454C4159202533755B
:1026F00020534547000053616972202020202D207F
:10270000202020202B20000054502044454C4159CB
:102710002025337520534547000020455354412060
:102720004E4120454550524F4D2000002052454C0F
:102730004553205041206520504620200000736101
:10274000697220202073696D2020206E616F000067
:102750002052454C455320504120652050462020B2
:102760000000202020204154495641444F5320204E
:10277000202000002052454C455320504120652028
:1027800050462020000020204445534154495641E2
:10279000444F532020200000504120652050462007
:1027A00050554C5345203F20000073616972202032
:1027B0002073696D2020206E616F00002050412041
:1027C000652050462050554C5345202000002020C5
:1027D00020204154495641444F53202020200000DE
:1027E00020504120652050462050554C5345202014
:1027F000000020204445534154495641444F532042
:1028000020200000504F5320444553415420464F50
:10281000544F313F00002020202020202073696D7C
:102820002020206E616F0000706F732061747561ED
:102830006C25364C6400706F73204646202020259E
:10284000364C64002020202020504F534943414FF4
:1028500020202020000020202020204752415641E7
:1028600044412020202000002020202020504F53D1
:102870004943414F20202020000020202020204DCF
:10288000414E544944412020202000002020204374
:102890004F4E5441544F5245532020200000736145
:1028A000697220202073696D2020206E616F000006
:1028B00053414944415320434F4E5441544F5220B9
:1028C0000000202020204154495641444F532020ED
:1028D0002020000053414944415320434F4E54416E
:1028E000544F522000002020444553415449564142
:1028F000444F53202020000020202020202020535F
:10290000696D20204E616F20000020202020436F41
:102910006E6669726D613F2020200000202020201B
:1029200020202053692020204E6F202000002020EE
:102930002020436F6E6669726D613F202020000089
:102940002020202020205965732020204E6F202039
:102950000000202020436F6E6669726D203F2020AA
:1029600020200000205041524120434F4E54494EF8
:10297000554152200000205041524120434F4E54B7
:10298000494E55415220000020464F522053455495
:1029900054494E472055502000004C49424552456D
:1029A000204F5320424F544F45530000204C494282
:1029B00045524520424F544F4E455320000052454A
:1029C0004C454153452020425554544F4E5300002E
:1029D00020202020202020202020202020202020F7
:1029E0000000202020202020202020202020202027
:1029F00020200000204449474954452041205345A8
:102A00004E4841200000454E54524520434F4E54FD
:102A1000524153454E41000020454E5445522050EE
:102A2000415353574F52442000004F6B2020202029
:102A30002020253175202020202025317520000000
:102A40002044494749544520412053454E484120A0
:102A50000000454E54524520434F4E545241534579
:102A60004E41000020454E5445522050415353578B
:102A70004F52442000004F6B202020202020253181
:102A80007520202020202531752000002044494752
:102A900049544520412053454E4841200000454EB1
:102AA00054524520434F4E54524153454E4100002D
:102AB00020454E5445522050415353574F524420C5
:102AC00000004F6B20202020202025317520202061
:102AD0002020253175200000202020202020534573
:102AE0004E48412020202020200020202020494E38
:102AF000434F5252455441212020200020202043A2
:102B00004F4E54524153454E41202020200020205A
:102B100020494E434F52524543544121202020002A
:102B2000202020202057524F4E47202020202020B8
:102B300020002020202050415353574F5244212041
:102B400020202000204C41444F204D4F544F522014
:102B50003F2020200000204C41444F204D4F544F37
:102B600052203F2020200000204D4F544F52205330
:102B7000494445203F202020000053696D2020203B
:102B80002020256320202020202563200000536979
:102B900020202020202025632020202020256320A5
:102BA000000059657320202020202563202020204C
:102BB000202563200000204C41444F204D4F544FAE
:102BC00052203F2020200000204C41444F204D4FF8
:102BD000544F52203F2020200000204D4F544F5290
:102BE0002053494445203F202020000053696D2098
:102BF0002020202025632020202020256320000085
:102C000053692020202020202563202020202025FB
:102C10006320000059657320202020202563202098
:102C200020202025632000002020204D4F544F52AB
:102C30002053494445202020000020204C41444F8F
:102C40002020204D4F544F522020000073616972A4
:102C50002020206573712020206469720000736158
:102C60006C69722020697A712020206465720000EE
:102C70004578697420204C656674205269676874D1
:102C80000000204D4F544F5220455351554552445A
:102C90004F3F00006772617661722065737120207A
:102CA0006469722000004D4F544F5220495A5155CB
:102CB000494552444F3F000067726162617220696A
:102CC0007A71202064657220000020204D4F544FFF
:102CD00052202020204C4546543F0000536574206C
:102CE000204C656674202052696768740000204D8E
:102CF0004F544F52204449524549544F203F000001
:102D00006772617661722065737120206469722038
:102D10000000204D4F544F52204445524543484FE8
:102D2000203F000067726162617220697A71202021
:102D300064657220000020204D4F544F52202052D5
:102D400049474854203F000053657420204C656675
:102D50007420205269676874000020204643204197
:102D600042455254555241203F20000053696D2086
:102D70002020202025632020202020256320000003
:102D800020204643204150455254555241203F2077
:102D900000005369202020202020256320202020AF
:102DA00020256320000020204C494D495420204F0D
:102DB00050454E203F2000005965732020202020E0
:102DC0002563202020202025632000006772617683
:102DD00061646F20202025364C64000053616972C5
:102DE0002020446573636520536F6265000067723D
:102DF000616261646F20202025364C6400005361BD
:102E00006C6972204162616A6F20537562650000CF
:102E10005365745F6F6B2020202025364C640000C2
:102E20004578697420202020446F776E20205570EB
:102E30000000706F7320617475616C2025364C64DE
:102E40000000477261766120446573636520536FAB
:102E500062650000706F732061637475616C253664
:102E60004C6400004772616261204162616A6F20B8
:102E7000537562650000706F732061637475616CD7
:102E800025364C6400004578697420202020446F6A
:102E9000776E202055700000464320414245525431
:102EA00055524120494E543F000053696D20202067
:102EB0002020256320202020202563200000464379
:102EC00020415045525455524120494E543F000034
:102ED0005369202020202020256320202020202529
:102EE00063200000494E54204F50454E20204C494D
:102EF0004D49543F00005965732020202020256350
:102F00002020202020256320000067726176616404
:102F10006F20202025364C64000053616972202008
:102F2000446573636520536F626500006772616278
:102F300061646F20202025364C64000053616C6969
:102F400072204162616A6F205375626500005365AB
:102F5000745F6F6B2020202025364C64000045787C
:102F6000697420202020446F776E20205570000067
:102F7000706F7320617475616C2025364C6400009D
:102F8000477261766120446573636520536F6265A3
:102F90000000706F732061637475616C25364C643A
:102FA00000004772616261204162616A6F2053755F
:102FB00062650000706F732061637475616C253603
:102FC0004C6400004578697420202020446F776E9F
:102FD0002020557000002046432046454348414D7F
:102FE000454E544F203F000053696D202020202083
:102FF000256320202020202563200000202020465B
:1030000043204349455252453F2020200000536948
:103010002020202020202563202020202025632020
:10302000000020204C494D49542020434C4F53452B
:103030003F20000059657320202020202563202098
:1030400020202025632000006772617661646F2074
:10305000202025364C6400005361697220204465AD
:1030600073636520536F626500006772616261641B
:103070006F20202025364C64000053616C6972205B
:103080004162616A6F205375626500005365745F29
:103090006F6B2020202025364C6400004578697431
:1030A00020202020446F776E202055700000706F24
:1030B0007320617475616C2025364C640000477282
:1030C00061766120446573636520536F626500001B
:1030D000706F732061637475616C25364C640000F9
:1030E0004772616261204162616A6F205375626557
:1030F0000000706F732061637475616C25364C64D9
:1031000000004578697420202020446F776E2020CD
:103110005570000020414A205245442056454C201D
:103120004645203F000053696D2020202020256364
:103130002020202020256320000020414A205245E5
:10314000442056454C204345203F00005369202031
:10315000202020202563202020202025632000001F
:1031600053455420534C4F2053504420434C203F50
:103170000000596573202020202025632020202076
:103180002025632000007265647563616F20202034
:1031900025357525250053616972202020202D20BA
:1031A000202020202B200000726564756363696F06
:1031B0006E2025357525250053616C69722020200D
:1031C0002D20202020202B200000736C6F207261A6
:1031D00074652020253575252500457869742020E3
:1031E00020202D20202020202B20000072656475D7
:1031F00063616F2020202535752525004772617693
:10320000617220202D20202020202B2000007265BC
:1032100064756363696F6E202535752525004772D7
:103220006162617220202D20202020202B200000B0
:10323000736C6F207261746520202535752525001B
:103240005365745F6F6B20202D20202020202B20C1
:103250000000677261766F752071756174726F20FE
:103260002020000020414A205245442056454C2051
:103270004142203F000053696D202020202025631B
:103280002020202020256320000020414A20524594
:10329000442056454C204150203F000053692020D7
:1032A00020202020256320202020202563200000CE
:1032B00053455420534C4F20535044204F50203FEF
:1032C0000000596573202020202025632020202025
:1032D0002025632000007265647563616F202020E3
:1032E00025357525250053616972202020202D2069
:1032F000202020202B200000726564756363696FB5
:103300006E2025357525250053616C6972202020BB
:103310002D20202020202B200000736C6F20726154
:103320007465202025357525250045786974202091
:1033300020202D20202020202B2000007265647585
:1033400063616F2020202535752525004772617641
:10335000617220202D20202020202B20000072656B
:1033600064756363696F6E20253575252500477286
:103370006162617220202D20202020202B2000005F
:10338000736C6F20726174652020253575252500CA
:1033900053657420202020202D20202020202B2049
:1033A0000000414A555354452020204C4F4F50496E
:1033B0004E470000414A555354452020204C4F4F62
:1033C00050494E470000204C4F4F50494E47202057
:1033D000534554555020000053696D202020202073
:1033E0002563202020202025632000005369202011
:1033F000202020202563202020202025632000007D
:10340000596573202020202025632020202020259E
:1034100063200000414A555354452020202020209D
:103420002025322E30662525000053616972202048
:1034300020202D202020202B20200000414A555301
:1034400054452020202020202025322E306625259E
:10345000000053616C69722020202D202020202B39
:1034600020200000536574202056616C7565202073
:103470002025322E306625250000457869742020ED
:1034800020202D202020202B20200000414A5553B1
:1034900054452020202020202025322E306625254E
:1034A000000047726176617220202D202020202BA1
:1034B00020200000414A5553544520202020202040
:1034C0002025322E30662525000047726162617228
:1034D00020202D202020202B202000005365742048
:1034E0002056616C756520202025322E30662525FA
:1034F000000053657420202020202D202020202B28
:103500002020000020434D44204D414E55414C2089
:103510003F202020000053696D20202020202563BB
:103520002020202020256320000053692020202017
:1035300020202563202020202025632000005965BD
:103540007320202020202563202020202025632098
:10355000000020434D44202020204D414E55414C39
:1035600020200000736169722066656368612061D4
:1035700062726520000073616C6972206162616A29
:103580006F207375626500004578697420202020E3
:10359000446F776E202055700000414A2054454DFD
:1035A000504F204645434841203F000053696D205D
:1035B00020202020256320202020202563200000BB
:1035C000414A205449454D50204349455252453FB8
:1035D0000000536920202020202025632020202067
:1035E00020256320000041444A20434C4F5345208E
:1035F00054494D45203F000059657320202020206C
:1036000025632020202020256320000054504645BB
:10361000434841202533752073656773000053616B
:103620006972202020202D20202020202B20000027
:1036300054504349455252452025337520736567E0
:10364000000053616C69722020202D202020202052
:103650002B2000005443434C4F5345202025337505
:1036600020736563000045786974202020202D2098
:10367000202020202B200000545046454348412064
:103680002533752073656773000047726176617238
:1036900020202D20202020202B20000054504349A2
:1036A00045525245202533752073656700004772E7
:1036B000616261722020202D20202020202B2000FC
:1036C0005443434C4F534520202533752073656385
:1036D00000005365742020202020202D2020202051
:1036E000202B20002054454D504F52495A41444F01
:1036F00052203F2000002054454D504F52495A411E
:10370000444F52203F200000202020202054494DCB
:103710004552203F20202020000053696D202020AA
:1037200020202563202020202025632000005369CD
:1037300020202020202025632020202020256320F9
:1037400000005965732020202020256320202020A0
:103750002025632000002054454D504F52495A41C6
:10376000444F52203F2000002054454D504F5249B5
:103770005A41444F52203F20000020202020205456
:10378000494D4552203F202020200000736169727E
:1037900020202073696D2020206E616F000073610E
:1037A0006C697220207369202020206E6F20000039
:1037B000457869742020796573202020206E6F2061
:1037C00000002054454D504F52495A41444F522019
:1037D000202000002054454D504F52495A41444F3B
:1037E000522020200000202020202054494D455206
:1037F0002020202020200000736169722020207387
:10380000696D2020206E616F000073616C69722009
:10381000207369202020206E6F2000004578697495
:103820002020796573202020206E6F200000205416
:10383000454D504F52495A41444F522020200000DC
:103840002054454D504F52495A41444F5220202058
:103850000000202020202054494D455220202020C7
:10386000202000006772617661722073696D2020EC
:103870006E616F200000677261626172207369205F
:1038800020206E6F20200000736574202020796551
:10389000732020206E6F202000002054454D504F93
:1038A00052495A41444F5220202000002054454D97
:1038B000504F52495A41444F5220202000002020AE
:1038C00020202054494D4552202020202020000057
:1038D0006772617661722073696D20206E616F205E
:1038E00000006772616261722073692020206E6F30
:1038F000202000007365742020207965732020202B
:103900006E6F202000004944494F4D412F4C414EDD
:1039100047554147453F0000532F59202020202084
:103920002563202020202025632000004944494FA2
:103930004D412F4C414E4755414745200000454ED3
:1039400047202020204553502020504F5254000043
:103950004944494F4D412F4C414E47554147452021
:103960000000454E47202020204553502020504F36
:10397000525400004944494F4D412F4C414E475548
:1039800041474520000020202020454E474C495308
:1039900048202020202000004944494F4D412F4C11
:1039A000414E4755414745200000202020204553E7
:1039B00050414E4F4C202020202000004944494FC8
:1039C0004D412F4C414E4755414745200000202096
:1039D00020504F5254554755455320202020000079
:1039E0002020202020524144494F203F20202020E9
:1039F000200053696D2020202020256320202020D6
:103A00002025632000002020202020524144494FDF
:103A100020203F202020200053692020202020202B
:103A20002563202020202025632000002020202046
:103A300020524144494F203F20202020200059653A
:103A40007320202020202563202020202025632093
:103A500000002020202020524144494F20202020D7
:103A6000202000007361697220202073696D20207E
:103A7000206E616F000073616C6972202073692091
:103A80002020206E6F200000457869742020796521
:103A900073202020206E6F200000202020555341ED
:103AA0005220524144494F20202020006772617605
:103AB00061722073696D20206E616F200000677253
:103AC000616261722073692020206E6F20200000E7
:103AD0007365742020207965732020206E6F20206C
:103AE000000020202053454D20524144494F2020C2
:103AF0002020202020006772617661722073696D3A
:103B000020206E616F200000677261626172207315
:103B1000692020206E6F2020000073657420202013
:103B20007965732020206E6F202000002020202047
:103B30002053616972203F2020202020000053691B
:103B40006D20202020202563202020202025632098
:103B50000000202020202053616C6972203F20202B
:103B600020200000536920202020202025632020D1
:103B70002020202563200000202020202045786977
:103B800074203F2020202020000059657320202031
:103B900020202563202020202025632000002020D5
:103BA00020204154454E43414F2120202020000039
:103BB00020564F43452056414920454E54524152CC
:103BC0000000202020204154454E43494F4E2020E4
:103BD000202000002020555354454420454E545287
:103BE000415241200000202020205741524E494E92
:103BF000472020202020000020202020454E544532
:103C000052494E472020202000002020454D2054BE
:103C1000524F4341204445202020000020202050C6
:103C20004152414D4554524F532020200000202046
:103C3000412043414D42494F20444520202000006F
:103C4000202020504152414D4554524F53202020B6
:103C50000000202020204348414E47494E47202065
:103C600020200000202020202020534554555020A3
:103C70002020202000002020434F4E5452412D533D
:103C8000454E4841202000004F6B2020202020205E
:103C9000253175202020202025317520000020208E
:103CA000434F4E5452412D53454E48412020000071
:103CB0004F6B20202020202025317520202020201F
:103CC0002531752000002020434F4E5452412D5382
:103CD000454E4841202000004F6B2020202020200E
:103CE000253175202020202025317520000020203E
:103CF0002020202053454E48412020202020200015
:103D000020202020494E434F52524554412120202B
:103D10002000414755415244414E444F20464543BF
:103D20004841000054454D504F20464543484152BC
:103D30002025334C75004553504552414E444F2089
:103D400043455252415200005449454D504F204383
:103D5000455252412025334C750057414954494E34
:103D60004720544F20434C4F5345000054494D4584
:103D70002020434C4F5345202025334C75004245AD
:103D80002020202020202020202020202020000073
:103D900042412020202020202020202020202020E0
:103DA000000042452F4241202020202020202020BA
:103DB00020200000425220202020202020202020EF
:103DC00020202020000042452F4252202020202089
:103DD000202020202020000042412F42522020207D
:103DE000202020202020202000002050415241444B
:103DF00041202041424552544120000042452F427B
:103E0000412F425220202020202020200000463137
:103E100020202020202020202020202020200000E2
:103E200042452F4631202020202020202020202005
:103E3000000042412F463120202020202020202039
:103E40002020000042452F42412F463120202020D3
:103E500020202020000042522F4631202020202008
:103E6000202020202020000042452F42522F4631A2
:103E70002020202020202020000042412F42522FCD
:103E800046312020202020202020000042452F42C3
:103E9000412F42522F463120202020200000463260
:103EA0002020202020202020202020202020000052
:103EB00042452F4632202020202020202020202074
:103EC000000042412F4632202020202020202020A8
:103ED0002020000042452F42412F46322020202042
:103EE00020202020000042522F4632202020202077
:103EF000202020202020000042452F42522F463211
:103F00002020202020202020000042412F42522F3C
:103F100046322020202020202020000042452F4231
:103F2000412F42522F4632202020202000004631CF
:103F30002F4632202020202020202020202000007A
:103F400042452F46312F463220202020202020209D
:103F5000000042412F46312F4632202020202020D1
:103F60002020000042452F42412F46312F4632206B
:103F700020202020000042522F46312F46322020A0
:103F8000202020202020000042452F42522F463181
:103F90002F46322020202020200042412F42522F45
:103FA00046312F46322020202020000042452F425B
:103FB000412F42522F46312F4632202000004C2004
:103FC0002020202020202020202020202020000031
:103FD00042452F4C2020202020202020202020205F
:103FE000000042412F4C2020202020202020202093
:103FF0002020000042452F42412F4C20202020202D
:1040000020202020000042522F4C20202020202061
:10401000202020202020000042452F42522F4C20FB
:104020002020202020202020000042412F42522F1B
:104030004C202020202020202020000042452F421C
:10404000412F42522F4C20202020202000004631BA
:104050002F4C202020202020202020202020000065
:1040600042452F46312F4C20202020202020202088
:10407000000042412F46312F4C20202020202020BC
:104080002020000042452F42412F46312F4C202056
:1040900020202020000042522F46312F4C2020208B
:1040A000202020202020000042452F42522F463160
:1040B0002F4C202020202020000042412F42522F50
:1040C00046312F4C202020202020000042452F4246
:1040D000412F42522F46312F4C20202000004632E3
:1040E0002F4C2020202020202020202020200000D5
:1040F00042452F46322F4C202020202020202020F7
:10410000000042412F46322F4C202020202020202A
:104110002020000042452F42412F46322F4C2020C4
:1041200020202020000042522F46322F4C202020F9
:10413000202020202020000042452F42522F4632CE
:104140002F4C000042412F42522F46322F4C20204C
:1041500020202020000042452F42412F42522F466E
:10416000322F4C202020000046312F46322F4C2089
:104170002020202020202020000042452F46312FE3
:1041800046322F4C202020202020000042412F4684
:10419000312F46322F4C2020202020200000424585
:1041A0002F42412F46312F46322F4C202020000035
:1041B00042522F46312F46322F4C202020202020E3
:1041C000000042452F42522F46312F46322F4C20BD
:1041D0002020000042412F42522F46312F46322FDD
:1041E0004C20200042452F42412F42522F46312F72
:1041F00046322F4C00004E414F20434845474F5513
:10420000204E412020200000253275202020202033
:1042100020202020202020202000205041524144F6
:10422000412020414245525441200000205041523B
:104230004144412020414249455254410000202040
:1042400020204F50454E2053544F50202020000036
:1042500020504F525441202050415241444120208F
:104260000000202020454D204D4F444F2053544FF7
:104270002020000058312025632563256325632510
:1042800063256325632563204C5020256300583146
:104290002025632563256325632563256325632521
:1042A0006320202020200000454D455247454E43C5
:1042B000494120424F54414F00004150502020447A
:1042C0004953504F4E4956454C200000454D4552EC
:1042D00047454E43494120424F54414F0000202062
:1042E000202020202020202020202020202000000E
:1042F000454D455247454E43494120424F544F4E4C
:1043000000002020202020202020202020202020ED
:1043100020200000454D455247454E435920425507
:1043200054544F4E00002020202020202020202008
:1043300020202020202000004D414E4F504C412095
:1043400041434F504C41444100004445534C494780
:10435000415220502F5245534554000058312025DA
:104360006325632563256325632563256325632012
:104370004C502025630020504F5254412046454365
:1043800048414441202000002020494E54455254C9
:10439000524156414441202000002050554552547E
:1043A0004120434552524144412000002020494EC3
:1043B000544552545241564144412020000020208F
:1043C00020434C4F53454420444F4F52202000007F
:1043D000202020494E5445524C4F434B4544202009
:1043E000000020454E434F4445522052455155450B
:1043F000522000002020205245494E494349415255
:1044000020202020000020202020504F53534956C8
:10441000454C20202020000053455249414C204962
:104420004E5645525449444100002020202020206F
:10443000202020202020202020200000656D657293
:1044400067656E6369612020206C636400006261AF
:10445000206163696F6E61646F202020202000005E
:10446000414755415244414E444F204645434841FF
:10447000000054454D504F204645434841522025A9
:10448000334C75004553504552414E444F204345EF
:104490005252415200005449454D504F204345521D
:1044A0005241522025324C75000057414954494E23
:1044B0004720544F20434C4F5345000054494D452D
:1044C00020544F20434C4F53452025324C7500005B
:1044D00074656D706F2066656368616D656E746F7D
:1044E00000007469656D706F206465206369657292
:1044F000726500002020636C6F7365202074696D05
:104500006520200020202020202020202020202086
:1045100020202020000020202020202020202020DB
:1045200020202020202000002020202020202020CB
:104530002020202020202020000045422032345F0F
:10454000302056434F4445522020000056455253D8
:10455000414F202020202025730056455253494FBB
:104560004E202020202573004D4F544F5220534998
:10457000444520202020202000004C41444F202092
:104580004D4F544F522020202020000045535155BC
:104590004552444F20202020202020200000444964
:1045A000524549544F202020202020202020000068
:1045B000495A5155494552444F202020202020205F
:1045C00000004445524543484F2020202020202011
:1045D000202000004C454654202020202020202070
:1045E000202020200000524947485420202020202D
:1045F000202020202020000054494D45522020201A
:104600002020202020202020000054454D504F52D3
:10461000495A41444F52202020200000464543483B
:10462000415220454D2025324C75207365670000AE
:1046300043455252415220454E2025324C7520733D
:1046400065670000434C4F534520494E20202532DA
:104650004C752073656300004349434C4F5320441D
:104660004120504F5254412000004349434C4F5386
:10467000202020202025354C75004349434C4F53C2
:104680002044412050554552544100004349434C79
:104690004F53202020202025354C75002020204419
:1046A0004F4F52204359434C45532020000043595B
:1046B000434C4553202020202025354C7500504F79
:1046C000525441202020465245455A455220000070
:1046D00054494D4552204154495641444F202020D1
:1046E000000050554552544120465245455A4552C6
:1046F0002020000054494D45522041435449564121
:10470000444F202000002020465245455A45522063
:10471000444F4F522020000020202054494D455244
:10472000204F4E20202020200000504F5254412086
:104730002020465245455A455220000054494D45D7
:1047400052204445534154495641444F000050556E
:104750004552544120465245455A455220200000BA
:1047600054494D4552204E4F414354495641444FC0
:1047700000002020465245455A455220444F4F5292
:104780002020000020202054494D4552204F46460D
:10479000202020200000414A555354452020204C21
:1047A0004F4F50494E47000053454E534942202039
:1047B000202020202025322E306625250000204C88
:1047C0004F4F50494E472041444A55535420000012
:1047D00053454E5349542020202020202025322E9E
:1047E0003066252500002052454C4553205041207D
:1047F00065205046202000002020202041544956AA
:1048000041444F532020202000002052454C455366
:1048100020504120652050432020000020202020EF
:10482000414354495641444F532020200000205218
:10483000454C41595320444F20262044432000003A
:10484000202020202020204F4E202020202020200B
:104850000000494E5445522D424C4F5155454F2072
:1048600020200000202020204154495641444F2060
:10487000202020200000494E5445522D424C4F51DB
:1048800055454F202020000020202020414354493E
:104890005641444F202020200000202020494E5423
:1048A00045524C4F434B2020202000002020202048
:1048B00020204F4E202020202020202000002020DB
:1048C000202020204D4F444F202020202020000079
:1048D00020202020205341464554592020202020CC
:1048E00000002020202020204D4F444F2020202059
:1048F0002020000020202020204E4F524D414C20EF
:104900002020202000002020564D4F5445204D4FA0
:104910004442555320200000202020204154495675
:1049200041444F202020202000002020564D4F548D
:1049300045204D4F44425553202000002020202088
:1049400020204F4E2020202020202020000020204A
:104950002020202020202020202020202020000097
:104960002020202020202020202020202020202047
:1049700000000101C5530CE0010E006EC451016E30
:1049800004E0D8900036012EFCD7005082130DD0E1
:10499000010E006EC451016E04E0D8900036012E65
:1049A000FCD70050FF0A8217836B00011200D8B2B7
:1049B00004D0010EEA6ECF0EE96E006A016A026A47
:1049C000036A0101CF6BD06BD16BD26BCE51CD118D
:1049D000CC11CB112CE0200ED36FD890C737C8373D
:1049E000C937CA37CF37D037D137D237CE51D25D5A
:1049F00008E1CD51D15D05E1CC51D05D02E1CB5153
:104A0000CF5D0FE3CB51CF5FCC51D8A0CC3DD05F71
:104A1000CD51D8A0CD3DD15FCE51D8A0CE3DD25FF3
:104A2000D8800036013602360336D32FD6D7600041
:104A30003FF7EFFF600043F7ECFF600047F7ECFF44
:104A400060004BF7ECFF0001120000010101C46B94
:104A500002C1C5F100018DDF010E0101C46F00C16B
:104A6000C5F1000186DF020E0101C46FFEC0C5F171
:104A700000017FDF000ECAB2010E0101C36F030EF9
:104A8000C46FC3C1C5F1000174DF000ECAB4010ECA
:104A90000101C36F040EC46FC3C1C5F1000169DF1A
:104AA000000ECAB6010E0101C36F050EC46FC3C16B
:104AB000C5F100015EDF000ECAB8010E0101C36F2F
:104AC000060EC46FC3C1C5F1000153DF000ECABAA0
:104AD000010E0101C36F070EC46FC3C1C5F1000110
:104AE00048DF39019491C3C01DF1C2C01CF1000E12
:104AF000000188B5010E01011E6F1F6B000E000141
:104B000088B7010E0101206F216B0001AA5306E155
:104B1000AB5304E1AC5302E1AD5328E088A526D0A5
:104B2000AA51AE5D0101C36F0001AB51AF59010144
:104B3000C46F0001AC51B0590101C56F0001AD5106
:104B4000B1590101C66FD892CA6FC5C1C9F1C4C1BC
:104B5000C8F1C3C1C7F1CE6BCD6BCC6B0A0ECB6F66
:104B6000000125DF01C023F100C022F1000E010188
:104B700016B7010E246F256B000E16B9010E266FB5
:104B8000276BB7C029F1B6C028F1BBC02BF1BAC062
:104B90002AF1CCC02CF1CDC02DF1C76BCAC02EF1CB
:104BA0000001CBC02FF1010183C131F182C130F18D
:104BB000000E17BD010E010A179DE8B0178D000EFB
:104BC000000169B5010E010A6995E8B06985662B97
:104BD000D8B4672B67BF08D0675303E1665102085A
:104BE00003E2676B666BBB943C0EB16EB00EB06EA9
:104BF00000003901A4919481A49100013CEF10F0D0
:104C000000018E2B8E5109080AE2000E88B1010EB8
:104C1000010A8891E8B088818E6BDE2BDF2B010EB4
:104C2000AA27D8B0AB2BD8B4AC2BD8B4AD2BB1518C
:104C3000AD5D15E30BE1B051AC5D11E307E1AF51A0
:104C4000AB5D0DE303E1AA51AE5D09E2AD6BAC6B68
:104C5000AB6BAA6BB56BB46BB36B010EB26FE02B91
:104C60003C0EA56EB00EA46E00003901A69DA69D57
:104C700000013CEF10F00001CDB806D0CDAA04D061
:104C8000CCAE02D0010E956FCDB806D0CDBA04D00F
:104C9000CCBE02D0020E956FCDA806D0CDBA04D0FE
:104CA000CCAE02D0030E956FCDA806D0CDAA04D00D
:104CB000CCBE02D0040E956FCDA806D0CDAA04D0EC
:104CC000CCAE02D0050E956FCDB806D0CDBA04D0CB
:104CD000CCAE02D0060E956FCDB806D0CDAA04D0CA
:104CE000CCBE02D0070E956FCDA806D0CDBA04D0A9
:104CF000CCBE02D0080E956FCC9C0A0E0101C36F8A
:104D0000020EC325C46F000187BF95D0F05327E181
:104D1000B7AF03D0C3AF0CD002D0C3BF07D0B751D9
:104D2000C35D04E305E1C251B65D02E3CAA205D04A
:104D3000F4970101169700018885C3AF03D0B7AF80
:104D40000AD002D0B7BF0AD0C351B75D07E303E171
:104D5000B651C25D03E2CAB201D0889515D0B7AF93
:104D600003D0C3AF0AD002D0C3BF0DD0B751C35DCB
:104D70000AE303E1C251B65D06E2F497010116971A
:104D80000001888501D08895C3AF03D0BBAF0AD09E
:104D900002D0BBBF0FD0C351BB5D0CE303E1BA51DE
:104DA000C25D08E2010116A906D0169B169D169950
:104DB0000001888701010001BBAF03D0C3AF0AD057
:104DC00002D0C3BF0ED0BB51C35D0BE303E1C251A0
:104DD000BA5D07E2010116B702D0000102D000015E
:104DE0008897BDAF03D0C3AF0AD002D0C3BF0DD0E8
:104DF000BD51C35D0AE303E1C251BC5D06E201019E
:104E000016A702D0169D168B0001C3AF03D0C1AF09
:104E10000AD002D0C1BF0FD0C351C15D0CE303E182
:104E2000C051C25D08E2010116A904D016BB02D030
:104E3000168B168D0001010116B71ED016B91CD0B5
:104E40000001E06B6997C56BC46BC769C669010156
:104E5000126B169B169D0001C3AF03D0BBAF0AD0E7
:104E600002D0BBBF08D0C351BB5D05E303E1BA511B
:104E7000C25D01E28887010116A707D0000187AF54
:104E800002D0010102D00101169D16B702D016A969
:104E900024D0122B1251320807E21251340804E3D5
:104EA000C3C0C5F0C2C0C4F01251640807E2125179
:104EB000660804E3C3C0C7F0C2C0C6F01251C808F8
:104EC0000CE20001C451C65D05E1C551C75D02E1B8
:104ED000698701D069970101126BBA9C0C5301E1FB
:104EE000BA8CCAA00DD00001FF2BFF510101C35D98
:104EF00006E2010E0001FE6FC4C1FFF0010104D003
:104F00000001FE6BFF6B01010001F53D12D0CAB636
:104F10000AD001010D2B0D51C35D03E20C6BC4C11E
:104F20000DF105D00001010E01010C6F0D6B11D0C8
:104F30000001CAA60BD00101112B1151C35D04E27F
:104F4000010E106FC4C111F104D000010101106BFA
:104F5000116B0001E85322E1CBB819D00101032BFA
:104F60000351C35D12E2C4C103F1132BD8B4142B57
:104F7000145303E11351050807E2010E146FF50EF7
:104F8000136F010E026F01D0026B07D00001010EFA
:104F90000101026F036B146B136B0001E83D11D02C
:104FA000CBB80AD00101032B0351C35D03E2026BAE
:104FB000C4C103F105D00001010E0101026F036BB2
:104FC0000001CBBA0AD00101012B0151C35D03E2FC
:104FD000006BC4C101F105D00001010E0101006F99
:104FE000016B0001F53D12D0010E01010E6FCAB434
:104FF00008D0052B0551C35D03E2046BC4C105F164
:1050000003D0010E046F056B11D00001010E0101E8
:10501000046FCAB408D00F2B0F51C35D03E20E6BAF
:10502000C4C10FF103D0010E0E6F0F6BCAA223D0C3
:1050300016A921D00001C3AF03D0BDAF12D004D058
:10504000BDAF02D0010117D0C351BD5DD8B002D0B1
:10505000010111D006E1BC51C25DD8A002D001010E
:105060000AD00101072B0751010804E2010E066F67
:10507000030E076F02D0066B076B0001C851BA25FB
:10508000016EC951BB21036E015003AE03D0C3AF03
:105090000AD002D0C3BF14D00350C35D11E303E1B3
:1050A000C251015C0DE2CAA80BD00101092B0951C4
:1050B000010804E2010E086F030E096F04D000011D
:1050C0000101086B096BCAAA09D00B2B0B5101080F
:1050D00004E2010E0A6F030E0B6F02D00A6B0B6B1A
:1050E0000001FE2D01D069D0F53D67D0F1534DE1AF
:1050F000010116910001F4AF03D0010116810001F6
:10510000F23D11D001011693000188A503D00101E1
:105110001683000101011695000188A703D0010143
:105120001685000131D0010116A703D00001888F38
:105130000101000169AB07D0010116B902D00001DD
:1051400002D00001F48188AF0ED088A50CD0F32BDB
:10515000010116830001F351320805E2889F010125
:1051600016930001F36BF4A10FD088A70DD0F32B99
:10517000010116850001F351320806E2F491699BA2
:10518000010116950001F36B18D001011691000181
:10519000F4AF03D001011681000101011693000153
:1051A000F4AF03D00101168300010101169500013F
:1051B000F4AF03D0010116850001F53D05D0EF3DA8
:1051C00001D002D0F489F49B0101025309E10001EE
:1051D000EF3D03D0010104D00001F48BF4990101EB
:1051E000025308E10001EF3D02D0010103D00101AB
:1051F00016B90FD0005310E10001F53D01D002D0E7
:1052000001010AD0EF3D02D0010106D0010116A92B
:1052100003D00001F48D01010001F55355E1FE5367
:105220001CE101011053D8B402D0000116D006537E
:10523000D8B402D0000111D00853D8B402D0000174
:105240000CD00A53D8B402D0000107D017A302D063
:10525000000103D017A503D000010101169F000132
:10526000FE531FE101011053D8B402D0000119D040
:105270000653D8B402D0000114D00853D8B402D0D9
:1052800000010FD00A53D8B402D000010AD017A3EE
:1052900002D0000106D017A502D0000102D0168F5F
:1052A0000001FE5304E10101105303E0000101017C
:1052B00017910001FE5308E101011053D8B402D048
:1052C000000102D017810001F63D2ED0F53D0FD030
:1052D000BE90F4BFBE80BE92010116B1BE82BE94E4
:1052E00016B3BE84BA9E16B5BA8E10D00001BE9019
:1052F000010117B1BE80BE9216BFBE82BE940001EE
:1053000088B5BE84BA9E88B7BA8E0101BC9616B71E
:10531000BC86BC9416B9BC84BC9216BBBC82BC9043
:1053200016BDBC802AD00001F53D09D0BE90010118
:1053300016B3BE80BE9216B5BE820DD00001BE90DF
:10534000010116BFBE80006A16BF002A010E001AB6
:10535000BE9200B0BE82BE9416B7BE84BA9E16B985
:10536000BA8EBC9616B7BC86BC9416B9BC84BC92E7
:1053700016BBBC82BC9016BDBC800001F55300E199
:105380003C0E996EB00E986E00003901A89D000188
:105390003CEF10F00001CC8C3D01E1B71BD0E1B334
:1053A00019D0E1AD08D06F0040F794F00001889D5E
:1053B000879B05D03D016F0040F7A9F00001A9C00F
:1053C000C3F094C0C2F088B903D0FF0EC21BC31B48
:1053D00003D03D01E1930001E06B3D01D051390163
:1053E000A69500013CEF10F000016983B8A802D037
:1053F000CF0EB76E2C0EB66E3901A39F00013CEFA5
:1054000010F03901A3A7FED73D01F9511A6EE851FA
:10541000016E1AA204D0F299F783F993F289000180
:1054200014EF2AF00001EDD701C0C3F1625315E17A
:1054300061513F0812E362C003F06151612BD8B49F
:10544000622B0101C46F210EC425E96E000E0320FA
:10545000EA6E60000FF7EFFF0001646B636B3901C8
:10546000A39700013CEF10F0202020444554454311
:1054700054414E444F20202000002020204C4F4F0C
:1054800050494E47202E2E2E2E2E00002020202068
:105490004C4F4F50494E4720202020200000202014
:1054A00020204445544543544544202020200000FA
:1054B000202020204C4F4F50494E472020202020B4
:1054C00000002020202050524553454E54452020B6
:1054D00020200000202020204C4F4F50494E4720D4
:1054E00020202020000020204E4F542044455445C9
:1054F0004354454420200000202020204C4F4F5092
:10550000494E472020202020000020202020415507
:1055100053454E544520202020200000444947494F
:105520004C494E4B202050524F4E544F00004D419D
:105530004320253032582530325825303258253016
:1055400032582530325825303258000044494749F6
:105550004C494E4B20415553454E544500004D415A
:10556000435F5F5F5F5F5F5F5F5F5F5F5F5F000025
:10557000564D4F5445202050524F4E544F2020201E
:1055800000004D4143202530325825303258253017
:1055900032582530325825303258253032580000E4
:1055A000564D4F544520415553454E5445202020DB
:1055B00000004D41435F5F5F5F5F5F5F5F5F5F5F05
:1055C0002020000020504F5254412020464543489F
:1055D0004144412000004349434C4F532025394C5E
:1055E0007500205055455254412043455252414484
:1055F000412000004349434C4F532025394C75004E
:105600002020434C4F53454420444F4F52202020EC
:1056100000004359434C45532025394C7500205018
:105620004F52544120204645434841444120000008
:105630004349434C4F532025394C75002050554564
:1056400052544120434552524144412000004349B5
:10565000434C4F532025394C75002020434C4F5369
:10566000454420444F4F5220202000004359434CD2
:1056700045532025394C7500504F52544120464522
:10568000434841444125334C75004349434C4F53F3
:105690002025394C750050554552544143455252CE
:1056A00041444125334C75004349434C4F53202519
:1056B000394C7500444F4F5220434C4F53454420C2
:1056C0002025334C75004359434C45532025394C14
:1056D00075005831202563256325632563256325DF
:1056E0006325632563204C5020256300202020552E
:1056F0005341522042462020000020202050415299
:10570000412052455345544152200000202020554D
:105710005341522042462020000020202050415278
:1057200041205245534554415220000020205553FA
:105730004152202042412020202020200000202013
:10574000504152412046454348415220202000000C
:10575000583120256325632563256325632563254B
:10576000632563204C502025630058312025632594
:1057700063256325632563256325632563204C50DA
:10578000202563004359434C45532025394C75006F
:105790004349434C4F532025394C7500583120253F
:1057A00063256325632563256325632563256320BE
:1057B0004C502025630020504F5254412020464534
:1057C00043484144412000004349434C4F53202566
:1057D000394C750020505545525441204345525292
:1057E0004144412000004349434C4F532025394C4C
:1057F00075002020434C4F53454420444F4F5220C6
:10580000202000004359434C45532025394C750056
:10581000583120256325632563256325632563258A
:10582000632563204C50202563002020454E5452B0
:105830004541424552544120202000004349434CF9
:105840004F532025394C75002020454E5452454178
:1058500042494552544F202000004349434C4F5386
:105860002025394C7500202020444F4F5220414ABA
:1058700041522020202000004359434C455320250D
:10588000394C750058312025632563256325632530
:1058900063256325632563204C5020256300205039
:1058A0004F5254412020414252494E444F20000063
:1058B0005055455254412041425249454E444F2093
:1058C00000002020444F4F52204F50454E494E4734
:1058D00020200000524544555A2020204142455284
:1058E00054555241000052454455434952204150BD
:1058F00045525455524100002020534C4F57204FE1
:1059000050454E494E472020000058312025632540
:1059100063256325632563256325632563204C5038
:105920002025630020504F525441204645434841B2
:105930004E444F200000505545525441204345529B
:1059400052414E444F2000002020444F4F522043EC
:105950004C4F53494E4720200000524544555A2091
:1059600046454348414D454E544F0000524544552D
:10597000434520454E2043494552524500002020D2
:10598000534C4F5720434C4F53494E472020000063
:105990004552524F2032202020202020434F4D4D91
:1059A0000000434F4E53554C544152204D414E55EB
:1059B000414C00004552524F203120202020202011
:1059C000434F4D4D0000434F4E53554C54415220D0
:1059D0004D414E55414C00004552524F203220203F
:1059E00020202020434F4D4D0000434F4E53554C37
:1059F000544152204D414E55414C00006F0048FF2C
:105A000091F1D29E3901E16B0F0EE06FE59DE59FAC
:105A1000E581E351E59DE58F010191BFD28E000143
:105A2000906F6F0048FF91F1D29E3901E16B100E2B
:105A3000E06FE59DE59FE581E351E59DE58F01017F
:105A400091BFD28E0001916F6F0048FF91F1D29EFD
:105A50003901E16B110EE06FE59DE59FE581E351B2
:105A6000E59DE58F010191BFD28E0001926F6F001D
:105A700048FF91F1D29E3901E16B120EE06FE59D76
:105A8000E59FE581E351E59DE58F010191BFD28E50
:105A90000001936F93C0CDF092C0CCF091C0CBF0D9
:105AA00090C0CAF0BDEF6AF00101A9B102D0BD9665
:105AB00001D0BD86C596A9B302D0BD9401D0BD84E6
:105AC000C594A9B502D0BD9201D0BD82C592A9B737
:105AD00002D0BD9001D0BD80C5900000C498BC88A4
:105AE0000400020E006E002EFED7C498BC98000180
:105AF0001200C49ABC9A04004F0E006E002EFED70E
:105B000000000101A65303E0C49ABC8A02D0C49AE3
:105B1000BC9A0000C498BC98A739A86F0F0EA817AC
:105B2000A8C1A9F10001C0DF0101A7510F0BA86FA7
:105B3000A96F0001B9DF1200010EEA6EA50EE96E31
:105B4000EF5011E0050E016EBF0E006E0400002E36
:105B5000FDD7012EF9D72E0E006E002EFED70000C5
:105B60000400EF2EEFD712000101A32D01D003D0C6
:105B7000400EA46F01D0A46B010EA25DA427A45116
:105B80008009A56FA66BA76F0001B3DF12000101AA
:105B9000A1510C0A000107E0060A11E0070A17E00C
:105BA000050A1CE022D00101A66B010EA76F0001BF
:105BB000A0DF020E0101A56F0001BEDF1DD0010EA6
:105BC0000101A26F020EA36F0001CEDF15D0010EFE
:105BD0000101A26FA36F0001C7DF0ED00101A66B08
:105BE000100EA76F000185DF07D0010E0101A66F1F
:105BF000A1C1A7F100017DDF12000C0E0101A16F10
:105C00000001C5DF1200C49ABC9AC498BC980F0E5C
:105C10000101A56F000190DF0101916B9151020814
:105C20000CE3030EA96F00013FDF050E0101A56F14
:105C3000000182DF0101912BF1D7020EA96F000153
:105C400033DF0101916B915103080EE3036A915117
:105C500000014FEC10F00101926FA66BA76F0001DD
:105C600048DF0101912BEFD7000112000101925191
:105C700094036F00CCFF01F06F00D0FF00F095039C
:105C8000F350002693519403F3500020026E00015C
:105C900012008E0E006E94C101F093C102F0036AEF
:105CA000015209E102C001F0026A080E005E0152D1
:105CB00002E1006A08D0D89001BE04D00236013655
:105CC0000006F9D7019E120001019351D8B4A5D066
:105CD0009F6F9751D8B4A1D09F5F05E37F0E9F2798
:105CE000D8B09BD006D0810E9F5FD8A096D0D8B4F4
:105CF00094D09FC100F0016A026A036A9E6B94C14E
:105D00009DF19D8F95C19CF196C19BF1190E9F6FDE
:105D10009A519B5F0DE2010E9C5F0AE29D5F08E2D3
:105D20009E5F06E29E2B9D2B9C2B9A519B2728D091
:105D300099519C5F12E2010E9D5F0FE29E5F0DE2A2
:105D40009E2B9D2B99519C279A519B2719E39C2BA5
:105D500017E19D2B15E19E2B13D0985180099D5F73
:105D60000EE2010E9E5F0BE29E2B985180099D274B
:105D700099519C27E9E39D2BE7E19E2BE5D7038012
:105D80009F2F01D00BD0D8909B379C379D379E37E3
:105D9000D890033602360136A037BAD7A0A106D074
:105DA000D890013202320332A03302D0000635E02F
:105DB000A0BF1ED0D8909B379C379D379E379A51F5
:105DC0009B5F07E2010E9C5F04E29D5F02E29E5F23
:105DD0001AE399519C5F05E2010E9D5F02E29E5F0E
:105DE00012E3985180099D5F03E2010E9E5F0BE371
:105DF000032A09E1022A07E1012A05E1002A0DE050
:105E000001320232033294C19FF198519F1B9FAF20
:105E100002D0018E06D0019E04D0006A016A026A97
:105E2000036A0001C7EF2FF001019E51D8B474D06E
:105E3000006EA251D8B470D0002604E3810E002673
:105E40006BE204D07F0E005E67E366E09FC1A6F1BF
:105E5000A351A61B9F8FA38FA151A5036F00D0FF55
:105E6000A8F1A051A4036F00D0FF03F06F00CCFF96
:105E7000A7F1A503F350A827F450A723000E03228F
:105E8000A151A403F350A827F450A723000E026ADF
:105E9000032202229F51A503F350A727F4500322A7
:105EA000000E02229F51A403F3500326F450022255
:105EB000000E016A0122A151A303F350A727F45059
:105EC0000322000E02220122A051A303F350032655
:105ED000F4500222000E01229F51A303F350022628
:105EE000F4500122002A01BE05D0A737033602363E
:105EF00001360006000EA7AF0AD0032A02220122B3
:105F0000015005E1025003E1035001E1002AA6BF60
:105F1000018EA6AF019E04D0006A016A026A036A7C
:105F2000000112008E0E006E01019351005E94C1BB
:105F300002F095C101F0028E005209E0D8900252A1
:105F400002E1015204E002320132002EF7D794AF91
:105F500005D0011E021E012AD8B4022A0001F6EF64
:105F60002FF092C194F191C193F193DE03C096F1A9
:105F700002C095F101C094F100C093F101019A6B48
:105F8000996B480E986F850E976F00019DD603C0E0
:105F9000D2F002C0D1F001C0D0F000C0CFF0BA51B1
:105FA000B65D006EBB51B75900C0D3F0D46FD4C0FA
:105FB00094F1D3C093F16DDE03C0A1F102C0A0F152
:105FC00001C09FF100C09EF1D2C0A5F1D1C0A4F1E3
:105FD000D0C0A3F1CFC0A2F127DF03C096F102C069
:105FE00095F101C094F100C093F19CD702C0D4F0A8
:105FF00001C0D3F0D3C001F0D4C002F012000A0EE9
:106000000101A56F000198DD010E0101A26FA36FD0
:106010000001AADD12000900F55211E06F00D8FF5F
:1060200095F16F00DCFF96F16F00D4FFA1F1AFDDB9
:10603000600057F6F6FF60005BF6F7FFECD7120042
:106040000A0E0101A56F000177DD010E0101A26FAB
:10605000020EA36F000188DD1200C39CBB9C080EDA
:10606000016E00D00000018E10D0019E010191331D
:106070000001D8B0BB8CD8A0BB9C018C06D0019C81
:10608000012EF4D700D00000BB8C840EE96EE92EFF
:10609000FED700D0000001BEE8D701BCF0D7120047
:1060A0000B0EA56EDC0EA46E000096C1ADF095C17E
:1060B000ACF094C1ABF093C1AAF09AC1B1F099C110
:1060C000B0F098C1AFF097C1AEF0B56BB46BB36BE5
:1060D000B26B39015B5104000001120095510508B3
:1060E00044E0A82D35D0D93D07D089DF640EF66E87
:1060F000290EF76E90DF12D0D95307E180DF760EBC
:10610000F66E290EF76E87DF09D0D9517F0806E1B8
:1061100076DF880EF66E290EF76E7DDFD93D06D04C
:106120008FDF9A0EF66E290EF76E75DFD95306E1F2
:1061300087DFAC0EF66E290EF76E6DDFD9517F0842
:1061400006E17EDFBE0EF66E290EF76E64DF0CD020
:1061500056DFD00EF66E290EF76E5DDF71DFE20EB0
:10616000F66E290EF76E57DFB9D7120009006F00DF
:10617000D8FF96F16F00DCFF97F16F00D4FFA1F11B
:1061800006DD60005BF6F6FF60005FF6F7FF0101D9
:10619000952F01D002D00001E9D7000112000101C2
:1061A0009551016A945D03E294C100F00CD0006A3D
:1061B000080E966F943700369551005CD8B0006E8B
:1061C0000136962FF7D700011200015092C194F1C9
:1061D000640E0101956F0001E2DF00C092F10150F1
:1061E000300E08E1010193A30FD093B70DD093B9FE
:1061F000200E04D00101939793999381012601C049
:10620000A1F10001C4DC010192C194F10A0E956F65
:106210000001C5DF00C092F10150300E08E101011C
:1062200093B70AD093A108D093B9200E000101269C
:1062300001C0A1F1ACDC0101300E922792C1A1F1A5
:106240000001A5DC12004ADFF96BFA6B01019191A4
:10625000000195510308D8B46FD0D1DE780EF66EE8
:10626000260EF76ED8DEECDE8A0EF66E260EF76E80
:10627000D2DE952D2CD0C3DE9C0EF66E260EF76E68
:10628000CADEDEDEAE0EF66E260EF76EC4DE6F00E0
:1062900048FF92F1D29E3901E16B330EE06FE59D2C
:1062A000E59FE581E351E59DE58F010192BFD28E27
:1062B0000001FD6F01019181080E926FFA0EA56F2A
:1062C00000013ADC0101922FF9D7000135D0955138
:1062D000040831E194DEC00EF66E260EF76E9BDEEA
:1062E000AFDED20EF66E260EF76E95DEFD69D25049
:1062F000006ED29E3901E16B330EE06F6000F7F360
:10630000E3F9E59DE59FE585550EE66FAA0EE66F7C
:10631000E583E5B3FED7E595E59DE58F0050D21204
:10632000080E0101926FFA0EA56F000105DC010154
:10633000922FF9D700018DD7010191A19BD00001C7
:106340005EDEE40EF66E260EF76E090E0101956F05
:1063500000010CDFFDC092F1130E0101936F0001EB
:1063600034DFF00EF66E260EF76E040E0101956F07
:106370000001FCDE65DEF60EF66E260EF76E4BDED5
:10638000640E0101A56F00019CEC2DF095510408ED
:1063900001E1FD2B640E0101A56F00019CEC2DF0C5
:1063A000952D01D0FD079551030862E1FF0EFD1BFD
:1063B000D250006ED29E3901E16B330EE06F600067
:1063C000F7F3E3F9E59DE59FE585550EE66FAA0E27
:1063D000E66FE583E5B3FED7E595E59DE58F0050D3
:1063E000D2120400840E006E002EFED700D06F0083
:1063F00048FF92F1D29EE16B330EE06FE59DE59F81
:10640000E581E351E59DE58F010192BFD28E000148
:10641000FD6FFF0EFD1BF3DD080EF66E270EF76E07
:10642000090E0101956F0001A1DEFDC092F1130E6E
:106430000101936F0001C9DE140EF66E270EF76E90
:10644000040E0101956F000191DEFADD1A0EF66E61
:10645000270EF76EE0DD080E0101926FFA0EA56FB0
:1064600000019CEC2DF00101922FF8D791910001D1
:1064700063D701010001A3EF3EF030DEF96BFA6B48
:1064800095510308D8B476D0BADD8C0EF66E280E7E
:10649000F76EC1DDD5DD9E0EF66E280EF76EBBDD04
:1064A000952D32D0ACDDB00EF66E280EF76EB3DD52
:1064B000C7DDC20EF66E280EF76EADDDF66BD2505C
:1064C000006ED29E3901E16B370EE06F6000DBF3A6
:1064D000E3F9E59DE59FE585550EE66FAA0EE66FAB
:1064E000E583E5B3FED7E595E59DE58F0050D21233
:1064F000080E0101916FFA0EA56F00019CEC2DF0C2
:106500000101912FF8D700019551040832E177DDA0
:10651000D40EF66E280EF76E7EDD92DDE60EF66E78
:10652000280EF76E78DDF669D250006ED29E3901E2
:10653000E16B370EE06F6000DBF3E3F9E59DE59F6B
:10654000E585550EE66FAA0EE66FE583E5B3FED747
:10655000E595E59DE58F0050D212080E0101916F7F
:10656000FA0EA56F00019CEC2DF00101912FF8D7D8
:10657000000186D7AAEF3EF0B1DDF96BFA6B01019D
:106580009191000195510308D8B471D038DDC40E43
:10659000F66E250EF76E3FDD53DDD60EF66E250E38
:1065A000F76E39DD952D2DD02ADDE80EF66E250E1D
:1065B000F76E31DD45DDFA0EF66E250EF76E2BDD3A
:1065C0006F0048FF92F1D29E3901E16B320EE06F0D
:1065D000E59DE59FE581E351E59DE58F010192BFD2
:1065E000D28E0001FB6F01019181080E926FFA0EAD
:1065F000A56F00019CEC2DF00101922FF8D700014E
:1066000036D09551040832E1FADC0C0EF66E260EF7
:10661000F76E01DD15DD1E0EF66E260EF76EFBDC45
:10662000FB69D250006ED29E3901E16B320EE06FF1
:106630006000EFF3E3F9E59DE59FE585550EE66F14
:10664000AA0EE66FE583E5B3FED7E595E59DE58FF8
:106650000050D212080E0101926FFA0EA56F0001D0
:106660009CEC2DF00101922FF8D700018BD701018E
:1066700091A185D00001C3DC300EF66E260EF76EB8
:106680000D0E0101956F000171DDFBC092F1130E3B
:106690000101936F000199DDD3DC420EF66E260EE8
:1066A000F76EB9DC640E0101A56F00019CEC2DF0C2
:1066B0009551040801E1FB2B640E0101A56F000157
:1066C0009CEC2DF0952D01D0FB079551030855E169
:1066D000D250006ED29E3901E16B320EE06F600045
:1066E000EFF3E3F9E59DE59FE585550EE66FAA0E0C
:1066F000E66FE583E5B3FED7E595E59DE58F0050B0
:10670000D2120400840E006E002EFED700D06F005F
:1067100048FF92F1D29EE16B320EE06FE59DE59F5E
:10672000E581E351E59DE58F010192BFD28E000125
:10673000FB6F65DC540EF66E260EF76E0D0E010132
:10674000956F000113DDFBC092F1130E0101936FF1
:1067500000013BDD75DC660EF66E260EF76E5BDC27
:10676000080E0101926FFA0EA56F00019CEC2DF04E
:106770000101922FF8D79191000179D70101000111
:10678000B1EF3EF0ABDCF96BFA6B95510308D8B46E
:1067900079D035DC580EF66E250EF76E3CDC50DCF9
:1067A0006A0EF66E250EF76E36DC952D32D027DC9C
:1067B0007C0EF66E250EF76E2EDC42DC8E0EF66E2B
:1067C000250EF76E28DCEF6BD250006ED29E390199
:1067D000E16B310EE06F6000BFF3E3F9E59DE59FEB
:1067E000E585550EE66FAA0EE66FE583E5B3FED7A5
:1067F000E595E59DE58F0050D212080E0101916FDD
:10680000FA0EA56F00019CEC2DF00101912FF8D735
:1068100000019551040835E1FFEC2FF0A00EF66E53
:10682000250EF76E0BEC30F00BDCB20EF66E250E7B
:10683000F76E0BEC30F0EF69D250006ED29E39014A
:10684000E16B310EE06F6000BFF3E3F9E59DE59F7A
:10685000E585550EE66FAA0EE66FE583E5B3FED734
:10686000E595E59DE58F0050D212080E0101916F6C
:10687000FA0EA56F00019CEC2DF00101912FF8D7C5
:10688000000183D7B8EF3EF029DCF96BFA6B955124
:106890000308D8B482D0FFEC2FF02C0EF66E270E32
:1068A000F76E0BEC30F020EC30F03E0EF66E270E5B
:1068B000F76E0BEC30F0952D36D0FFEC2FF0500E2C
:1068C000F66E270EF76E0BEC30F020EC30F0620E17
:1068D000F66E270EF76E0BEC30F0F16BD250006EB7
:1068E000D29E3901E16B2F0EE06F6000C7F3E3F930
:1068F000E59DE59FE585550EE66FAA0EE66FE583FB
:10690000E5B3FED7E595E59DE58F0050D212080E60
:106910000101916FFA0EA56F00019CEC2DF00101B1
:10692000912FF8D700019551040836E1FFEC2FF0C4
:10693000740EF66E270EF76E0BEC30F020EC30F094
:10694000860EF66E270EF76E0BEC30F0F169D25022
:10695000006ED29E3901E16B2F0EE06F6000C7F32D
:10696000E3F9E59DE59FE585550EE66FAA0EE66F16
:10697000E583E5B3FED7E595E59DE58F0050D2129E
:10698000080E0101916FFA0EA56F00019CEC2DF02D
:106990000101912FF8D700017AD7BFEF3EF06EECDE
:1069A00030F0F96BFA6B95510308D8B482D0FFEC44
:1069B0002FF0980EF66E270EF76E0BEC30F020ECF1
:1069C00030F0AA0EF66E270EF76E0BEC30F0952D18
:1069D00036D0FFEC2FF0BC0EF66E270EF76E0BECE8
:1069E00030F020EC30F0CE0EF66E270EF76E0BEC8A
:1069F00030F0F26BD250006ED29E3901E16B380E4E
:106A0000E06F6000CBF3E3F9E59DE59FE585550E6A
:106A1000E66FAA0EE66FE583E5B3FED7E595E59D43
:106A2000E58F0050D212080E0101916FFA0EA56F8A
:106A300000019CEC2DF00101912FF8D70001955138
:106A4000040836E1FFEC2FF0E00EF66E270EF76E2D
:106A50000BEC30F020EC30F0F20EF66E270EF76EF5
:106A60000BEC30F0F269D250006ED29E3901E16B2E
:106A7000380EE06F6000CBF3E3F9E59DE59FE58517
:106A8000550EE66FAA0EE66FE583E5B3FED7E595F2
:106A9000E59DE58F0050D212080E0101916FFA0EAC
:106AA000A56F00019CEC2DF00101912FF8D700019A
:106AB0007AD7C6EF3EF06F00A8FF99F16F00A4FFF0
:106AC00098F1010192AF08D0988F98A9982B911F47
:106AD000921F912BD8B4922B9239F009946F94277E
:106AE000E20F956F320F976F92510F0B95279527F5
:106AF0009727E90F966F9627962791390F0B9627C0
:106B0000972796379737971F973791510F0B9727EE
:106B10009437070E936F0A0E96079727FDE39507A4
:106B20009627FDE394079527FDE393079427FDE35C
:106B3000010EEA6E930EE96E070E9815989DED52C0
:106B4000981507E198B9EE5298B903D0200E006E5F
:106B500020D0E926000EEA22E950970803E1EA2C4A
:106B600001D0988DEF50006E08E198BD06D098B91D
:106B700022D098B702D0200E0BD098AF06D02D0EA1
:106B8000006EED50989D989F04D098879899300E8C
:106B900000266F00A8FF92F16F00A4FF91F100C0E2
:106BA000A1F10001C7EC2DF060004BF6EAFF600098
:106BB00047F6E9FF0101EE5098ADCED70001120073
:106BC000966BCAB0962B976BCBBA972B986BCBB8BA
:106BD000982B996BCAB4992B9A6BCAB29A2B9B6B60
:106BE000CAB89B2B9C6BCABA9C2B9D6BCAB69D2BBB
:106BF0009D51800DF3500101916F00019C51400D9A
:106C0000F3500101912700019B51200DF350010128
:106C1000912700019A51100DF350010191270001B5
:106C20009951080DF3500101912700019851040D6D
:106C3000F35001019127D89000019735010191256A
:106C400000019625A76F8AEF36F0C80E0101A56FE7
:106C500000019CEC2DF0010ECD6EC80E0101A56F58
:106C600000019CEC2DF0020ECD6EC80E0101A56F47
:106C700000019CEC2DF0040ECD6EC80E0101A56F35
:106C800000019CEC2DF0080ECD6EC80E0101A56F21
:106C900000019CEC2DF0100ECD6EC80E0101A56F09
:106CA00000019CEC2DF0200ECD6EC80E0101A56FE9
:106CB00000019CEC2DF0CD6A1200C00ED2123901F9
:106CC00093870001FFEC2FF0F40EF66E220EF76EA4
:106CD0000A0E0101956F0001B6EC30F0000EE96E6E
:106CE000C3C092F1C2C091F1E6DE20EC30F0040E98
:106CF000F66E230EF76E0D0E0101956F0001B6ECD6
:106D000030F095C092F1030E0101936F0001E5ECA4
:106D100030F056D7A751FE0A0FE0030A0FE0060A2B
:106D20000FE00C0A0FE0180A0FE0300A0FE0600ACB
:106D30000FE0C00A0FE010D088DF0FD086DF0DD043
:106D400084DF0BD082DF09D080DF07D07EDF05D063
:106D50007CDF03D07ADF01D0CD6AB4D7CDEF3EF02F
:106D6000CD6BCC6BCB6BCA6B878DCAC090F0CBC0A0
:106D700091F0CCC092F0CDC093F0D250006ED29E74
:106D80003901E16B0F0EE06F600043F2E3F9E59D1E
:106D9000E59FE585550EE66FAA0EE66FE583E5B340
:106DA000FED7E595E59DE58F0050D212D250006EDA
:106DB000D29EE16B100EE06F600047F2E3F9E59DB3
:106DC000E59FE585550EE66FAA0EE66FE583E5B310
:106DD000FED7E595E59DE58F0050D212D250006EAA
:106DE000D29EE16B110EE06F60004BF2E3F9E59D7E
:106DF000E59FE585550EE66FAA0EE66FE583E5B3E0
:106E0000FED7E595E59DE58F0050D212D250006E79
:106E1000D29EE16B120EE06F60004FF2E3F9E59D48
:106E2000E59FE585550EE66FAA0EE66FE583E5B3AF
:106E3000FED7E595E59DE58F0050D2126F0048FF23
:106E400095F1D29EE16B0F0EE06FE59DE59FE58128
:106E5000E351E59DE58F010195BFD28E0001906F52
:106E60006F0048FF95F1D29E3901E16B100EE06F83
:106E7000E59DE59FE581E351E59DE58F010195BF26
:106E8000D28E0001916F6F0048FF95F1D29E3901BB
:106E9000E16B110EE06FE59DE59FE581E351E59D16
:106EA000E58F010195BFD28E0001926F6F0048FF00
:106EB00095F1D29E3901E16B120EE06FE59DE59FE1
:106EC000E581E351E59DE58F010195BFD28E00017B
:106ED000936F93C0CDF092C0CCF091C0CBF090C036
:106EE000CAF077EF38F08889000E88B9010E0101E9
:106EF000956FD250006ED29E3901E16B140EE06F97
:106F0000600057F6E3F9E59DE59FE585550EE66FD0
:106F1000AA0EE66FE583E5B3FED7E595E59DE58F1F
:106F20000050D212050E0001CE6FD250006ED29EDC
:106F30003901E16B050EE06F60003BF3E3F9E59D7D
:106F4000E59FE585550EE66FAA0EE66FE583E5B38E
:106F5000FED7E595E59DE58F0050D212050E0101A3
:106F6000926F140E916F91C195F1D250006ED29E26
:106F70003901E16B060EE06F600047F6E3F9E59D2D
:106F8000E59FE585550EE66FAA0EE66FE583E5B34E
:106F9000FED7E595E59DE58F0050D21292C195F19F
:106FA000D250006ED29EE16B070EE06F60004BF690
:106FB000E3F9E59DE59FE585550EE66FAA0EE66FC0
:106FC000E583E5B3FED7E595E59DE58F0050D21248
:106FD000FE0E0101946FD40E936F93C195F1D250C0
:106FE000006ED29E3901E16B080EE06F60004FF633
:106FF000E3F9E59DE59FE585550EE66FAA0EE66F80
:10700000E583E5B3FED7E595E59DE58F0050D21207
:1070100094C195F1D250006ED29EE16B090EE06FE3
:10702000600053F6E3F9E59DE59FE585550EE66FB3
:10703000AA0EE66FE583E5B3FED7E595E59DE58FFE
:107040000050D2120001E869D250006ED29E390180
:10705000E16B150EE06F6000A3F3E3F9E59DE59F9A
:10706000E585550EE66FAA0EE66FE583E5B3FED71C
:10707000E595E59DE58F0050D212140E0001F76FE3
:10708000D250006ED29E3901E16B0D0EE06F6000B0
:10709000DFF3E3F9E59DE59FE585550EE66FAA0E62
:1070A000E66FE583E5B3FED7E595E59DE58F0050F6
:1070B000D212140E0001F86FD250006ED29E390128
:1070C000E16B0B0EE06F6000E3F3E3F9E59DE59FF4
:1070D000E585550EE66FAA0EE66FE583E5B3FED7AC
:1070E000E595E59DE58F0050D212000139D6FFEC01
:1070F0002FF0160EF66E230EF76E0BEC30F020EC30
:1071000030F0280EF66E230EF76E0BEC30F0080E02
:107110000101956FFA0EA56F00019CEC2DF00101A5
:10712000952FF8D70001D4EF3EF06EEC30F0F96BFC
:10713000FA6B6EEC30F095510308D8B4B1D0FFEC87
:107140002FF0040EF66E280EF76E0BEC30F020ECEC
:1071500030F0160EF66E280EF76E0BEC30F0878FBF
:10716000952D7DD0BA51C25D006EBB51C35900C090
:10717000C8F0C96FFFEC2FF0280EF66E280EF76EE0
:10718000090E0101956F0001B6EC30F0000EE96EBA
:10719000C3C092F1C2C091F18EDC20EC30F0360E0B
:1071A000F66E280EF76E090E0101956F0001B6EC20
:1071B00030F0000EE96EBBC092F1BAC091F17BDCF9
:1071C000600023F3E3F9D250006ED29E3901E16BE7
:1071D000390EE06FE59DE59FE585550EE66FAA0E39
:1071E000E66FE583E5B3FED7E595E59DE58F0050B5
:1071F000D212600027F3E3F9D250006ED29EE16B09
:107200003A0EE06FE59DE59FE585550EE66FAA0E07
:10721000E66FE583E5B3FED7E595E59DE58F005084
:10722000D2120001FFEC2FF0440EF66E280EF76E1E
:107230000BEC30F020EC30F0560EF66E280EF76EA8
:107240000BEC30F0080E0101916FFA0EA56F0001F2
:107250009CEC2DF00101912FF8D7000121D0955120
:1072600004081DE1FFEC2FF0680EF66E280EF76E95
:107270000BEC30F020EC30F07A0EF66E280EF76E44
:107280000BEC30F0080E0101916FFA0EA56F0001B2
:107290009CEC2DF00101912FF8D7000101D04BD7C4
:1072A000DCEF3EF001019E51B6089E6F036A9FC15C
:1072B000A2F19F8FD8909F33A033A13303320232C3
:1072C000013200329E2FF6D7A2AF0BD0001E011E56
:1072D000021E031E002AD8B4012AD8B4022AD8B448
:1072E000032A0001A0EF39F0E9500101966F955192
:1072F000986F1CE094C1A1F193C1A0F192C19FF1DC
:1073000091C19EF1A56BA46B200EA36F820EA26F9C
:10731000000114EC2FF003C094F102C093F101C0FE
:1073200092F100C091F10101982FE4D794C1A1F12D
:1073300093C1A0F192C19FF191C19EF10001B2D71A
:1073400003C094F102C093F101C092F100C091F129
:10735000010194AF0DD09607968B911F921F931F3A
:10736000941F912BD8B4922BD8B4932BD8B4942BD0
:107370003B0E9D6F9A0E9C6FCA0E9B6F9A6B0A0E06
:10738000986F9551D8B4962BD882010EEA6E910E63
:10739000E96E196AD2BE198ED29E94C1CAF193C108
:1073A000C9F192C1C8F191C1C7F19DC1CEF19CC193
:1073B000CDF19BC1CCF19AC1CBF10001D7EC24F007
:1073C00019BED28E0150005213E101019529985D3A
:1073D000D8A402D000010CD096510DE00F0B985D9F
:1073E00001E044E296BF42D096BD05D0200E37D0D2
:1073F000200E0101961796AB0FD0969B9551D8A4FD
:1074000096070050966F2D0EA16F0001C7EC2DF06E
:1074100001019651006E966B9551985D0DE10050FB
:10742000966F2E0EA16F0001C7EC2DF00101965151
:10743000006E200E9617000E300E96AB10D0969B65
:107440009551D8A496070050966F2D0EA16F00019C
:10745000C7EC2DF001019651006E966B300E0026A0
:1074600000C0A1F10001C7EC2DF00101D892196A0A
:10747000D2BE198ED29E9DC1CAF19CC1C9F19BC1D9
:10748000C8F19AC1C7F1CE6BCD6BCC6B0A0ECB6F36
:107490000001D7EC24F019BED28E03C09DF102C0CA
:1074A0009CF101C09BF100C09AF10101982F6CD7AB
:1074B000000112009551030811E1FFEC2FF03A0E84
:1074C000F66E230EF76E0BEC30F020EC30F04C0E25
:1074D000F66E230EF76E0BEC30F0ECD795510308E7
:1074E00075E0EDC0EEF0ED51FF0AEE6F0101946B17
:1074F000EEC093F1000149EC2EF003C0A1F102C0EF
:10750000A0F101C09FF100C09EF1550E0101A56FD1
:10751000C10EA46F480EA36F7D0EA26F000114EC84
:107520002FF003C0ECF002C0EBF001C0EAF000C0A5
:10753000E9F0FFEC2FF05E0EF66E230EF76E0D0EE7
:107540000101956F0001B6EC30F0010EE96EECC060
:1075500094F1EBC093F1EAC092F1E9C091F101011D
:10756000956B0001C1DE250E0101A16F0001C7EC82
:107570002DF020EC30F0740EF66E230EF76E0BEC4F
:1075800030F0952D0BD0ED2B0A0E0101A56F0001F7
:107590009CEC2DF0EDC091F12DEC30F095510408EC
:1075A0000BE1ED070A0E0101A56F00019CEC2DF027
:1075B000EDC091F12DEC30F09551050806E1010187
:1075C00016971699169B169D000188D7020E010189
:1075D000916FFA0EA56F00019CEC2DF00101912F27
:1075E000F8D70001E3EF3EF06EEC30F0F96BFA6B88
:1075F0006F0048FF92F1D29E3901E16B3D0EE06FC2
:10760000E59DE59FE581E351E59DE58F010192BF91
:10761000D28E0001E26FF053D8A423D19551030814
:1076200050E0FFEC2FF0F20EF66E230EF76E0BEC2F
:1076300030F020EC30F0040EF66E240EF76E0BECFA
:1076400030F0952D1ED0FFEC2FF0160EF66E240EA6
:10765000F76E0BEC30F020EC30F0280EF66E240EB6
:10766000F76E0BEC30F001019181080E926FFA0E6B
:10767000A56F00019CEC2DF00101922FF8D70001BD
:1076800020D0955104081CE1FFEC2FF03A0EF66E65
:10769000240EF76E0BEC30F020EC30F04C0EF66E52
:1076A000240EF76E0BEC30F0080E0101926FFA0E0B
:1076B000A56F00019CEC2DF00101922FF8D700017D
:1076C000ADD76F0048FF92F1D29E3901E16B3D0EBC
:1076D000E06FE59DE59FE581E351E59DE58F0101C3
:1076E00092BFD28E0001E26F010191A1B8D00001DA
:1076F000E2515A0801E2E26BFFEC2FF05C0EF66EED
:10770000240EF76E090E0101956F0001B6EC30F002
:10771000E2C092F1130E0101936F0001E5EC30F02D
:10772000680EF66E240EF76E040E0101956F0001CF
:10773000B6EC30F020EC30F06E0EF66E240EF76EE4
:107740000BEC30F0640E0101A56F00019CEC2DF0F4
:107750009551040801E1E22B640E0101A56F0001BF
:107760009CEC2DF0952D01D0E2079551030875E1B1
:10777000D250006ED29E3901E16B3D0EE06F600089
:107780008BF3E3F9E59DE59FE585550EE66FAA0EBF
:10779000E66FE583E5B3FED7E595E59DE58F0050FF
:1077A000D2120400840E006E002EFED700D06F00AF
:1077B00048FF92F1D29EE16B3D0EE06FE59DE59FA3
:1077C000E581E351E59DE58F010192BFD28E000175
:1077D000E26FFFEC2FF0800EF66E240EF76E090EAE
:1077E0000101956F0001B6EC30F0E2C092F1130E8A
:1077F0000101936F0001E5EC30F08C0EF66E240E63
:10780000F76E040E0101956F0001B6EC30F020EC2C
:1078100030F0920EF66E240EF76E0BEC30F0010194
:10782000936BE2C092F1020E956F580E946F0001B7
:1078300036EC2EF0E66BE56B02C0E4F001C0E3F03D
:10784000080E0101926FFA0EA56F00019CEC2DF05D
:107850000101922FF8D79191000146D701011CD068
:107860000001FFEC2FF0A40EF66E240EF76E0BEC69
:1078700030F020EC30F0B60EF66E240EF76E0BEC06
:1078800030F0080E0101926FFA0EA56F00019CEC1A
:107890002DF00101922FF8D70001EAEF3EF06EECD7
:1078A00030F0F96BFA6B95510308D8B4A7D0F53DC9
:1078B00094D0FFEC2FF0C80EF66E240EF76E0BEC92
:1078C00030F020EC30F0DA0EF66E240EF76E0BEC92
:1078D00030F0952D48D0FFEC2FF0EC0EF66E240E14
:1078E000F76E0BEC30F020EC30F0FE0EF66E240E4E
:1078F000F76E0BEC30F0F06BD250006ED29E390177
:10790000E16B2D0EE06F6000C3F3E3F9E59DE59FA9
:10791000E585550EE66FAA0EE66FE583E5B3FED763
:10792000E595E59DE58F0050D2126F0048FF91F17B
:10793000D29EE16B2D0EE06FE59DE59FE581E35161
:10794000E59DE58F010191BFD28E0001F06F080E19
:107950000101916FFA0EA56F00019CEC2DF0010161
:10796000912FF8D700019551040836E1FFEC2FF074
:10797000100EF66E250EF76E0BEC30F020EC30F0AA
:10798000220EF66E250EF76E0BEC30F0F069D25039
:10799000006ED29E3901E16B2D0EE06F6000C3F3E3
:1079A000E3F9E59DE59FE585550EE66FAA0EE66FC6
:1079B000E583E5B3FED7E595E59DE58F0050D2124E
:1079C000080E0101916FFA0EA56F00019CEC2DF0DD
:1079D0000101912FF8D7000110D0FFEC2FF0340EE9
:1079E000F66E250EF76E0BEC30F020EC30F0460E04
:1079F000F66E250EF76E0BEC30F055D7F0EF3EF03B
:107A00006EEC30F0F96BFA6B95510308D8B482D064
:107A1000FFEC2FF0860EF66E230EF76E0BEC30F0B7
:107A200020EC30F0980EF66E230EF76E0BEC30F073
:107A3000952D36D0FFEC2FF0AA0EF66E230EF76EC2
:107A40000BEC30F020EC30F0BC0EF66E230EF76E2F
:107A50000BEC30F0F56BD250006ED29E3901E16B29
:107A6000300EE06F6000D7F3E3F9E59DE59FE58513
:107A7000550EE66FAA0EE66FE583E5B3FED7E595F2
:107A8000E59DE58F0050D212080E0101916FFA0EAC
:107A9000A56F00019CEC2DF00101912FF8D700019A
:107AA0009551040836E1FFEC2FF0CE0EF66E230E52
:107AB000F76E0BEC30F020EC30F0E00EF66E230E9B
:107AC000F76E0BEC30F0F569D250006ED29E3901A2
:107AD000E16B300EE06F6000D7F3E3F9E59DE59FC1
:107AE000E585550EE66FAA0EE66FE583E5B3FED792
:107AF000E595E59DE58F0050D212080E0101916FCA
:107B0000FA0EA56F00019CEC2DF00101912FF8D722
:107B100000017AD7F6EF3EF06EEC30F0F96BFA6BBD
:107B200095510308D8B4BBD0F951090801E2F96BAB
:107B3000FA51090801E2FA6BFFEC2FF0760EF66EAF
:107B40003C0EF76E0BEC30F020EC30F0880EF66E49
:107B50003C0EF76E080E0101956F0001B6EC30F097
:107B6000F9C092F1180E0101936F0001E5EC30F0BD
:107B7000930EF66E3C0EF76E050E0101956F000137
:107B8000B6EC30F0FAC092F1180E0101936F0001CB
:107B9000E5EC30F0200E0101A16F0001C7EC2DF0E3
:107BA000955104083DE1FA2B9551040839E1FA5149
:107BB000090801E2FA6BFFEC2FF09E0EF66E3C0E08
:107BC000F76E0BEC30F020EC30F0B00EF66E3C0EA1
:107BD000F76E080E0101956F0001B6EC30F0F9C0A8
:107BE00092F1180E0101936F0001E5EC30F0BB0E2D
:107BF000F66E3C0EF76E050E0101956F0001B6ECB6
:107C000030F0FAC092F1180E0101936F0001E5EC1B
:107C100030F0200E0101A16F0001C7EC2DF0C4D798
:107C2000952D3CD0F92B952D39D0F951090801E259
:107C3000F96BFFEC2FF0C60EF66E3C0EF76E0BECF8
:107C400030F020EC30F0D80EF66E3C0EF76E080ED9
:107C50000101956F0001B6EC30F0F9C092F1180EF9
:107C60000101936F0001E5EC30F0E30EF66E3C0E7F
:107C7000F76E050E0101956F0001B6EC30F0FAC009
:107C800092F1180E0101936F0001E5EC30F0200E27
:107C90000101A16F0001C7EC2DF0C5D741D7F95103
:107CA000040802E1FA5348E0F951050802E1FA53E9
:107CB00043E0F951060802E1FA533EE0F9510608A3
:107CC00003E1FA51060838E0F951070802E1FA53D6
:107CD00033E0F951070803E1FA5105082DE0F951A5
:107CE000080802E1FA5328E0F951090802E1FA53C1
:107CF00023E0F951090803E1FA2D01D01DD0F95113
:107D0000030802E1FA5318E0F951020802E1FA53BC
:107D100013E0F951020803E1FA2D01D00DD0F95119
:107D2000050803E1FA2D01D007D0F9510808D8A4BD
:107D30005ED0FA5109085BE1F951020804E1FA53F7
:107D4000D8B423EF31F0F951020804E1FA2D02D042
:107D50003DEF32F0F951030804E1FA53D8B4BCEF17
:107D600032F0F951040804E1FA53D8B4C2EF33F009
:107D7000F951050804E1FA53D8B444EF34F0F9514D
:107D8000050804E1FA2D02D0CFEF34F0F9510608CE
:107D900004E1FA53D8B45DEF36F0F951070804E175
:107DA000FA53D8B473EF37F0F951070805E1FA51E7
:107DB0000508D8B495EF38F0F951080804E1FA53F2
:107DC000D8B45AEF3AF0F951080804E1FA51090819
:107DD000D8B40AD4F951090803E1FA53D8B45FD5ED
:107DE000F951090803E1FA2D01D00AD61DD0FFECA4
:107DF0002FF0EE0EF66E3C0EF76E0BEC30F020EC32
:107E000030F0000EF66E3D0EF76E0BEC30F0020E09
:107E10000101916FFA0EA56F00019CEC2DF001019C
:107E2000912FF8D7FF0000017BD6B5EF40F00A0E86
:107E30000101A56F00019CEC2DF0D93D10D020EC84
:107E400030F0F80EF66E280EF76E0BEC30F0FFEC0B
:107E50002FF00A0EF66E290EF76E0BEC30F0D953A8
:107E600010E120EC30F01C0EF66E290EF76E0BECD4
:107E700030F0FFEC2FF02E0EF66E290EF76E0BECA5
:107E800030F0D9517F0810E120EC30F0400EF66E52
:107E9000290EF76E0BEC30F0FFEC2FF0520EF66E61
:107EA000290EF76E0BEC30F01200010EA86F6EEC8D
:107EB00030F0F96BFA6BA851010A35E0030AD8B427
:107EC0009DD1010AD8B44FEF43F0070AD8B43EEF72
:107ED00045F0010AD8B42FEF47F0030AD8B41BEFDE
:107EE00049F0010AD8B480EF4BF00F0AD8B4DBEFA9
:107EF0004DF0010AD8B425EF50F0030AD8B41BEFB7
:107F000051F0010AD8B439EF53F0070AD8B44CEF56
:107F100055F0010AD8B460EF56F0030AD8B4D2EF96
:107F200057F07BEF58F06EEC30F095510308D8B461
:107F300000D1F951090801E2F96BFA51090801E28F
:107F4000FA6BD93D08D0FFEC2FF0F40EF66E290E37
:107F5000F76E0BEC30F0D95308E1FFEC2FF0060E72
:107F6000F66E2A0EF76E0BEC30F0D9517F0808E15F
:107F7000FFEC2FF0180EF66E2A0EF76E0BEC30F0B9
:107F800020EC30F02A0EF66E2A0EF76E080E010174
:107F9000956F0001B6EC30F0F9C092F1180E0101B6
:107FA000936F0001E5EC30F0350EF66E2A0EF76E99
:107FB000050E0101956F0001B6EC30F0FAC092F1A8
:107FC000180E0101936F0001E5EC30F0200E010165
:107FD000A16F0001C7EC2DF09551040854E1FA2B74
:107FE0009551040850E1FA51090801E2FA6BD93DB4
:107FF00008D0FFEC2FF0400EF66E2A0EF76E0BEC59
:1080000030F0D95308E1FFEC2FF0520EF66E2A0E35
:10801000F76E0BEC30F0D9517F0808E1FFEC2FF040
:10802000640EF66E2A0EF76E0BEC30F020EC30F09A
:10803000760EF66E2A0EF76E080E0101956F00019E
:10804000B6EC30F0F9C092F1180E0101936F000107
:10805000E5EC30F0810EF66E2A0EF76E050E01018A
:10806000956F0001B6EC30F0FAC092F1180E0101E4
:10807000936F0001E5EC30F0200E0101A16F0001CB
:10808000C7EC2DF0ADD7952D53D0F92B952D50D0B1
:10809000F951090801E2F96BD93D08D0FFEC2FF046
:1080A0008C0EF66E2A0EF76E0BEC30F0D95308E109
:1080B000FFEC2FF09E0EF66E2A0EF76E0BEC30F0F2
:1080C000D9517F0808E1FFEC2FF0B00EF66E2A0EB2
:1080D000F76E0BEC30F020EC30F0C20EF66E2A0E8C
:1080E000F76E080E0101956F0001B6EC30F0F9C093
:1080F00092F1180E0101936F0001E5EC30F0CD0E06
:10810000F66E2A0EF76E050E0101956F0001B6ECB2
:1081100030F0FAC092F1180E0101936F0001E5EC06
:1081200030F0200E0101A16F0001C7EC2DF0AED799
:10813000FCD6640E0101A56F00019CEC2DF0F951F5
:10814000090803E1FA5109080AE0F92D03D0FA51B0
:10815000030805E0F9530BE1FA51040808E1F9536B
:1081600004E1FA510408D8B4D7D4A82B45D0D93D9E
:1081700010D0FFEC2FF0D80EF66E2A0EF76E0BEC37
:1081800030F020EC30F0EA0EF66E2A0EF76E0BECB3
:1081900030F0D95310E1FFEC2FF0FC0EF66E2A0EF2
:1081A000F76E0BEC30F020EC30F00E0EF66E2B0E6E
:1081B000F76E0BEC30F0D9517F0810E1FFEC2FF097
:1081C000200EF66E2B0EF76E0BEC30F020EC30F03C
:1081D000320EF66E2B0EF76E0BEC30F0020E010134
:1081E000916FFA0EA56F00019CEC2DF00101912F0B
:1081F000F8D783EF58F000017BEF58F0F92D06D047
:10820000FA51030803E1A82B7BEF58F06EEC30F035
:10821000D93D09D0FFEC2FF0440EF66E2B0EF76E11
:108220000BEC30F016D0D95309E1FFEC2FF0560ECD
:10823000F66E2B0EF76E0BEC30F00BD0D9517F0899
:1082400008E1FFEC2FF0680EF66E2B0EF76E0BECCC
:1082500030F0D93D29D020EC30F07A0EF66E2B0E9E
:10826000F76E080E0101956F0001B6EC30F07F0E3D
:108270000101A16F0001C7EC2DF0840EF66E2B0EEC
:10828000F76E050E0101956F0001B6EC30F07E0E21
:108290000101A16F0001C7EC2DF0200E0101A16FBB
:1082A0000001C7EC2DF056D0D95329E120EC30F075
:1082B0008E0EF66E2B0EF76E080E0101956F000103
:1082C000B6EC30F07F0E0101A16F0001C7EC2DF07C
:1082D000980EF66E2B0EF76E050E0101956F0001DC
:1082E000B6EC30F07E0E0101A16F0001C7EC2DF05D
:1082F000200E0101A16F0001C7EC2DF02BD0D95148
:108300007F0828E120EC30F0A20EF66E2B0EF76EFF
:10831000080E0101956F0001B6EC30F07F0E0101EF
:10832000A16F0001C7EC2DF0AC0EF66E2B0EF76EB0
:10833000050E0101956F0001B6EC30F07E0E0101D3
:10834000A16F0001C7EC2DF0200E0101A16F00010B
:10835000C7EC2DF09551040801E1A82B952D01D013
:10836000A807A85302E1010EA86F95510308D8A4ED
:1083700094D1D93D09D0FFEC2FF0B60EF66E2B0E3E
:10838000F76E0BEC30F016D0D95309E1FFEC2FF06B
:10839000C80EF66E2B0EF76E0BEC30F00BD0D951E9
:1083A0007F0808E1FFEC2FF0DA0EF66E2B0EF76E69
:1083B0000BEC30F0D93D29D020EC30F0EC0EF66E0D
:1083C0002B0EF76E080E0101956F0001B6EC30F030
:1083D0007F0E0101A16F0001C7EC2DF0F60EF66EC5
:1083E0002B0EF76E050E0101956F0001B6EC30F013
:1083F0007E0E0101A16F0001C7EC2DF0200E0101DE
:10840000A16F0001C7EC2DF056D0D95329E120EC23
:1084100030F0000EF66E2C0EF76E080E0101956F0F
:108420000001B6EC30F07F0E0101A16F0001C7EC36
:108430002DF00A0EF66E2C0EF76E050E0101956FEB
:108440000001B6EC30F07E0E0101A16F0001C7EC17
:108450002DF0200E0101A16F0001C7EC2DF02BD0F3
:10846000D9517F0828E120EC30F0140EF66E2C0E66
:10847000F76E080E0101956F0001B6EC30F07F0E2B
:108480000101A16F0001C7EC2DF01E0EF66E2C0E3F
:10849000F76E050E0101956F0001B6EC30F07E0E0F
:1084A0000101A16F0001C7EC2DF0200E0101A16FA9
:1084B0000001C7EC2DF06EEC30F095510308D8B4F4
:1084C000BDD0D9517F0809E1FFEC2FF0280EF66EE0
:1084D0002C0EF76E0BEC30F008D0FFEC2FF03A0EBC
:1084E000F66E2C0EF76E0BEC30F0D93D08D020EC78
:1084F00030F04C0EF66E2C0EF76E0BEC30F0D953BC
:1085000008E120EC30F05E0EF66E2C0EF76E0BECF0
:1085100030F0D9517F0808E120EC30F0700EF66E93
:108520002C0EF76E0BEC30F095510308D8B4B2D096
:10853000952D40D06EEC30F0955105083BE1D93DCA
:1085400011D0FFEC2FF0820EF66E2C0EF76E0BECB6
:1085500030F020EC30F0940EF66E2C0EF76E0BEC33
:1085600030F026D0D95311E1FFEC2FF0A60EF66EB5
:108570002C0EF76E0BEC30F020EC30F0B80EF66EEF
:108580002C0EF76E0BEC30F013D0D9517F0810E1B0
:10859000FFEC2FF0CA0EF66E2C0EF76E0BEC30F0DF
:1085A00020EC30F0DC0EF66E2C0EF76E0BEC30F09B
:1085B0008889C2D79551040840E16EEC30F095519E
:1085C00005083BE1D93D11D0FFEC2FF0EE0EF66E21
:1085D0002C0EF76E0BEC30F020EC30F0000EF66E47
:1085E0002D0EF76E0BEC30F026D0D95311E1FFECD5
:1085F0002FF0120EF66E2D0EF76E0BEC30F020EC15
:1086000030F0240EF66E2D0EF76E0BEC30F013D01A
:10861000D9517F0810E1FFEC2FF0360EF66E2D0ECB
:10862000F76E0BEC30F020EC30F0480EF66E2D0EAD
:10863000F76E0BEC30F08899C2D73FD717EC3FF0BC
:10864000952D21D0000E88B9010E0101916FD250F5
:10865000006ED29E3901E16B140EE06F600047F6A8
:10866000E3F9E59DE59FE585550EE66FAA0EE66FF9
:10867000E583E5B3FED7E595E59DE58F0050D21281
:108680000AD006D000019551040803E1390103D056
:108690000001D4D739010001A82B7BEF58F0F92D48
:1086A00006D0FA51030803E1A82B7BEF58F06EECDB
:1086B00030F0D93D31D0FFEC2FF05A0EF66E2D0E72
:1086C000F76E0BEC30F020EC30F06C0EF66E2D0EE9
:1086D000F76E080E0101956F0001B6EC30F07F0EC9
:1086E0000101A16F0001C7EC2DF0760EF66E2D0E84
:1086F000F76E050E0101956F0001B6EC30F07E0EAD
:108700000101A16F0001C7EC2DF0200E0101A16F46
:108710000001C7EC2DF066D0D95331E1FFEC2FF00A
:10872000800EF66E2D0EF76E0BEC30F020EC30F074
:10873000920EF66E2D0EF76E080E0101956F000178
:10874000B6EC30F07F0E0101A16F0001C7EC2DF0F7
:108750009C0EF66E2D0EF76E050E0101956F000151
:10876000B6EC30F07E0E0101A16F0001C7EC2DF0D8
:10877000200E0101A16F0001C7EC2DF033D0D951BB
:108780007F0830E1FFEC2FF0A60EF66E2D0EF76E8F
:108790000BEC30F020EC30F0B80EF66E2D0EF76ECC
:1087A000080E0101956F0001B6EC30F07F0E01015B
:1087B000A16F0001C7EC2DF0C20EF66E2D0EF76E04
:1087C000050E0101956F0001B6EC30F07E0E01013F
:1087D000A16F0001C7EC2DF0200E0101A16F000177
:1087E000C7EC2DF09551040801E1A82B952D01D07F
:1087F000A807A85302E1010EA86F95510308D8A459
:108800003BD16EEC30F0699D95510308D8B4E6D0A9
:10881000878F69BD5ED0D93D1DD0FFEC2FF0CC0E07
:10882000F66E2D0EF76E0A0E0101956F0001B6EC83
:1088300030F0000EE96EB7C092F1B6C091F15BEC7A
:1088400035F020EC30F0DC0EF66E2D0EF76E0BECF2
:1088500030F03ED0D9531DE1FFEC2FF0EE0EF66E56
:108860002D0EF76E0A0E0101956F0001B6EC30F087
:10887000000EE96EB7C092F1B6C091F15BEC35F035
:1088800020EC30F0FE0EF66E2D0EF76E0BEC30F095
:108890001FD0D9517F081CE1FFEC2FF0100EF66EAF
:1088A0002E0EF76E0A0E0101956F0001B6EC30F046
:1088B000000EE96EB7C092F1B6C091F15BEC35F0F5
:1088C00020EC30F0200EF66E2E0EF76E0BEC30F032
:1088D0005DD0D93D1DD0FFEC2FF0320EF66E2E0E7E
:1088E000F76E0A0E0101956F0001B6EC30F0000E34
:1088F000E96EC3C092F1C2C091F15BEC35F020EC9F
:1089000030F0420EF66E2E0EF76E0BEC30F03ED0CD
:10891000D9531DE1FFEC2FF0540EF66E2E0EF76EBC
:108920000A0E0101956F0001B6EC30F0000EE96E01
:10893000C3C092F1C2C091F15BEC35F020EC30F095
:10894000640EF66E2E0EF76E0BEC30F01FD0D95180
:108950007F081CE1FFEC2FF0760EF66E2E0EF76E00
:108960000A0E0101956F0001B6EC30F0000EE96EC1
:10897000C3C092F1C2C091F15BEC35F020EC30F055
:10898000860EF66E2E0EF76E0BEC30F0952D06D09F
:1089900001011689168B169D0001698D95510408F9
:1089A00006E101011687168B169D0001698D955110
:1089B000050813E1010116971699169B169D0001F3
:1089C000AD6BAC6BAB6BAA6BB16BB06BAF6B030EEB
:1089D000AE6FB56BB46BB36BB26B16D7640E01019F
:1089E000A56F00019CEC2DF069AD43D017EC3FF072
:1089F000952D38D0C3C0B7F0C2C0B6F06000DBF22E
:108A0000E3F9D250006ED29E3901E16B060EE06FA1
:108A1000E59DE59FE585550EE66FAA0EE66FE583B9
:108A2000E5B3FED7E595E59DE58F0050D2126000D5
:108A3000DFF2E3F9D250006ED29EE16B070EE06FD9
:108A4000E59DE59FE585550EE66FAA0EE66FE58389
:108A5000E5B3FED7E595E59DE58F0050D2120AD02B
:108A600006D000019551040803E1390103D000014B
:108A7000BDD739010001A82B7BEF58F0F92D03D0A9
:108A8000FA51030802E0EF3D03D0A82B7BEF58F02A
:108A90006EEC30F0D93D31D0FFEC2FF0980EF66E31
:108AA0002E0EF76E0BEC30F020EC30F0AA0EF66EC6
:108AB0002E0EF76E080E0101956F0001B6EC30F036
:108AC0007F0E0101A16F0001C7EC2DF0B40EF66E10
:108AD0002E0EF76E050E0101956F0001B6EC30F019
:108AE0007E0E0101A16F0001C7EC2DF0200E0101E7
:108AF000A16F0001C7EC2DF066D0D95331E1FFEC36
:108B00002FF0BE0EF66E2E0EF76E0BEC30F020EC52
:108B100030F0D00EF66E2E0EF76E080E0101956F36
:108B20000001B6EC30F07F0E0101A16F0001C7EC2F
:108B30002DF0DA0EF66E2E0EF76E050E0101956F12
:108B40000001B6EC30F07E0E0101A16F0001C7EC10
:108B50002DF0200E0101A16F0001C7EC2DF033D0E4
:108B6000D9517F0830E1FFEC2FF0E40EF66E2E0EA7
:108B7000F76E0BEC30F020EC30F0F60EF66E2E0EA9
:108B8000F76E080E0101956F0001B6EC30F07F0E14
:108B90000101A16F0001C7EC2DF0000EF66E2F0E43
:108BA000F76E050E0101956F0001B6EC30F07E0EF8
:108BB0000101A16F0001C7EC2DF0200E0101A16F92
:108BC0000001C7EC2DF09551040801E1A82B952D6B
:108BD00001D0A807A85302E1010EA86F9551030820
:108BE000D8A43BD16EEC30F0699D95510308D8B400
:108BF000E6D0878F69BD5ED0D93D1DD0FFEC2FF048
:108C00000A0EF66E2F0EF76E0A0E0101956F000127
:108C1000B6EC30F0000EE96EB9C092F1B8C091F137
:108C20005BEC35F020EC30F01A0EF66E2F0EF76E7E
:108C30000BEC30F03ED0D9531DE1FFEC2FF02C0EA1
:108C4000F66E2F0EF76E0A0E0101956F0001B6EC5D
:108C500030F0000EE96EB9C092F1B8C091F15BEC52
:108C600035F020EC30F03C0EF66E2F0EF76E0BEC6C
:108C700030F01FD0D9517F081CE1FFEC2FF04E0ED1
:108C8000F66E2F0EF76E0A0E0101956F0001B6EC1D
:108C900030F0000EE96EB9C092F1B8C091F15BEC12
:108CA00035F020EC30F05E0EF66E2F0EF76E0BEC0A
:108CB00030F05DD0D93D1DD0FFEC2FF0700EF66E78
:108CC0002F0EF76E0A0E0101956F0001B6EC30F021
:108CD000000EE96EC3C092F1C2C091F15BEC35F0B9
:108CE00020EC30F0800EF66E2F0EF76E0BEC30F0AD
:108CF0003ED0D9531DE1FFEC2FF0920EF66E2F0EF1
:108D0000F76E0A0E0101956F0001B6EC30F0000E0F
:108D1000E96EC3C092F1C2C091F15BEC35F020EC7A
:108D200030F0A20EF66E2F0EF76E0BEC30F01FD067
:108D3000D9517F081CE1FFEC2FF0B40EF66E2F0E18
:108D4000F76E0A0E0101956F0001B6EC30F0000ECF
:108D5000E96EC3C092F1C2C091F15BEC35F020EC3A
:108D600030F0C40EF66E2F0EF76E0BEC30F0952D32
:108D700006D001011689168B169D0001698D95514B
:108D8000040806E101011687168B169D0001698D06
:108D90009551050813E1010116971699169B169D2A
:108DA0000001AD6BAC6BAB6BAA6BB16BB06BAF6B17
:108DB000030EAE6FB56BB46BB36BB26B16D7640EAC
:108DC0000101A56F00019CEC2DF069AD43D017ECBB
:108DD0003FF0952D38D0C3C0B9F0C2C0B8F06000E4
:108DE000E3F2E3F9D250006ED29E3901E16B280E16
:108DF000E06FE59DE59FE585550EE66FAA0EE66FEF
:108E0000E583E5B3FED7E595E59DE58F0050D212E9
:108E10006000E7F2E3F9D250006ED29EE16B290EBA
:108E2000E06FE59DE59FE585550EE66FAA0EE66FBE
:108E3000E583E5B3FED7E595E59DE58F0050D212B9
:108E40000AD006D000019551040803E1390103D08E
:108E50000001BDD739010001A82B7BEF58F0F92D97
:108E600006D0FA51030803E1A82B7BEF58F06EEC13
:108E700030F0D93D31D0FFEC2FF0D60EF66E2F0E2C
:108E8000F76E0BEC30F020EC30F0E80EF66E2F0EA3
:108E9000F76E080E0101956F0001B6EC30F07F0E01
:108EA0000101A16F0001C7EC2DF0F20EF66E2F0E3E
:108EB000F76E050E0101956F0001B6EC30F07E0EE5
:108EC0000101A16F0001C7EC2DF0200E0101A16F7F
:108ED0000001C7EC2DF066D0D95331E1FFEC2FF043
:108EE000FC0EF66E2F0EF76E0BEC30F020EC30F02F
:108EF0000E0EF66E300EF76E080E0101956F000132
:108F0000B6EC30F07F0E0101A16F0001C7EC2DF02F
:108F1000180EF66E300EF76E050E0101956F00010A
:108F2000B6EC30F07E0E0101A16F0001C7EC2DF010
:108F3000200E0101A16F0001C7EC2DF033D0D951F3
:108F40007F0830E1FFEC2FF0220EF66E300EF76E48
:108F50000BEC30F020EC30F0340EF66E300EF76E85
:108F6000080E0101956F0001B6EC30F07F0E010193
:108F7000A16F0001C7EC2DF03E0EF66E300EF76EBD
:108F8000050E0101956F0001B6EC30F07E0E010177
:108F9000A16F0001C7EC2DF0200E0101A16F0001AF
:108FA000C7EC2DF09551040801E1A82B952D09D0AF
:108FB000A807F92D03D0FA51030802E0EF3D01D0D4
:108FC000A807A85302E1010EA86F95510308D8A481
:108FD00030D16EEC30F0699F95510308D8B4DBD0E6
:108FE000878F69BF5ED0D93D1DD0FFEC2FF0480EB2
:108FF000F66E300EF76E0A0E0101956F0001B6ECA9
:1090000030F0000EE96EBBC092F1BAC091F15BEC9A
:1090100035F020EC30F0580EF66E300EF76E0BEC9B
:1090200030F03ED0D9531DE1FFEC2FF06A0EF66E02
:10903000300EF76E0A0E0101956F0001B6EC30F0AC
:10904000000EE96EBBC092F1BAC091F15BEC35F055
:1090500020EC30F07A0EF66E300EF76E0BEC30F03E
:109060001FD0D9517F081CE1FFEC2FF08C0EF66E5B
:10907000300EF76E0A0E0101956F0001B6EC30F06C
:10908000000EE96EBBC092F1BAC091F15BEC35F015
:1090900020EC30F09C0EF66E300EF76E0BEC30F0DC
:1090A0005DD0D93D1DD0FFEC2FF0AE0EF66E300E28
:1090B000F76E0A0E0101956F0001B6EC30F0000E5C
:1090C000E96EC3C092F1C2C091F15BEC35F020ECC7
:1090D00030F0BE0EF66E300EF76E0BEC30F03ED078
:1090E000D9531DE1FFEC2FF0D00EF66E300EF76E67
:1090F0000A0E0101956F0001B6EC30F0000EE96E2A
:10910000C3C092F1C2C091F15BEC35F020EC30F0BD
:10911000E00EF66E300EF76E0BEC30F01FD0D9512A
:109120007F081CE1FFEC2FF0F20EF66E300EF76EAA
:109130000A0E0101956F0001B6EC30F0000EE96EE9
:10914000C3C092F1C2C091F15BEC35F020EC30F07D
:10915000020EF66E310EF76E0BEC30F0952D07D047
:1091600001011689168B168D0001698F13D0955158
:10917000040807E101011687168B169D0001698F0F
:1091800009D09551050806E1010116971699169B1D
:10919000169D000121D7640E0101A56F00019CEC12
:1091A0002DF069AF43D017EC3FF0952D38D0C3C0F8
:1091B000BBF0C2C0BAF06000EBF2E3F9D250006E2F
:1091C000D29E3901E16B080EE06FE59DE59FE585D4
:1091D000550EE66FAA0EE66FE583E5B3FED7E5957B
:1091E000E59DE58F0050D2126000EFF2E3F9D25016
:1091F000006ED29EE16B090EE06FE59DE59FE5856F
:10920000550EE66FAA0EE66FE583E5B3FED7E5954A
:10921000E59DE58F0050D2120AD006D0000195518D
:10922000040803E1390103D00001BDD73901000171
:10923000A82B7BEF58F0F92D06D0FA51030803E173
:10924000A82B7BEF58F06EEC30F0D93D31D0FFEC1D
:109250002FF0140EF66E310EF76E0BEC30F020ECA2
:1092600030F0260EF66E310EF76E080E0101956F86
:109270000001B6EC30F07F0E0101A16F0001C7ECD8
:109280002DF0300EF66E310EF76E050E0101956F62
:109290000001B6EC30F07E0E0101A16F0001C7ECB9
:1092A0002DF0200E0101A16F0001C7EC2DF066D05A
:1092B000D95331E1FFEC2FF03A0EF66E310EF76E16
:1092C0000BEC30F020EC30F04C0EF66E310EF76EF9
:1092D000080E0101956F0001B6EC30F07F0E010120
:1092E000A16F0001C7EC2DF0560EF66E310EF76E31
:1092F000050E0101956F0001B6EC30F07E0E010104
:10930000A16F0001C7EC2DF0200E0101A16F00013B
:10931000C7EC2DF033D0D9517F0830E1FFEC2FF0AE
:10932000600EF66E310EF76E0BEC30F020EC30F084
:10933000720EF66E310EF76E080E0101956F000188
:10934000B6EC30F07F0E0101A16F0001C7EC2DF0EB
:109350007C0EF66E310EF76E050E0101956F000161
:10936000B6EC30F07E0E0101A16F0001C7EC2DF0CC
:10937000200E0101A16F0001C7EC2DF095510408EA
:1093800001E1A82B952D01D0A8076F0048FF91F1AE
:10939000D29E3901E16B0B0EE06FE59DE59FE58103
:1093A000E351E59DE58F010191BFD28E0001F86F79
:1093B00095510308D8A4A2D16EEC30F08791955155
:1093C0000308D8B462D187B1B2D0D93D2DD0FFEC1B
:1093D0002FF0860EF66E310EF76E0A0E0101956FB4
:1093E0000001B6EC30F0020E0101916F200EA16F6A
:1093F0000001C7EC2DF00101912FF8D7F8C092F1D0
:10940000130E936F0001E5EC30F0250E0101A16F02
:109410000001C7EC2DF020EC30F0960EF66E310E08
:10942000F76E0BEC30F05ED0D9532DE1FFEC2FF04E
:10943000A80EF66E310EF76E0A0E0101956F00014F
:10944000B6EC30F0020E0101916F200EA16F000109
:10945000C7EC2DF00101912FF8D7F8C092F1130E4F
:10946000936F0001E5EC30F0250E0101A16F0001C2
:10947000C7EC2DF020EC30F0B80EF66E310EF76E22
:109480000BEC30F02FD0D9517F082CE1FFEC2FF0FE
:10949000CA0EF66E310EF76E0A0E0101956F0001CD
:1094A000B6EC30F0020E0101916F200EA16F0001A9
:1094B000C7EC2DF00101912FF8D7F8C092F1130EEF
:1094C000936F0001E5EC30F0250E0101A16F000162
:1094D000C7EC2DF020EC30F0DA0EF66E310EF76EA0
:1094E0000BEC30F00101926BF8C091F10001B1EC8E
:1094F0002FF002C0DDF001C0DCF0010E0101A56F0C
:1095000000019CEC2DF09551040802E1F82B8781B5
:10951000010E0101A56F00019CEC2DF0952D02D0EC
:10952000F8078781F851630801E2F86BADD0D93DA7
:109530002CD0FFEC2FF0EC0EF66E310EF76E0A0E0B
:109540000101956F0001B6EC30F0020E0101916F40
:10955000200EA16F0001C7EC2DF00101912FF8D76B
:10956000F8C092F1130E936F0001E5EC30F0250E78
:109570000101A16F0001C7EC2DF020EC30F0FC0ED2
:10958000F66E310EF76E0BEC30F0D9532CE1FFEC98
:109590002FF00E0EF66E320EF76E0A0E0101956F69
:1095A0000001B6EC30F0020E0101916F200EA16FA8
:1095B0000001C7EC2DF00101912FF8D7F8C092F10E
:1095C000130E936F0001E5EC30F0250E0101A16F41
:1095D0000001C7EC2DF020EC30F01E0EF66E320EBE
:1095E000F76E0BEC30F0D9517F082CE1FFEC2FF037
:1095F000300EF66E320EF76E0A0E0101956F000105
:10960000B6EC30F0020E0101916F200EA16F000147
:10961000C7EC2DF00101912FF8D7F8C092F1130E8D
:10962000936F0001E5EC30F0250E0101A16F000100
:10963000C7EC2DF020EC30F0400EF66E320EF76ED7
:109640000BEC30F00101926BF8C091F10001B1EC2C
:109650002FF002C0DDF001C0DCF0320E0101A56F79
:1096600000019CEC2DF09551040801E1F82B320E1D
:109670000101A56F00019CEC2DF0952D01D0F8079C
:10968000F851630801E2F86B9AD6FFEC2FF0520E06
:10969000F66E320EF76E0BEC30F087A127D017EC88
:1096A0003FF0952D1CD0D250006ED29E3901E16B57
:1096B0000B0EE06F6000E3F3E3F9E59DE59FE585C0
:1096C000550EE66FAA0EE66FE583E5B3FED7E59586
:1096D000E59DE58F0050D2120AD006D000019551C9
:1096E000040803E1390103D00001D9D73901640E20
:1096F0000101A56F00019CEC2DF0A82B7BEF58F029
:10970000F92D06D0FA51030803E1A82B7BEF58F09E
:109710006EEC30F0D93D31D0FFEC2FF0640EF66ED8
:10972000320EF76E0BEC30F020EC30F0760EF66E69
:10973000320EF76E080E0101956F0001B6EC30F0A5
:109740007F0E0101A16F0001C7EC2DF0800EF66EB7
:10975000320EF76E050E0101956F0001B6EC30F088
:109760007E0E0101A16F0001C7EC2DF0200E01015A
:10977000A16F0001C7EC2DF066D0D95331E1FFECA9
:109780002FF08A0EF66E320EF76E0BEC30F020ECF6
:1097900030F09C0EF66E320EF76E080E0101956FDA
:1097A0000001B6EC30F07F0E0101A16F0001C7ECA3
:1097B0002DF0A60EF66E320EF76E050E0101956FB6
:1097C0000001B6EC30F07E0E0101A16F0001C7EC84
:1097D0002DF0200E0101A16F0001C7EC2DF033D058
:1097E000D9517F0830E1FFEC2FF0B00EF66E320E4B
:1097F000F76E0BEC30F020EC30F0C20EF66E320E4D
:10980000F76E080E0101956F0001B6EC30F07F0E87
:109810000101A16F0001C7EC2DF0CC0EF66E320EE7
:10982000F76E050E0101956F0001B6EC30F07E0E6B
:109830000101A16F0001C7EC2DF0200E0101A16F05
:109840000001C7EC2DF09551040801E1A82B952DDE
:1098500001D0A8076F0048FF91F1D29E3901E16B5A
:109860000D0EE06FE59DE59FE581E351E59DE58FF8
:10987000010191BFD28E0001F76F95510308D8A462
:1098800098D16EEC30F0879395510308D8B460D12D
:1098900087B3B0D0D93D2CD0FFEC2FF0D60EF66EAA
:1098A000320EF76E0A0E0101956F0001B6EC30F032
:1098B000020E0101916F200EA16F0001C7EC2DF087
:1098C0000101912FF8D7F7C092F1130E936F0001A9
:1098D000E5EC30F0250E0101A16F0001C7EC2DF081
:1098E00020EC30F0E60EF66E320EF76E0BEC30F038
:1098F000D9532CE1FFEC2FF0F80EF66E320EF76E16
:109900000A0E0101956F0001B6EC30F0020E010164
:10991000916F200EA16F0001C7EC2DF00101912F76
:10992000F8D7F7C092F1130E936F0001E5EC30F019
:10993000250E0101A16F0001C7EC2DF020EC30F0E5
:10994000080EF66E330EF76E0BEC30F0D9517F082F
:109950002CE1FFEC2FF01A0EF66E330EF76E0A0EA6
:109960000101956F0001B6EC30F0020E0101916F1C
:10997000200EA16F0001C7EC2DF00101912FF8D747
:10998000F7C092F1130E936F0001E5EC30F0250E55
:109990000101A16F0001C7EC2DF020EC30F02A0E80
:1099A000F66E330EF76E0BEC30F00101926BF7C0E0
:1099B00091F10001B1EC2FF002C0DDF001C0DCF04C
:1099C000010E0101A56F00019CEC2DF095510408DA
:1099D00002E1F72B8783010E0101A56F00019CECCA
:1099E0002DF0952D02D0F7078783F751630801E228
:1099F000F76BADD0D93D2CD0FFEC2FF03C0EF66EBE
:109A0000330EF76E0A0E0101956F0001B6EC30F0CF
:109A1000020E0101916F200EA16F0001C7EC2DF025
:109A20000101912FF8D7F7C092F1130E936F000147
:109A3000E5EC30F0250E0101A16F0001C7EC2DF01F
:109A400020EC30F04C0EF66E330EF76E0BEC30F06F
:109A5000D9532CE1FFEC2FF05E0EF66E330EF76E4D
:109A60000A0E0101956F0001B6EC30F0020E010103
:109A7000916F200EA16F0001C7EC2DF00101912F15
:109A8000F8D7F7C092F1130E936F0001E5EC30F0B8
:109A9000250E0101A16F0001C7EC2DF020EC30F084
:109AA0006E0EF66E330EF76E0BEC30F0D9517F0868
:109AB0002CE1FFEC2FF0800EF66E330EF76E0A0EDF
:109AC0000101956F0001B6EC30F0020E0101916FBB
:109AD000200EA16F0001C7EC2DF00101912FF8D7E6
:109AE000F7C092F1130E936F0001E5EC30F0250EF4
:109AF0000101A16F0001C7EC2DF020EC30F0900EB9
:109B0000F66E330EF76E0BEC30F00101926BF7C07E
:109B100091F10001B1EC2FF002C0DBF001C0DAF0EE
:109B2000320E0101A56F00019CEC2DF09551040847
:109B300001E1F72B320E0101A56F00019CEC2DF025
:109B4000952D01D0F707F751630801E2F76B9CD61A
:109B500087A327D017EC3FF0952D1CD0D250006E74
:109B6000D29E3901E16B0D0EE06F6000DFF3E3F987
:109B7000E59DE59FE585550EE66FAA0EE66FE58348
:109B8000E5B3FED7E595E59DE58F0050D2120AD0EA
:109B900006D000019551040803E1390103D000010A
:109BA000D9D73901640E0101A56F00019CEC2DF09D
:109BB000A82B7BEF58F069B903D0A82B7BEF58F0A6
:109BC0006EEC30F0D93D09D0FFEC2FF0A20EF66E0E
:109BD000330EF76E0BEC30F016D0D95309E1FFECE1
:109BE0002FF0B40EF66E330EF76E0BEC30F00BD098
:109BF000D9517F0808E1FFEC2FF0C60EF66E330E48
:109C0000F76E0BEC30F0D93D29D020EC30F0D80EB7
:109C1000F66E330EF76E080E0101956F0001B6EC7B
:109C200030F07F0E0101A16F0001C7EC2DF0E20EB4
:109C3000F66E330EF76E050E0101956F0001B6EC5E
:109C400030F07E0E0101A16F0001C7EC2DF0200E57
:109C50000101A16F0001C7EC2DF056D0D95329E1C5
:109C600020EC30F0EC0EF66E330EF76E080E0101AC
:109C7000956F0001B6EC30F07F0E0101A16F00017D
:109C8000C7EC2DF0F60EF66E330EF76E050E0101E1
:109C9000956F0001B6EC30F07E0E0101A16F00015E
:109CA000C7EC2DF0200E0101A16F0001C7EC2DF0D3
:109CB0002BD0D9517F0828E120EC30F0000EF66E51
:109CC000340EF76E080E0101956F0001B6EC30F00E
:109CD0007F0E0101A16F0001C7EC2DF00A0EF66E98
:109CE000340EF76E050E0101956F0001B6EC30F0F1
:109CF0007E0E0101A16F0001C7EC2DF0200E0101C5
:109D0000A16F0001C7EC2DF09551040801E1A82BCB
:109D1000952D01D0A80795510308D8A494D16EECD5
:109D200030F0879795510308D8B45CD1EDC0EEF0C0
:109D3000ED51FF0AEE6F0101946BEEC093F100014B
:109D400049EC2EF003C0A1F102C0A0F101C09FF1C7
:109D500000C09EF1550E0101A56FC10EA46F480E03
:109D6000A36F7D0EA26F000114EC2FF003C0ECF086
:109D700002C0EBF001C0EAF000C0E9F087B785D07F
:109D8000D93D2AD0FFEC2FF0140EF66E340EF76E8C
:109D90000D0E0101956F0001B6EC30F0010EE96E79
:109DA000ECC094F1EBC093F1EAC092F1E9C091F1FB
:109DB0000101956B000174EC39F0250E0101A16FD2
:109DC0000001C7EC2DF020EC30F02A0EF66E340EB8
:109DD000F76E0BEC30F058D0D9532AE1FFEC2FF09E
:109DE0003C0EF66E340EF76E0D0E0101956F0001FC
:109DF000B6EC30F0010EE96EECC094F1EBC093F1DB
:109E0000EAC092F1E9C091F10101956B000174EC97
:109E100039F0250E0101A16F0001C7EC2DF020ECF7
:109E200030F0520EF66E340EF76E0BEC30F02CD094
:109E3000D9517F0829E1FFEC2FF0640EF66E340E45
:109E4000F76E0D0E0101956F0001B6EC30F0010EBA
:109E5000E96EECC094F1EBC093F1EAC092F1E9C075
:109E600091F10101956B000174EC39F0250E0101AF
:109E7000A16F0001C7EC2DF020EC30F07A0EF66EE9
:109E8000340EF76E0BEC30F084D0D93D2AD0FFECC5
:109E90002FF08C0EF66E340EF76E0D0E0101956FDD
:109EA0000001B6EC30F0010EE96EECC094F1EBC0AD
:109EB00093F1EAC092F1E9C091F10101956B0001C3
:109EC00074EC39F0250E0101A16F0001C7EC2DF0F3
:109ED00020EC30F0A20EF66E340EF76E0BEC30F084
:109EE00058D0D9532AE1FFEC2FF0B40EF66E340EA1
:109EF000F76E0D0E0101956F0001B6EC30F0010E0A
:109F0000E96EECC094F1EBC093F1EAC092F1E9C0C4
:109F100091F10101956B000174EC39F0250E0101FE
:109F2000A16F0001C7EC2DF020EC30F0CA0EF66EE8
:109F3000340EF76E0BEC30F02CD0D9517F0829E1AC
:109F4000FFEC2FF0DC0EF66E340EF76E0D0E0101F5
:109F5000956F0001B6EC30F0010EE96EECC094F1A3
:109F6000EBC093F1EAC092F1E9C091F10101956B68
:109F7000000174EC39F0250E0101A16F0001C7EC5E
:109F80002DF020EC30F0F20EF66E340EF76E0BEC86
:109F900030F0952D0DD08787ED2B640E0101A56F54
:109FA00000019CEC2DF0EDC091F12DEC30F019D0BA
:109FB000955104080DE18787ED07640E0101A56F37
:109FC00000019CEC2DF0EDC091F12DEC30F009D0AA
:109FD0009551050806E1010116971699169B169DE5
:109FE0000001A0D6640E0101A56F00019CEC2DF0CC
:109FF00087A728D017EC3FF0952D1FD0D250006EC8
:10A00000D29E3901E16B0C0EE06F6000B7F3E3F90B
:10A01000E59DE59FE585550EE66FAA0EE66FE583A3
:10A02000E5B3FED7E595E59DE58F0050D212EDC072
:10A0300091F100012DEC30F005D09551040801E1BB
:10A0400001D0D8D7A82B7BEF58F0879F6EEC30F06B
:10A05000FFEC2FF0040EF66E350EF76E0BEC30F0C1
:10A06000D93D28D020EC30F0160EF66E350EF76E86
:10A07000080E0101956F0001B6EC30F07F0E010172
:10A08000A16F0001C7EC2DF0200EF66E350EF76EB5
:10A09000050E0101956F0001B6EC30F07E0E010156
:10A0A000A16F0001C7EC2DF0200E0101A16F00018E
:10A0B000C7EC2DF0D95328E120EC30F02A0EF66ED3
:10A0C000350EF76E080E0101956F0001B6EC30F009
:10A0D0007F0E0101A16F0001C7EC2DF0340EF66E6A
:10A0E000350EF76E050E0101956F0001B6EC30F0EC
:10A0F0007E0E0101A16F0001C7EC2DF0200E0101C1
:10A10000A16F0001C7EC2DF0D9517F0828E120ECA8
:10A1100030F03E0EF66E350EF76E080E0101956FAB
:10A120000001B6EC30F07F0E0101A16F0001C7EC19
:10A130002DF0480EF66E350EF76E050E0101956F87
:10A140000001B6EC30F07E0E0101A16F0001C7ECFA
:10A150002DF0200E0101A16F0001C7EC2DF09551EB
:10A16000040801E1A82B952D03D0CBAE01D0A807A0
:10A17000952D04D0CBBE02D0A807A807952D09D0F5
:10A18000F92D07D0FA51030804E1020EA86F7BEF06
:10A1900058F0955103084CE16EEC30F095510308EE
:10A1A00046E0FFEC2FF0520EF66E350EF76E0BEC1C
:10A1B00030F0D93D09D020EC30F0640EF66E350E4B
:10A1C000F76E0BEC30F016D0D95309E120EC30F0EB
:10A1D000760EF66E350EF76E0BEC30F00BD0D951D3
:10A1E0007F0808E120EC30F0880EF66E350EF76E31
:10A1F0000BEC30F0952D07D088B705D001011689FA
:10A20000168B168D00019551040807E188B505D01D
:10A2100001011687168B169D00019551050806E170
:10A22000010116971699169B169D0001B7D7A82B0A
:10A23000878F7BEF58F0E85303E1A82B7BEF58F0B2
:10A240006EEC30F06F0048FF91F1D29E3901E16B66
:10A25000050EE06FE59DE59FE581E351E59DE58F06
:10A26000010191BFD28E0001CE6FCE515A0802E299
:10A27000050ECE6FD66BCEC0D5F0D93D31D0FFECF8
:10A280002FF09A0EF66E350EF76E0BEC30F020ECD8
:10A2900030F0AC0EF66E350EF76E080E0101956FBC
:10A2A0000001B6EC30F07F0E0101A16F0001C7EC98
:10A2B0002DF0B60EF66E350EF76E050E0101956F98
:10A2C0000001B6EC30F07E0E0101A16F0001C7EC79
:10A2D0002DF0200E0101A16F0001C7EC2DF066D01A
:10A2E000D95331E1FFEC2FF0C00EF66E350EF76E4C
:10A2F0000BEC30F020EC30F0D20EF66E350EF76E2F
:10A30000080E0101956F0001B6EC30F07F0E0101DF
:10A31000A16F0001C7EC2DF0DC0EF66E350EF76E66
:10A32000050E0101956F0001B6EC30F07E0E0101C3
:10A33000A16F0001C7EC2DF0200E0101A16F0001FB
:10A34000C7EC2DF033D0D9517F0830E1FFEC2FF06E
:10A35000E60EF66E350EF76E0BEC30F020EC30F0BA
:10A36000F80EF66E350EF76E080E0101956F0001BE
:10A37000B6EC30F07F0E0101A16F0001C7EC2DF0AB
:10A38000020EF66E360EF76E050E0101956F000196
:10A39000B6EC30F07E0E0101A16F0001C7EC2DF08C
:10A3A000200E0101A16F0001C7EC2DF095510408AA
:10A3B00001E1A82B952D01D0A807A85302E1010EB9
:10A3C000A86F95510308D8A452D16EEC30F0879550
:10A3D00095510308D8B414D187B57CD0D93D27D086
:10A3E000FFEC2FF00C0EF66E360EF76E080E010124
:10A3F000956F0001B6EC30F0CEC092F1130E010162
:10A40000936F0001E5EC30F0170EF66E360EF76E26
:10A41000050E0101956F0001B6EC30F020EC30F034
:10A420001E0EF66E360EF76E0BEC30F052D0D9538E
:10A4300027E1FFEC2FF0300EF66E360EF76E090EA8
:10A440000101956F0001B6EC30F0CEC092F1130E11
:10A450000101936F0001E5EC30F03C0EF66E360E14
:10A46000F76E040E0101956F0001B6EC30F020ECA0
:10A4700030F0420EF66E360EF76E0BEC30F029D04F
:10A48000D9517F0826E1FFEC2FF0540EF66E360E00
:10A49000F76E090E0101956F0001B6EC30F0CEC0E9
:10A4A00092F1130E0101936F0001E5EC30F0600EA4
:10A4B000F66E360EF76E040E0101956F0001B6ECD4
:10A4C00030F020EC30F0660EF66E360EF76E0BECC8
:10A4D00030F07BD0D93D27D0FFEC2FF0780EF66E10
:10A4E000360EF76E080E0101956F0001B6EC30F0E4
:10A4F000CEC092F1130E0101936F0001E5EC30F034
:10A50000830EF66E360EF76E050E0101956F000193
:10A51000B6EC30F020EC30F08A0EF66E360EF76EA8
:10A520000BEC30F052D0D95327E1FFEC2FF09C0E0A
:10A53000F66E360EF76E090E0101956F0001B6EC4E
:10A5400030F0CEC092F1130E0101936F0001E5ECE3
:10A5500030F0A80EF66E360EF76E040E0101956F00
:10A560000001B6EC30F020EC30F0AE0EF66E360E98
:10A57000F76E0BEC30F029D0D9517F0826E1FFECC3
:10A580002FF0C00EF66E360EF76E090E0101956FB4
:10A590000001B6EC30F0CEC092F1130E0101936FC2
:10A5A0000001E5EC30F0CC0EF66E360EF76E040EC0
:10A5B0000101956F0001B6EC30F020EC30F0D20EC6
:10A5C000F66E360EF76E0BEC30F0640E0101A56FDF
:10A5D00000019CEC2DF09551040805E18785CE51D2
:10A5E000590801E3CE2B640E0101A56F00019CEC1C
:10A5F0002DF0952D04D08785CE5301E0CE07E8D607
:10A60000640E0101A56F00019CEC2DF087A52ED0F2
:10A6100017EC3FF00A0E0101A56F00019CEC2DF034
:10A62000952D1FD0D250006ED29E3901E16B050EE0
:10A63000E06F60003BF3E3F9E59DE59FE585550E8E
:10A64000E66FAA0EE66FE583E5B3FED7E595E59DD7
:10A65000E58F0050D2120001D66BCEC0D5F006D0E7
:10A6600004D09551040801E101D0D2D7A82B7BEF8B
:10A6700058F0F92D06D0FA51030803E1A82B7BEF1F
:10A6800058F06EEC30F0D93D09D0FFEC2FF0E40E1D
:10A69000F66E360EF76E0BEC30F016D0D95309E19A
:10A6A000FFEC2FF0F60EF66E360EF76E0BEC30F078
:10A6B0000BD0D9517F0808E1FFEC2FF0080EF66EA1
:10A6C000370EF76E0BEC30F0D93D29D020EC30F08E
:10A6D0001A0EF66E370EF76E080E0101956F000127
:10A6E000B6EC30F07F0E0101A16F0001C7EC2DF038
:10A6F000240EF66E370EF76E050E0101956F000100
:10A70000B6EC30F07E0E0101A16F0001C7EC2DF018
:10A71000200E0101A16F0001C7EC2DF056D0D953D6
:10A7200029E120EC30F02E0EF66E370EF76E080E93
:10A730000101956F0001B6EC30F07F0E0101A16FB1
:10A740000001C7EC2DF0380EF66E370EF76E050ED1
:10A750000101956F0001B6EC30F07E0E0101A16F92
:10A760000001C7EC2DF0200E0101A16F0001C7EC24
:10A770002DF02BD0D9517F0828E120EC30F0420E8B
:10A78000F66E370EF76E080E0101956F0001B6ECFC
:10A7900030F07F0E0101A16F0001C7EC2DF04C0ECF
:10A7A000F66E370EF76E050E0101956F0001B6ECDF
:10A7B00030F07E0E0101A16F0001C7EC2DF0200EDC
:10A7C0000101A16F0001C7EC2DF09551040801E1D2
:10A7D000A82B952D07D0A807F92D04D0FA5103080E
:10A7E00001E1A807A85302E1010EA86F95510308E3
:10A7F000D8A451D1D93D09D0FFEC2FF0560EF66EFA
:10A80000370EF76E0BEC30F016D0D95309E1FFECA0
:10A810002FF0680EF66E370EF76E0BEC30F00BD0A3
:10A82000D9517F0808E1FFEC2FF07A0EF66E370E53
:10A83000F76E0BEC30F0D93D09D020EC30F08C0EE7
:10A84000F66E370EF76E0BEC30F016D0D95309E1E7
:10A8500020EC30F09E0EF66E370EF76E0BEC30F0FB
:10A860000BD0D9517F0808E120EC30F0B00EF66E25
:10A87000370EF76E0BEC30F06EEC30F095510308AC
:10A88000D8B4DFD0D93D09D0FFEC2FF0C20EF66E60
:10A89000370EF76E0BEC30F016D0D95309E1FFEC10
:10A8A0002FF0D40EF66E370EF76E0BEC30F00BD0A7
:10A8B000D9517F0808E1FFEC2FF0E60EF66E370E57
:10A8C000F76E0BEC30F0D93D09D020EC30F0F80EEB
:10A8D000F66E370EF76E0BEC30F01BD0D95309E152
:10A8E00020EC30F00A0EF66E380EF76E0BEC30F0FE
:10A8F00010D0D9517F0809E120EC30F01C0EF66E23
:10A90000380EF76E0BEC30F004D095510308D8B434
:10A91000BFD0952D49D06EEC30F09551050844E13B
:10A92000D93D09D0FFEC2FF02E0EF66E380EF76EE3
:10A930000BEC30F016D0D95309E1FFEC2FF0400EAC
:10A94000F66E380EF76E0BEC30F00BD0D9517F0855
:10A9500008E1FFEC2FF0520EF66E380EF76E0BEC9E
:10A9600030F0D93D09D020EC30F0640EF66E380E90
:10A97000F76E0BEC30F016D0D95309E120EC30F033
:10A98000760EF66E380EF76E0BEC30F00BD0D95118
:10A990007F0808E120EC30F0880EF66E380EF76E76
:10A9A0000BEC30F0E869B9D79551040849E16EEC39
:10A9B00030F09551050844E1D93D09D0FFEC2FF066
:10A9C0009A0EF66E380EF76E0BEC30F016D0D953A7
:10A9D00009E1FFEC2FF0AC0EF66E380EF76E0BECC3
:10A9E00030F00BD0D9517F0808E1FFEC2FF0BE0EFC
:10A9F000F66E380EF76E0BEC30F0D93D09D020EC36
:10AA000030F0D00EF66E380EF76E0BEC30F016D03C
:10AA1000D95309E120EC30F0E20EF66E380EF76EF5
:10AA20000BEC30F00BD0D9517F0808E120EC30F06E
:10AA3000F40EF66E380EF76E0BEC30F0E86BB9D70B
:10AA40001DD717EC3FF0952D1CD0D250006ED29E32
:10AA50003901E16B150EE06F6000A3F3E3F9E59DAA
:10AA6000E59FE585550EE66FAA0EE66FE583E5B333
:10AA7000FED7E595E59DE58F0050D2120AD006D0AD
:10AA800000019551040803E1390103D00001D9D731
:10AA900039010001A82B2FD3F92D05D0FA51030855
:10AAA00002E1A82B28D36EEC30F0FFEC2FF0060E5D
:10AAB000F66E390EF76E0BEC30F020EC30F0180E1D
:10AAC000F66E390EF76E080E0101956F0001B6ECB7
:10AAD00030F07F0E0101A16F0001C7EC2DF0220EB6
:10AAE000F66E390EF76E050E0101956F0001B6EC9A
:10AAF00030F07E0E0101A16F0001C7EC2DF0200E99
:10AB00000101A16F0001C7EC2DF09551040801E18E
:10AB1000A82B952D07D0A807F92D04D0FA510308CA
:10AB200001E1A807A85302E1010EA86F955103089F
:10AB3000D8A4C5D0FFEC2FF02C0EF66E390EF76EB0
:10AB40000BEC30F020EC30F03E0EF66E390EF76E66
:10AB50000BEC30F06EEC30F09551030805E1952DCB
:10AB600003D09551040862E0FFEC2FF0500EF66E12
:10AB7000390EF76E0BEC30F020EC30F0620EF66E12
:10AB8000390EF76E0BEC30F09551030819E16EECBD
:10AB900030F09551050814E1FFEC2FF0740EF66EBD
:10ABA000390EF76E0BEC30F020EC30F0860EF66EBE
:10ABB000390EF76E0BEC30F07F0ED96F37D0E9D736
:10ABC000952D18D06EEC30F09551050813E1FFEC8F
:10ABD0002FF0980EF66E390EF76E0BEC30F020EC7D
:10ABE00030F0AA0EF66E390EF76E0BEC30F0D96B22
:10ABF0001DD0EAD79551040818E16EEC30F095515C
:10AC0000050813E1FFEC2FF0BC0EF66E390EF76E5F
:10AC10000BEC30F020EC30F0CE0EF66E390EF76E05
:10AC20000BEC30F0D96902D0EAD796D7080E0101B3
:10AC3000916FFA0EA56F00019CEC2DF00101912F90
:10AC4000F8D7000117EC3FF0952D1CD0D250006EC4
:10AC5000D29E3901E16B3C0EE06F600067F3E3F9CF
:10AC6000E59DE59FE585550EE66FAA0EE66FE58347
:10AC7000E5B3FED7E595E59DE58F0050D2121DD0D6
:10AC800019D000019551040816E16F0048FF91F1B9
:10AC9000D29E3901E16B3C0EE06FE59DE59FE581B9
:10ACA000E351E59DE58F010191BFD28E0001D96F7F
:10ACB000390103D00001C6D739010001A82B1BD2EE
:10ACC0006EEC30F0D93D31D0FFEC2FF0E00EF66E97
:10ACD000390EF76E0BEC30F020EC30F0F20EF66E21
:10ACE000390EF76E080E0101956F0001B6EC30F0D9
:10ACF0007F0E0101A16F0001C7EC2DF0FC0EF66E76
:10AD0000390EF76E050E0101956F0001B6EC30F0BB
:10AD10007E0E0101A16F0001C7EC2DF0200E010194
:10AD2000A16F0001C7EC2DF066D0D95331E1FFECE3
:10AD30002FF0060EF66E3A0EF76E0BEC30F020ECAC
:10AD400030F0180EF66E3A0EF76E080E0101956F90
:10AD50000001B6EC30F07F0E0101A16F0001C7ECDD
:10AD60002DF0220EF66E3A0EF76E050E0101956F6C
:10AD70000001B6EC30F07E0E0101A16F0001C7ECBE
:10AD80002DF0200E0101A16F0001C7EC2DF033D092
:10AD9000D9517F0830E1FFEC2FF02C0EF66E3A0E01
:10ADA000F76E0BEC30F020EC30F03E0EF66E3A0E03
:10ADB000F76E080E0101956F0001B6EC30F07F0EC2
:10ADC0000101A16F0001C7EC2DF0480EF66E3A0E9E
:10ADD000F76E050E0101956F0001B6EC30F07E0EA6
:10ADE0000101A16F0001C7EC2DF0200E0101A16F40
:10ADF0000001C7EC2DF09551040801E1A82B952D19
:10AE000001D0A80795510308D8A4CAD06EEC30F041
:10AE100095510308D8B498D0FFEC2FF0520EF66E7F
:10AE20003A0EF76E0BEC30F0D93D09D020EC30F043
:10AE3000640EF66E3A0EF76E0BEC30F01BD0D95361
:10AE400009E120EC30F0760EF66E3A0EF76E0BEC60
:10AE500030F010D0D9517F0809E120EC30F0880E95
:10AE6000F66E3A0EF76E0BEC30F004D095510308F5
:10AE7000D8B496D0952D32D06EEC30F095510508AF
:10AE80002DE1FFEC2FF09A0EF66E3A0EF76E0BECFA
:10AE900030F0D93D09D020EC30F0AC0EF66E3A0E11
:10AEA000F76E0BEC30F016D0D95309E120EC30F0FE
:10AEB000BE0EF66E3A0EF76E0BEC30F00BD0D95199
:10AEC0007F0808E120EC30F0D00EF66E3A0EF76EF7
:10AED0000BEC30F00101186B0001D0D7955104083C
:10AEE00032E16EEC30F0955105082DE1FFEC2FF0CA
:10AEF000E20EF66E3A0EF76E0BEC30F0D93D09D04B
:10AF000020EC30F0F60EF66E3A0EF76E0BEC30F0E9
:10AF100016D0D95309E120EC30F0080EF66E3B0E46
:10AF2000F76E0BEC30F00BD0D9517F0808E120EC24
:10AF300030F01A0EF66E3B0EF76E0BEC30F001019E
:10AF400018690001D0D764D76EEC30F017EC3FF0F1
:10AF5000952D1CD0D250006ED29E3901E16B010EAE
:10AF6000E06F600063F4E3F9E59DE59FE585550E2C
:10AF7000E66FAA0EE66FE583E5B3FED7E595E59D9E
:10AF8000E58F0050D2120AD006D000019551040876
:10AF900003E1390103D00001D9D739010001A82B01
:10AFA0000001A9D06EEC30F0D93D31D0FFEC2FF08C
:10AFB0002C0EF66E3B0EF76E0BEC30F020EC30F002
:10AFC0003E0EF66E3B0EF76E080E0101956F000106
:10AFD000B6EC30F07F0E0101A16F0001C7EC2DF03F
:10AFE000480EF66E3B0EF76E050E0101956F0001DF
:10AFF000B6EC30F07E0E0101A16F0001C7EC2DF020
:10B00000200E0101A16F0001C7EC2DF066D0D953CD
:10B0100031E1FFEC2FF0520EF66E3B0EF76E0BECAB
:10B0200030F020EC30F0640EF66E3B0EF76E080E3A
:10B030000101956F0001B6EC30F07F0E0101A16FA8
:10B040000001C7EC2DF06E0EF66E3B0EF76E050E8E
:10B050000101956F0001B6EC30F07E0E0101A16F89
:10B060000001C7EC2DF0200E0101A16F0001C7EC1B
:10B070002DF033D0D9517F0830E1FFEC2FF0780E5E
:10B08000F66E3B0EF76E0BEC30F020EC30F08A0ED3
:10B09000F66E3B0EF76E080E0101956F0001B6ECDF
:10B0A00030F07F0E0101A16F0001C7EC2DF0940E6E
:10B0B000F66E3B0EF76E050E0101956F0001B6ECC2
:10B0C00030F07E0E0101A16F0001C7EC2DF0200EC3
:10B0D0000101A16F0001C7EC2DF09551040802E1B8
:10B0E000010EA86F952D02D00D0EA86F9551030883
:10B0F000D8B403D000D05BEF3FF0010116B703D006
:10B1000016B901D0FF003901988D000136EF59F0D2
:10B110000101966B956B946B936B9A6B996B986B23
:10B12000320E976F000150EC30F088918E6BB25365
:10B13000D8A4A1D0B353D8A49ED0B453D8A49BD044
:10B14000B553D8A498D0010116971699169B169D51
:10B15000000188B14AD0D93D16D0FFEC2FF09E0EE9
:10B16000F66E3B0EF76E0BEC30F00A0E0101A56F88
:10B1700000019CEC2DF020EC30F0B00EF66E3B0E92
:10B18000F76E0BEC30F0D95316E1FFEC2FF0C20E46
:10B19000F66E3B0EF76E0BEC30F00A0E0101A56F58
:10B1A00000019CEC2DF020EC30F0D40EF66E3B0E3E
:10B1B000F76E0BEC30F0D9517F0816E1FFEC2FF061
:10B1C000E60EF66E3B0EF76E0BEC30F00A0E010148
:10B1D000A56F00019CEC2DF020EC30F0F80EF66E1F
:10B1E0003B0EF76E0BEC30F037D0D93D10D0FFECB2
:10B1F0002FF00A0EF66E3C0EF76E0BEC30F020ECE2
:10B2000030F01C0EF66E3C0EF76E0BEC30F0D9539E
:10B2100010E1FFEC2FF02E0EF66E3C0EF76E0BECED
:10B2200030F020EC30F0400EF66E3C0EF76E0BEC7A
:10B2300030F0D9517F0810E1FFEC2FF0520EF66E7E
:10B240003C0EF76E0BEC30F020EC30F0640EF66E36
:10B250003C0EF76E0BEC30F0B25306E1B35304E151
:10B26000B45302E1B553D8A455EF3FF0955102080D
:10B27000D8A401D05CD7F0530DE10101966B956B1A
:10B28000946B936B9A6B996B986BE2C097F100018A
:10B2900050EC30F0FDEC2DF01200016603D0026698
:10B2A00002D008D0022A600003F0EEFF012EFBD787
:10B2B000022EF9D7AFEF59F00101C069BF69BC5147
:10B2C000BC07000A28E06000EFF6EAFFBA51BA2B8B
:10B2D000D8B4BB2BE96EEF50BF19BD6FC0C1BEF132
:10B2E000C0C1BFF1C06BBDC1C1F1C26BD890BD354B
:10B2F000026EC235036E025060000FF0F7FF0001CE
:10B3000059EC10F009006F00D4FF03F00101BF1BDE
:10B310000350C01BD4D7BFC101F0C0C102F000016F
:10B3200012003901A3A9FED73D01EA6F0001120006
:10B330000101945303E1000E016EA3D1D89094351E
:10B34000030F020F996F9A6BD8B09A2BEA6A7C0EA2
:10B35000E96E006A026A0A0E016E00019ED791C171
:10B360007CF0030E7D6F93C17EF0000192C17FF0EF
:10B3700000010001806B94C181F000010101BB6BF1
:10B380007C0EBA6F060EBC6F000196DF02C098F10A
:10B3900001C097F197C182F0000198C183F00001CC
:10B3A00001019F6B9F510408D8A069D10001626B15
:10B3B000616B646B636BBB84050E0101A56F0001BB
:10B3C0009CEC2DF001019C6B9B6B9C5314E19B51F9
:10B3D000070811E37C0E9B25E96E000E9C21EA6EA6
:10B3E0006F00BCFFA5F1A55100019BDF01019B2B64
:10B3F000D8B49C2BEAD73D01F9AFFED7F98F3901BC
:10B400009387BB940001626B616B050E01019E6F17
:10B41000DC0E9D6F9D519E1119E0000162510101EA
:10B420009A5D14E308E199510001615DD8A002D052
:10B4300001010CD00101010EA56F00019CEC2DF063
:10B4400001019D51D8B49E079D07E4D73901939718
:10B450000001625101019A5D0AE308E1995100017E
:10B46000615DD8A002D0010102D0010106D19A513C
:10B470000001625D12E305E1010199510001615D86
:10B480000CE3010199510001615D006E01019A51C7
:10B4900000016259036E005002D0036A000E0101E0
:10B4A000A26F03C0A3F1A46BA16BA06BA151A35D1C
:10B4B000D8A0DDD004E1A051A25DD8A0D8D0210E43
:10B4C000A025E96E000EA121EA6E9151EF5CD8A48F
:10B4D000CAD0010EA025A56F000EA121A66F210ED6
:10B4E000A525E96E000EA621EA6EEF500308D8A448
:10B4F000BAD0020EA025A56F000EA121A66F210EC5
:10B50000A525E96E000EA621EA6E6F00BCFFA7F12B
:10B51000D8909435A75DD8A4A6D0210EA025016EA1
:10B52000000EA121036E01C0A5F1A66F020E995D68
:10B53000A76F000E9A59A86F03C0BBF101C0BAF102
:10B54000A7C1BCF10001B8DE02C098F101C097F1BB
:10B5500097C1A5F101019951A025A66F9A51A1218A
:10B56000A76F020EA65F000EA75B210EA625E96E4F
:10B57000000EA721EA6EEF50975DD8A474D098C151
:10B58000A5F19951A025A66F9A51A121A76F010E8F
:10B59000A65F000EA75B210EA625E96E000EA7216F
:10B5A000EA6EEF50A55DD8A45ED09551961154E097
:10B5B0009C6B9B6B9C5350E194519B5D4DE2D890EA
:10B5C0009B35026E9C35036E02509525016E965197
:10B5D000032203C0A6F1030EA025A76F000EA12130
:10B5E000A86FD8909B35026E9C35036E0250A7273A
:10B5F0000350A823210EA725E96E000EA821EA6EAC
:10B600006F00BCFFA9F1040EA025AA6F000EA121B6
:10B61000AB6FD8909B35026E9C35036E0250AA2703
:10B620000350AB23210EAA25E96E000EAB21EA6E72
:10B630006F00BCFFACF160009BF6EAFF600007F012
:10B64000E9FF6000A7F6ECFFED526000B3F6EFFFF4
:10B650009B2BD8B49C2BAED7010EA46F0001626B5C
:10B66000616B010104D0A02BD8B4A12B1FD7A45328
:10B67000D8B403D0010E016E04D09F2B93D6000ED8
:10B68000016E00011200010192BF12D00F0E006E78
:10B69000913900160A0E005C03E2300E002602D03B
:10B6A0009251002600C0A1F10001C7EC2DF001016C
:10B6B0000F0E91170A0E915D02E2300E02D0929F9A
:10B6C0009251912791C1A1F10001C7EC2DF0120018
:10B6D000010E656F91C192F1100E0101936F946B91
:10B6E000956B966B0E0E976F1C0E986FB96BB951D8
:10B6F0000A0846E3D890B935070F036A920F016E26
:10B70000010E032203C0BBF1D890B935036A1C0FA8
:10B71000E96E010E0320EA6E6F00B0FFBDF1ED523D
:10B720006F00BCFFBCF16000EFF6EAFF600007F0BD
:10B73000E9FF6000F7F6EFFFD890B935080F036A0C
:10B74000920F016E010E032203C0BBF1D890B935F0
:10B75000036A1C0FE96E010E0320EA6E6F00B0FF52
:10B76000BDF1ED526F00BCFFBCF16000EFF6EAFFE7
:10B77000600007F0E9FF6000F3F6EFFFB92BB7D7E1
:10B78000AF6B1BC0B0F1B16B1DC0B2F1B36B1FC08A
:10B79000B4F1010EBB6F920EBA6F230EBC6F0001A5
:10B7A0008BDD02C0B8F101C0B7F1B7C1B5F101013D
:10B7B000B851B66FBB843D01F98F0101B96BB95126
:10B7C000240810E3036AB951920FE96E010E0320B9
:10B7D000EA6E6F00BCFFBAF1BA510001A2DD0101AF
:10B7E000B92BEDD73D01F9AFFED7F98FBB9400011E
:10B7F000120069A308D00101916B000169DF69A300
:10B8000002D06993FCD71200FFEC2FF0C00EF66E49
:10B81000220EF76E030E0101956F0001B6EC30F0B9
:10B820009FC0A1F1C7EC2DF0A0C0A1F1C7EC2DF095
:10B83000A1C0A1F1C7EC2DF0A2C0A1F1C7EC2DF081
:10B84000A3C0A1F1C7EC2DF0A4C0A1F1C7EC2DF06D
:10B85000A5C0A1F1C7EC2DF0A6C0A1F1C7EC2DF059
:10B86000D30EF66E220EF76E050E0101956F0001E4
:10B87000B6EC30F01200F55322E101011053D8A4C8
:10B8800002D000011CD00001FFEC2FF0500EF66E2C
:10B89000420EF76E0BEC30F020EC30F0620EF66EDC
:10B8A000420EF76E0BEC30F0BC96BC94BC92BC9090
:10B8B000010116971699169B169D0001DCD7120000
:10B8C000FE5303E02F0E966F02D07C0E966F01019F
:10B8D000005305E02F0E0001976F04D001017C0E8C
:10B8E0000001976F0101025305E02F0E0001986FD0
:10B8F00004D001017C0E0001986F0101045305E0A2
:10B900002F0E0001996F04D001017C0E0001996F88
:10B910000101065305E02F0E00019A6F04D00101CA
:10B920007C0E00019A6F0101085305E02F0E000103
:10B930009B6F04D001017C0E00019B6F01010A5333
:10B9400005E02F0E00019C6F04D001017C0E000168
:10B950009C6F01010C5305E02F0E00019D6F04D078
:10B9600001017C0E00019D6FCBAE03D02F0E9E6FA8
:10B9700002D07C0E9E6FF63D55D0F4AF03D07C0E06
:10B980009F6F02D02F0E9F6F010116A105D07C0E74
:10B990000001A06F04D001012F0E0001A06F010172
:10B9A00016A305D07C0E0001A16F04D001012F0E5B
:10B9B0000001A16F010116A505D07C0E0001A26F48
:10B9C00004D001012F0E0001A26F010116A705D0BE
:10B9D0007C0E0001A36F04D001012F0E0001A36FA4
:10B9E000010116A905D07C0E0001A46F04D001014D
:10B9F0002F0E0001A46F010116AB05D07C0E0001D3
:10BA0000A56F04D001012F0E0001A56F010116AD35
:10BA100005D07C0E0001A66F04D001012F0E00019D
:10BA2000A66F54D0F4AF03D07C0E9F6F02D02F0EC0
:10BA30009F6F010116A105D07C0E0001A06F04D0FC
:10BA400001012F0E0001A06F010116A305D07C0E8D
:10BA50000001A16F04D001012F0E0001A16F0101AF
:10BA600016A505D07C0E0001A26F04D001012F0E97
:10BA70000001A26F010116A705D07C0E0001A36F83
:10BA800004D001012F0E0001A36F010116A905D0FA
:10BA90007C0E0001A46F04D001012F0E0001A46FE1
:10BAA000010116AB05D07C0E0001A56F04D0010189
:10BAB0002F0E0001A56F010116AD05D07C0E00010F
:10BAC000A66F04D001012F0E0001A66F120020EC1A
:10BAD00030F0DA0EF66E220EF76E030E0101956F4E
:10BAE0000001B6EC30F096C0A1F1C7EC2DF097C084
:10BAF000A1F1C7EC2DF098C0A1F1C7EC2DF099C0D1
:10BB0000A1F1C7EC2DF09AC0A1F1C7EC2DF09BC0BC
:10BB1000A1F1C7EC2DF09CC0A1F1C7EC2DF09DC0A8
:10BB2000A1F1C7EC2DF0ED0EF66E220EF76E050EAC
:10BB30000101956F0001B6EC30F01200952D74D024
:10BB400069A93BD020EC30F0740EF66E420EF76E11
:10BB5000030E0101956F0001B6EC30F096C0A1F123
:10BB6000C7EC2DF097C0A1F1C7EC2DF098C0A1F162
:10BB7000C7EC2DF099C0A1F1C7EC2DF09AC0A1F14E
:10BB8000C7EC2DF09BC0A1F1C7EC2DF09CC0A1F13A
:10BB9000C7EC2DF09DC0A1F1C7EC2DF0870EF66E1D
:10BBA000420EF76E040E0101956F0001B6EC30F005
:10BBB0009EC0A1F1C7EC2DF036D020EC30F08E0EF7
:10BBC000F66E420EF76E030E0101956F0001B6ECA2
:10BBD00030F096C0A1F1C7EC2DF097C0A1F1C7ECF1
:10BBE0002DF098C0A1F1C7EC2DF099C0A1F1C7ECE0
:10BBF0002DF09AC0A1F1C7EC2DF09BC0A1F1C7ECCC
:10BC00002DF09CC0A1F1C7EC2DF09DC0A1F1C7ECB7
:10BC10002DF0A10EF66E420EF76E050E0101956F26
:10BC20000001B6EC30F0F0DD706B716BFE53D8B4F0
:10BC3000B5D0D6C093F1D5C092F10101956B0A0E33
:10BC4000946F000136EC2EF002C092F101C091F128
:10BC50000101966B956B946B936B9A6B996B02C019
:10BC600098F101C097F1000150EC30F004DE0101C1
:10BC700016971699169B169D0001F487952D01D0F5
:10BC800089D0D93D23D0772D11D0FFEC2FF0A80E0D
:10BC9000F66E420EF76E0BEC30F020EC30F0BA0E80
:10BCA000F66E420EF76E0BEC30F010D0FFEC2FF07A
:10BCB000CC0EF66E420EF76E0BEC30F020EC30F04E
:10BCC000DE0EF66E420EF76E0BEC30F0D95310E13B
:10BCD000FFEC2FF0F00EF66E420EF76E0BEC30F02C
:10BCE00020EC30F0020EF66E430EF76E0BEC30F0E7
:10BCF000D9517F0810E1FFEC2FF0140EF66E430EC1
:10BD0000F76E0BEC30F020EC30F0260EF66E430EA2
:10BD1000F76E0BEC30F00101916B0001D9DC320EB3
:10BD20000101A56F00019CEC2DF0050E0101916F42
:10BD3000936B030E926F010E946F966B780E956F56
:10BD4000000198EC59F0015224E079C076F078C0F7
:10BD500077F0772D1ED0D250006ED29E3901E16B64
:10BD6000020EE06FE36BE59DE59FE585550EE66FFE
:10BD7000AA0EE66FE583E5B3FED7E595E59DE58F71
:10BD80000050D212640E0101A56F00019CEC2DF051
:10BD9000FF0003D095DD38DD9ADE48D71200E95068
:10BDA0000101996F3B0EA06F9A0E9F6FCA0E9E6F96
:10BDB0009D6B0A0E9B6FD882010EEA6E950EE96E9E
:10BDC000196AD2BE198ED29E98C1CAF197C1C9F123
:10BDD00096C1C8F195C1C7F1A0C1CEF19FC1CDF107
:10BDE0009EC1CCF19DC1CBF10001D7EC24F019BE6E
:10BDF000D28E0150005213E101019B51010AD8A4D7
:10BE000002D000010CD099510CE00F0B9B5D01E0BA
:10BE100010E299BF0ED099BD04D0200E03D00101CD
:10BE2000996B300E002600C0A1F10001C7EC2DF087
:10BE30000101D892196AD2BE198ED29EA0C1CAF150
:10BE40009FC1C9F19EC1C8F19DC1C7F1CE6BCD6B39
:10BE5000CC6B0A0ECB6F0001D7EC24F019BED28E4A
:10BE600003C0A0F102C09FF101C09EF100C09DF18E
:10BE700001019B2FA0D700011200EF5215E06F00C7
:10BE8000A8FF92F16F00A4FF91F16F00BCFFA1F138
:10BE9000C7EC2DF060004BF6EAFF600047F6E9FFC3
:10BEA000E92AD8B4EA2AE9D71200016A026A006ACC
:10BEB000036A0101965102E1955118E0100E976F47
:10BEC000D89093379437003603369651035C02E1DD
:10BED0009551005C07E39551005ED8A0030696518A
:10BEE000035ED88001360236972FEAD70001120090
:10BEF0006F00A8FF9BF16F00A4FF9AF10101943934
:10BF0000F009966F9627E20F976F320F996F945151
:10BF10000F0B972797279927E90F986F982798274E
:10BF200093390F0B9827992798379937991F993785
:10BF300093510F0B99279637070E956F0A0E9807A6
:10BF40009927FDE397079827FDE396079727FDE3D9
:10BF500095079627FDE3010EEA6E950EE96E070E32
:10BF60009A159A9DE926000EEA22E950990803E104
:10BF7000EA2C01D09A8DEF50006E08E19ABD06D0F0
:10BF80009AB91AD09AB702D0200E03D09A879A99FC
:10BF9000300E00266F00A8FF94F16F00A4FF93F10C
:10BFA00000C0A1F10001C7EC2DF0600053F6EAFFDC
:10BFB00060004FF6E9FF0101EE509AADD6D70001BF
:10BFC00012008F6B95510308D8A4E6EF63F08789C0
:10BFD0008F51080801E28F6B010116971699169B85
:10BFE000169D0001878F8F5118E0010A42E0030A75
:10BFF000D8B491D0010AD8B458D1070AD8B4BAD16C
:10C00000010AD8B42AD2030AD8B4ABD2010AD8B4F0
:10C010001BD30F0AD8B43ED36ED3FFEC2FF03A0EE9
:10C02000F66E450EF76E0BEC30F0D93D11D020ECDA
:10C0300030F04C0EF66E450EF76E0B0E0101956F4B
:10C040000001B6EC30F0EA6A1B0EE96E16DF10D084
:10C0500020EC30F05A0EF66E450EF76E0B0E010115
:10C06000956F0001B6EC30F0EA6A1B0EE96E05DF51
:10C0700042D3D9517F0809E1FFEC2FF0680EF66E2C
:10C08000450EF76E0BEC30F008D0FFEC2FF07A0E77
:10C09000F66E450EF76E0BEC30F0D93D12D088B934
:10C0A00020EC30F08C0EF66E450EF76E0BEC30F097
:10C0B00088A920EC30F09E0EF66E450EF76E0BEC64
:10C0C00030F0D95312E188B920EC30F0B00EF66EA2
:10C0D000450EF76E0BEC30F088A920EC30F0C20E64
:10C0E000F66E450EF76E0BEC30F0D9517F0812E179
:10C0F00088B920EC30F0D40EF66E450EF76E0BECDE
:10C1000030F088A920EC30F0E60EF66E450EF76EA2
:10C110000BEC30F0F0D2D9517F0809E1FFEC2FF0A1
:10C12000F80EF66E450EF76E0BEC30F008D0FFEC13
:10C130002FF00A0EF66E460EF76E0BEC30F0D93D7E
:10C140003AD020EC30F0D6C093F1D5C092F1010185
:10C15000956B0A0E946F000136EC2EF002C092F13E
:10C1600001C091F102C094F101C093F10101966BFD
:10C170000A0E956F000199DE02C092F101C091F1A3
:10C180001C0EF66E460EF76E0A0E0101956F000149
:10C19000B6EC30F0030EE96E92C194F191C193F1C7
:10C1A000A7DE2A0EF66E460EF76E040E0101956F9D
:10C1B0000001B6EC30F0D9533AE120EC30F0D6C0B3
:10C1C00093F1D5C092F10101956B0A0E946F0001B5
:10C1D00036EC2EF002C092F101C091F102C094F150
:10C1E00001C093F10101966B0A0E956F00015DDEAF
:10C1F00002C092F101C091F1300EF66E460EF76E5C
:10C200000A0E0101956F0001B6EC30F0030EE96EE5
:10C2100092C194F191C193F16BDE3E0EF66E460E23
:10C22000F76E040E0101956F0001B6EC30F0D951A4
:10C230007F083AE120EC30F0D6C093F1D5C092F1FE
:10C240000101956B0A0E946F000136EC2EF002C0CE
:10C2500092F101C091F102C094F101C093F101018A
:10C26000966B0A0E956F000120DE02C092F101C0AC
:10C2700091F1440EF66E460EF76E0A0E0101956FAF
:10C280000001B6EC30F0030EE96E92C194F191C159
:10C2900093F12EDE520EF66E460EF76E040E01017D
:10C2A000956F0001B6EC30F026D2D93D1FD0FFECDF
:10C2B0002FF0580EF66E460EF76E0BEC30F020ECB9
:10C2C00030F06A0EF66E460EF76E0B0E0101956F9A
:10C2D0000001B6EC30F0050EE96ECDC098F1CCC08F
:10C2E00097F1CBC096F1CAC095F159DDD9531FE142
:10C2F000FFEC2FF07A0EF66E460EF76E0BEC30F078
:10C3000020EC30F08C0EF66E460EF76E0B0E01012F
:10C31000956F0001B6EC30F0050EE96ECDC098F1D6
:10C32000CCC097F1CBC096F1CAC095F138DDD95198
:10C330007F081FE1FFEC2FF09C0EF66E460EF76EA5
:10C340000BEC30F020EC30F0AE0EF66E460EF76ED1
:10C350000B0E0101956F0001B6EC30F0050EE96E91
:10C36000CDC098F1CCC097F1CBC096F1CAC095F181
:10C3700016DDC1D1F05337E1D93D10D0FFEC2FF0DD
:10C38000BE0EF66E460EF76E0BEC30F020EC30F081
:10C39000D00EF66E460EF76E0BEC30F0D95310E16E
:10C3A000FFEC2FF0E20EF66E460EF76E0BEC30F05F
:10C3B00020EC30F0F40EF66E460EF76E0BEC30F01B
:10C3C000D9517F0810E1FFEC2FF0060EF66E470EF4
:10C3D000F76E0BEC30F020EC30F0180EF66E470ED6
:10C3E000F76E0BEC30F0F03D37D0D93D10D0FFECBC
:10C3F0002FF02A0EF66E470EF76E0BEC30F020ECA5
:10C4000030F03C0EF66E470EF76E0BEC30F0D95361
:10C4100010E1FFEC2FF04E0EF66E470EF76E0BECB0
:10C4200030F020EC30F0600EF66E470EF76E0BEC3D
:10C4300030F0D9517F0810E1FFEC2FF0720EF66E4C
:10C44000470EF76E0BEC30F020EC30F0840EF66EF9
:10C45000470EF76E0BEC30F04ED169B901D04BD1DD
:10C46000CBAE7ED0EDC0EEF0ED51FF0AEE6F0101D4
:10C47000946BEEC093F1000149EC2EF003C0A1F1E2
:10C4800002C0A0F101C09FF100C09EF1550E010154
:10C49000A56FC10EA46F480EA36F7D0EA26F0001A1
:10C4A00014EC2FF003C0ECF002C0EBF001C0EAF096
:10C4B00000C0E9F0D9517F082AE1FFEC2FF0960E79
:10C4C000F66E470EF76E0BEC30F020EC30F0A80E55
:10C4D000F66E470EF76E0D0E0101956F0001B6EC7A
:10C4E00030F0010EE96EECC094F1EBC093F1EAC0BC
:10C4F00092F1E9C091F10101956B000174EC39F002
:10C50000250E0101A16F0001C7EC2DF029D0FFEC31
:10C510002FF0BE0EF66E470EF76E0BEC30F020ECEF
:10C5200030F0D00EF66E470EF76E0D0E0101956FCE
:10C530000001B6EC30F0010EE96EECC094F1EBC0F6
:10C5400093F1EAC092F1E9C091F10101956B00010C
:10C5500074EC39F0250E0101A16F0001C7EC2DF03C
:10C56000CAD0F15337E1D93D10D0FFEC2FF0E60EE1
:10C57000F66E470EF76E0BEC30F020EC30F0F80E54
:10C58000F66E470EF76E0BEC30F0D95310E1FFEC6E
:10C590002FF00A0EF66E480EF76E0BEC30F020EC22
:10C5A00030F01C0EF66E480EF76E0BEC30F0D951E1
:10C5B0007F0810E1FFEC2FF02E0EF66E480EF76E9E
:10C5C0000BEC30F020EC30F0400EF66E480EF76EBB
:10C5D0000BEC30F0F13D37D0D93D10D0FFEC2FF00F
:10C5E000520EF66E480EF76E0BEC30F020EC30F089
:10C5F000640EF66E480EF76E0BEC30F0D95310E176
:10C60000FFEC2FF0760EF66E480EF76E0BEC30F066
:10C6100020EC30F0880EF66E480EF76E0BEC30F022
:10C62000D9517F0810E1FFEC2FF09A0EF66E480EFC
:10C63000F76E0BEC30F020EC30F0AC0EF66E480EDE
:10C64000F76E0BEC30F057D0F55311E1FFEC2FF003
:10C65000BE0EF66E480EF76E0BEC30F020EC30F0AC
:10C66000D00EF66E480EF76E0BEC30F012D0F53DA2
:10C6700010D0FFEC2FF0E20EF66E480EF76E0BECCA
:10C6800030F020EC30F0F40EF66E480EF76E0BEC46
:10C6900030F031D0D93D16D0010117BF02D00001D2
:10C6A00011D00001FFEC2FF0060EF66E490EF76E6A
:10C6B0000BEC30F020EC30F0180EF66E490EF76EF1
:10C6C0000BEC30F0D95316E1010117BF02D0000185
:10C6D00011D00001FFEC2FF02A0EF66E490EF76E16
:10C6E0000BEC30F020EC30F03C0EF66E490EF76E9D
:10C6F0000BEC30F000D00101966B956B946B936B53
:10C700009A6B996B986B0A0E976F000150EC30F0A2
:10C71000B2530FE1B3530DE1B4530BE1B55309E14B
:10C7200095510308D8A405D039015B5104000001DC
:10C73000EFD78F5107082EE0FFEC2FF04E0EF66E6C
:10C74000490EF76E0BEC30F020EC30F0600EF66E18
:10C75000490EF76E0BEC30F00101966B956B946B04
:10C76000936B9A6B996B986B050E976F000150EC69
:10C7700030F0B2530FE1B3530DE1B4530BE1B553B5
:10C7800009E195510308D8A405D039015B51040093
:10C790000001EFD78F2B69B904D08F51050801E153
:10C7A0008F2BF0530DE10101966B956B946B936B9E
:10C7B0009A6B996B986BE2C097F1000150EC30F0E6
:10C7C00095510308D8A402D0E2EF5FF012000101F6
:10C7D000045308E10001F53D01D002D0010102D06F
:10C7E0000AD001010E53D8B4D2D00001F553D8B409
:10C7F00002D00101CCD0F4AF05D0F53D03D001014A
:10C80000C6D00001F5531DE101010E5318E00001EF
:10C81000FFEC2FF0380EF66E430EF76E0BEC30F097
:10C8200020EC30F04A0EF66E430EF76E0BEC30F053
:10C83000010116971699169B169D1785E8D7A6D065
:10C840000001010116971699000160EC5CF0FE539F
:10C8500009E10101105303E00001F55303E0000179
:10C86000952D02D09EEC5DF09551020802E188EC16
:10C8700058F0952D01D003D09551070841E169A9E1
:10C880003BD020EC30F05C0EF66E430EF76E030EDC
:10C890000101956F0001B6EC30F096C0A1F1C7EC34
:10C8A0002DF097C0A1F1C7EC2DF098C0A1F1C7EC15
:10C8B0002DF099C0A1F1C7EC2DF09AC0A1F1C7EC01
:10C8C0002DF09BC0A1F1C7EC2DF09CC0A1F1C7ECED
:10C8D0002DF09DC0A1F1C7EC2DF06F0EF66E430E4A
:10C8E000F76E040E0101956F0001B6EC30F09EC0AA
:10C8F000A1F1C7EC2DF002D067EC5DF004EC5CF028
:10C90000952D03D09551070840E0D93D13D0952DC2
:10C9100001D010D0FFEC2FF0760EF66E430EF76EBE
:10C920000BEC30F020EC30F0880EF66E430EF76E14
:10C930000BEC30F0D95313E1952D01D010D0FFEC62
:10C940002FF09A0EF66E430EF76E0BEC30F020ECE3
:10C9500030F0AC0EF66E430EF76E0BEC30F0D951A2
:10C960007F0813E1952D01D010D0FFEC2FF0BE0E03
:10C97000F66E430EF76E0BEC30F020EC30F0D00E7C
:10C98000F66E430EF76E0BEC30F0010121D700017B
:10C990001200D93D08D020EC30F01A0EF66E420E8F
:10C9A000F76E0BEC30F0D95308E120EC30F02C0E90
:10C9B000F66E420EF76E0BEC30F0D9517F0808E1AD
:10C9C00020EC30F03E0EF66E420EF76E0BEC30F0BF
:10C9D0001200FEC015F101010251010A006ED8904B
:10C9E0000036005015130635006E0036FC0E00169A
:10C9F000005015130835006E00360036F80E00168C
:10CA0000005015130A39006EF00E00160050151371
:10CA1000000169A90ED0000ECBBE010E010A006E06
:10CA2000003A0036E00E001600500101151303D045
:10CA300000010101159B159D159F1551000A00016C
:10CA4000D8B4BED0010AD8B4B6D1030AD8B4BDD187
:10CA5000010AD8B4C4D1070AD8B4CBD1010AD8B4DA
:10CA6000D2D1030AD8B4D9D1010AD8B4E7D10F0A78
:10CA7000D8B4EED1010AD8B4F5D1030AD8B4FCD1A8
:10CA8000010AD8B403D2070AD8B40AD2010AD8B42A
:10CA900011D2030AD8B418D2010AD8B41FD21F0A7F
:10CAA000D8B426D2010AD8B42DD2030AD8B434D2CD
:10CAB000010AD8B43BD2070AD8B442D2010AD8B48A
:10CAC00049D2030AD8B450D2010AD8B457D20F0AB7
:10CAD000D8B45ED2010AD8B465D2030AD8B46CD2F5
:10CAE000010AD8B473D2070AD8B47AD2010AD8B4EA
:10CAF00081D2030AD8B488D2010AD8B48FD23F0AAF
:10CB0000D8B496D2010AD8B49DD2030AD8B4A4D21C
:10CB1000010AD8B4ABD2070AD8B4B2D2010AD8B449
:10CB2000B9D2030AD8B4C0D2010AD8B4C7D20F0A06
:10CB3000D8B4CED2010AD8B4D5D2030AD8B4DCD244
:10CB4000010AD8B4E3D2070AD8B4EAD2010AD8B4A9
:10CB5000F1D2030AD8B4F8D2010AD8B4FFD21F0A1E
:10CB6000D8B406D3010AD8B40DD3030AD8B415D368
:10CB7000010AD8B41DD3070AD8B425D3010AD8B402
:10CB80002DD3030AD8B435D3010AD8B43DD30F0A44
:10CB9000D8B445D3010AD8B44DD3030AD8B455D379
:10CBA000010AD8B45DD3070AD8B465D3010AD8B452
:10CBB0006DD3030AD8B475D3010AD8B47DD387D313
:10CBC000D93D51D0FFEC2FF0120EF66E3D0EF76EF0
:10CBD0000BEC30F020EC30F0AA51AE5D0101916F0A
:10CBE0000001AB51AF590101926F0001AC51B05936
:10CBF0000101936F0001AD51B1590101946FD892B9
:10CC0000196AD2BE198ED29ECA6F93C1C9F192C160
:10CC1000C8F191C1C7F1CE6BCD6BCC6B0A0ECB6F57
:10CC20000001D7EC24F019BED28E03C094F102C0EB
:10CC300093F101C092F100C091F1240EF66E3D0E09
:10CC4000F76E0D0E0101956F0001B6EC30F0030E8A
:10CC5000E96E94C198F193C197F192C196F191C197
:10CC600095F1CFEC5EF0D95351E1FFEC2FF0360E89
:10CC7000F66E3D0EF76E0BEC30F020EC30F0AA5162
:10CC8000AE5D0101916F0001AB51AF590101926F8F
:10CC90000001AC51B0590101936F0001AD51B15980
:10CCA0000101946FD892196AD2BE198ED29ECA6FB2
:10CCB00093C1C9F192C1C8F191C1C7F1CE6BCD6BDF
:10CCC000CC6B0A0ECB6F0001D7EC24F019BED28ECC
:10CCD00003C094F102C093F101C092F100C091F140
:10CCE000480EF66E3D0EF76E0D0E0101956F0001B8
:10CCF000B6EC30F0030EE96E94C198F193C197F150
:10CD000092C196F191C195F1CFEC5EF0D9517F08B7
:10CD100051E1FFEC2FF05A0EF66E3D0EF76E0BEC64
:10CD200030F020EC30F0AA51AE5D0101916F0001AE
:10CD3000AB51AF590101926F0001AC51B0590101E3
:10CD4000936F0001AD51B1590101946FD892196AE6
:10CD5000D2BE198ED29ECA6F93C1C9F192C1C8F1D9
:10CD600091C1C7F1CE6BCD6BCC6B0A0ECB6F0001BE
:10CD7000D7EC24F019BED28E03C094F102C093F117
:10CD800001C092F100C091F16C0EF66E3D0EF76E8F
:10CD90000D0E0101956F0001B6EC30F0030EE96E47
:10CDA00094C198F193C197F192C196F191C195F117
:10CDB000CFEC5EF0A8D2FFEC2FF07E0EF66E3D0EAB
:10CDC000F76E0BEC30F0E5DD9ED2FFEC2FF0900E0D
:10CDD000F66E3D0EF76E0BEC30F0DBDD94D2FFEC1F
:10CDE0002FF0A20EF66E3D0EF76E0BEC30F0D1DD9B
:10CDF0008AD2FFEC2FF0B40EF66E3D0EF76E0BEC00
:10CE000030F0C7DD80D2FFEC2FF0C60EF66E3D0E7F
:10CE1000F76E0BEC30F0BDDD76D2FFEC2FF0D80EC4
:10CE2000F66E3D0EF76E0BEC30F020EC30F0EA0EB3
:10CE3000F66E3D0EF76E0BEC30F065D2FFEC2FF086
:10CE4000FC0EF66E3D0EF76E0BEC30F0A2DD5BD201
:10CE5000FFEC2FF00E0EF66E3E0EF76E0BEC30F080
:10CE600098DD51D2FFEC2FF0200EF66E3E0EF76EDD
:10CE70000BEC30F08EDD47D2FFEC2FF0320EF66E69
:10CE80003E0EF76E0BEC30F084DD3DD2FFEC2FF060
:10CE9000440EF66E3E0EF76E0BEC30F07ADD33D2B8
:10CEA000FFEC2FF0560EF66E3E0EF76E0BEC30F0E8
:10CEB00070DD29D2FFEC2FF0680EF66E3E0EF76E95
:10CEC0000BEC30F066DD1FD2FFEC2FF07A0EF66E21
:10CED0003E0EF76E0BEC30F05CDD15D2FFEC2FF060
:10CEE0008C0EF66E3E0EF76E0BEC30F052DD0BD270
:10CEF000FFEC2FF09E0EF66E3E0EF76E0BEC30F050
:10CF000048DD01D2FFEC2FF0B00EF66E3E0EF76E4C
:10CF10000BEC30F03EDDF7D1FFEC2FF0C20EF66ED9
:10CF20003E0EF76E0BEC30F034DDEDD1FFEC2FF060
:10CF3000D40EF66E3E0EF76E0BEC30F02ADDE3D128
:10CF4000FFEC2FF0E60EF66E3E0EF76E0BEC30F0B7
:10CF500020DDD9D1FFEC2FF0F80EF66E3E0EF76E05
:10CF60000BEC30F016DDCFD1FFEC2FF00A0EF66E91
:10CF70003F0EF76E0BEC30F00CDDC5D1FFEC2FF05F
:10CF80001C0EF66E3F0EF76E0BEC30F002DDBBD1DF
:10CF9000FFEC2FF02E0EF66E3F0EF76E0BEC30F01E
:10CFA000F8DCB1D1FFEC2FF0400EF66E3F0EF76EBD
:10CFB0000BEC30F0EEDCA7D1FFEC2FF0520EF66E4A
:10CFC0003F0EF76E0BEC30F0E4DC9DD1FFEC2FF060
:10CFD000640EF66E3F0EF76E0BEC30F0DADC93D198
:10CFE000FFEC2FF0760EF66E3F0EF76E0BEC30F086
:10CFF000D0DC89D1FFEC2FF0880EF66E3F0EF76E75
:10D000000BEC30F0C6DC7FD1FFEC2FF09A0EF66E01
:10D010003F0EF76E0BEC30F0BCDC75D1FFEC2FF05F
:10D02000AC0EF66E3F0EF76E0BEC30F0B2DC6BD14F
:10D03000FFEC2FF0BE0EF66E3F0EF76E0BEC30F0ED
:10D04000A8DC61D1FFEC2FF0D00EF66E3F0EF76E2C
:10D050000BEC30F09EDC57D1FFEC2FF0E20EF66EB9
:10D060003F0EF76E0BEC30F094DC4DD1FFEC2FF05F
:10D07000F40EF66E3F0EF76E0BEC30F08ADC43D107
:10D08000FFEC2FF0060EF66E400EF76E0BEC30F054
:10D0900080DC39D1FFEC2FF0180EF66E400EF76EE3
:10D0A0000BEC30F076DC2FD1FFEC2FF02A0EF66E71
:10D0B000400EF76E0BEC30F06CDC25D1FFEC2FF05E
:10D0C0003C0EF66E400EF76E0BEC30F062DC1BD1BE
:10D0D000FFEC2FF04E0EF66E400EF76E0BEC30F0BC
:10D0E00058DC11D1FFEC2FF0600EF66E400EF76E9B
:10D0F0000BEC30F04EDC07D1FFEC2FF0720EF66E29
:10D10000400EF76E0BEC30F044DCFDD0FFEC2FF05E
:10D11000840EF66E400EF76E0BEC30F03ADCF3D076
:10D12000FFEC2FF0960EF66E400EF76E0BEC30F023
:10D1300030DCE9D0FFEC2FF0A80EF66E400EF76E53
:10D140000BEC30F026DCDFD0FFEC2FF0BA0EF66EE1
:10D15000400EF76E0BEC30F01CDCD5D0FFEC2FF05E
:10D16000CC0EF66E400EF76E0BEC30F012DCCBD02E
:10D17000FFEC2FF0DE0EF66E400EF76E0BEC30F08B
:10D1800008DCC1D0FFEC2FF0F00EF66E400EF76E0B
:10D190000BEC30F0C9EC64F0B6D0FFEC2FF0020ECF
:10D1A000F66E410EF76E0BEC30F0C9EC64F0ABD0CC
:10D1B000FFEC2FF0140EF66E410EF76E0BEC30F014
:10D1C000C9EC64F0A0D0FFEC2FF0260EF66E410EF5
:10D1D000F76E0BEC30F0C9EC64F095D0FFEC2FF05B
:10D1E000380EF66E410EF76E0BEC30F0C9EC64F0C1
:10D1F0008AD0FFEC2FF0440EF66E410EF76E0BEC6A
:10D2000030F0C9EC64F07FD0FFEC2FF0560EF66ED4
:10D21000410EF76E0BEC30F0C9EC64F074D0FFEC0B
:10D220002FF0680EF66E410EF76E0BEC30F0C9EC85
:10D2300064F069D0FFEC2FF07A0EF66E410EF76EB7
:10D240000BEC30F0C9EC64F05ED0FFEC2FF08C0EEC
:10D25000F66E410EF76E0BEC30F0C9EC64F053D073
:10D26000FFEC2FF09E0EF66E410EF76E0BEC30F0D9
:10D27000C9EC64F048D0FFEC2FF0B00EF66E410E12
:10D28000F76E0BEC30F0C9EC64F03DD0FFEC2FF002
:10D29000C20EF66E410EF76E0BEC30F0C9EC64F086
:10D2A00032D0FFEC2FF0D40EF66E410EF76E0BEC81
:10D2B00030F0C9EC64F027D0FFEC2FF0E40EF66EEE
:10D2C000410EF76E0BEC30F0C9EC64F01CD0FFECB3
:10D2D0002FF0F60EF66E410EF76E0BEC30F020ECF0
:10D2E00030F015C192F1110E0101936F0001E5ECD0
:10D2F00030F00B0EF66E420EF76E0E0E0101956FBA
:10D300000001B6EC30F01200CA51906FCBC091F022
:10D31000CCC092F0CDC093F0D250006ED29E3901B5
:10D32000E16B0F0EE06F600043F2E3F9E59DE59FCE
:10D33000E585550EE66FAA0EE66FE583E5B3FED7E9
:10D34000E595E59DE58F0050D212D250006ED29E39
:10D35000E16B100EE06F600047F2E3F9E59DE59F99
:10D36000E585550EE66FAA0EE66FE583E5B3FED7B9
:10D37000E595E59DE58F0050D212D250006ED29E09
:10D38000E16B110EE06F60004BF2E3F9E59DE59F64
:10D39000E585550EE66FAA0EE66FE583E5B3FED789
:10D3A000E595E59DE58F0050D212D250006ED29ED9
:10D3B000E16B120EE06F60004FF2E3F9E59DE59F2F
:10D3C000E585550EE66FAA0EE66FE583E5B3FED759
:10D3D000E595E59DE58F0050D212000198EF7AF0B7
:10D3E0003901E58FE59DF86AD29A078E0E01550E38
:10D3F0003A01BF6FAA0EBF6FBF910B0EE56F080E0B
:10D40000E86F130E096F160E1E6F550EBF6FAA0E32
:10D41000BF6FBF813901DE6BDB6BDD6B050EDF6F2C
:10D42000600ED96F1A6A3D01F39FC392BB82B00EA2
:10D43000F26FF66B220EF56FF46BF38FDB9FC59CDA
:10D44000BD8C340EDA6FDE6B330EDD6FDC6BDB8F81
:10D45000C39CBB8C0001626B616B646B636B6991F5
:10D4600069930101816B8C6B8B6B3A01406B506B44
:10D47000606B706B806B3E01BD6BBE6BBF6BBC6B3A
:10D48000B96BBA6BBB6BB86B330E1B6E2E0E1C6E7A
:10D49000300E1D6E2E0E1E6E340E1F6E206A0101A0
:10D4A000846B856B3F0EC26EB90EC36E800EC46E68
:10D4B000700EC56EC690C692C694C686800E3A019E
:10D4C000616F300E716F000E3E01FD6F3A01406FCB
:10D4D000506F606F706F806F3E01BD6B070EBE6F47
:10D4E000BF6FBC6BB96BBA6FBB6FB86BBD9EBB94A3
:10D4F000BA9CB8A802D0CF0EB76E2C0EB66E900EA6
:10D50000B86E450EB96E010EB56E370EB26EB36AC7
:10D51000B46A3C0EB16EB00EB06E0000010E9D6E8E
:10D52000070E9A6E9B6A9C6A630E996EC00E986E87
:10D530000000010EA96E370EA66EA76AA86A3C0EFF
:10D54000A56EB00EA46E000001011A6B196B179B3B
:10D55000BE90BE92BE94BA9EBC96BC94BC92BC9047
:10D5600016971699169B169D0001F49F01011691BE
:10D57000169316950001FEEF2CF0010117931795F5
:10D580000001FDEC2DF003EC2EF088936F0048FFB6
:10D5900091F1D29E3901E16B300EE06FE59DE59F80
:10D5A000E581E351E59DE58F010191BFD28E000138
:10D5B000F56F6F0048FF91F1D29E3901E16B3C0E8F
:10D5C000E06FE59DE59FE581E351E59DE58F010174
:10D5D00091BFD28E0001D96F6F0048FF91F1D29EAA
:10D5E0003901E16B140EE06FE59DE59FE581E351A4
:10D5F000E59DE58F010191BFD28E016E00018899F2
:10D6000001B088896F0048FF91F1D29E3901E16B2A
:10D61000320EE06FE59DE59FE581E351E59DE58FE5
:10D62000010191BFD28E0001FB6F6F0048FF91F1A5
:10D63000D29E3901E16B330EE06FE59DE59FE581F8
:10D64000E351E59DE58F010191BFD28E0001FD6F91
:10D65000FF0EFD1B6F0048FF91F1D29E3901E16B77
:10D660002F0EE06FE59DE59FE581E351E59DE58F98
:10D67000010191BFD28E0001F16F6F0048FF91F15F
:10D68000D29E3901E16B380EE06FE59DE59FE581A3
:10D69000E351E59DE58F010191BFD28E0001F26F4C
:10D6A0006F0048FF91F1D29E3901E16B310EE06FBE
:10D6B000E59DE59FE581E351E59DE58F010191BF82
:10D6C000D28E0001EF6F6F0048FF91F1D29E3901B9
:10D6D000E16B2D0EE06FE59DE59FE581E351E59D52
:10D6E000E58F010191BFD28E0001F06F6F0048FFFE
:10D6F00091F1D29E3901E16B050EE06FE59DE59F4A
:10D70000E581E351E59DE58F010191BFD28E0001D6
:10D71000CE6FCE515A0802E2050ECE6F6F0048FF61
:10D7200091F1D29E3901E16B3D0EE06FE59DE59FE1
:10D73000E581E351E59DE58F010191BFD28E0001A6
:10D74000E26F0101936BE2C092F1020E956F580EE9
:10D75000946F000136EC2EF0E66BE56B02C0E4F04E
:10D7600001C0E3F0D66BCEC0D5F06F0048FF91F159
:10D77000D29E3901E16B3A0EE06FE59DE59FE581B0
:10D78000E351E59DE58F010191BFD28E926F6F004D
:10D7900048FF93F1D29E3901E16B390EE06FE59DB0
:10D7A000E59FE581E351E59DE58F010193BFD28EB1
:10D7B000946F92C1C9F094C1C8F00001C83D06D071
:10D7C000C93D04D0010EC96F2C0EC86F6F0048FF11
:10D7D00091F1D29E3901E16B070EE06FE59DE59F67
:10D7E000E581E351E59DE58F010191BFD28E926FF6
:10D7F0006F0048FF93F1D29E3901E16B060EE06F96
:10D80000E59DE59FE581E351E59DE58F010193BF2E
:10D81000D28E946F92C1B7F094C1B6F06F0048FFFA
:10D8200091F1D29E3901E16B290EE06FE59DE59FF4
:10D83000E581E351E59DE58F010191BFD28E926FA5
:10D840006F0048FF93F1D29E3901E16B280EE06F23
:10D85000E59DE59FE581E351E59DE58F010193BFDE
:10D86000D28E946F92C1B9F094C1B8F06F0048FFA6
:10D8700091F1D29E3901E16B090EE06FE59DE59FC4
:10D88000E581E351E59DE58F010191BFD28E926F55
:10D890006F0048FF93F1D29E3901E16B080EE06FF3
:10D8A000E59DE59FE581E351E59DE58F010193BF8E
:10D8B000D28E946F92C1BBF094C1BAF06F0048FF52
:10D8C00091F1D29E3901E16B150EE06FE59DE59F68
:10D8D000E581E351E59DE58F010191BFD28E000105
:10D8E000E86F6F0048FF91F1D29E3901E16B370E6E
:10D8F000E06FE59DE59FE581E351E59DE58F010141
:10D9000091BFD28E0001F66FF76B6F0048FF91F167
:10D91000D29E3901E16B0D0EE06FE59DE59FE5813B
:10D92000E351E59DE58F010191BFD28E0001F76FB4
:10D930000101926BF7C091F10001B1EC2FF002C030
:10D94000DBF001C0DAF0F86B6F0048FF91F1D29E76
:10D950003901E16B0B0EE06FE59DE59FE581E35139
:10D96000E59DE58F010191BFD28E0001F86F0101A5
:10D97000926BF8C091F10001B1EC2FF002C0DDF024
:10D9800001C0DCF0889B686B6F0048FF91F1D29E6C
:10D990003901E16B0C0EE06FE59DE59FE581E351F8
:10D9A000E59DE58F010191BFD28E0001ED6FC4921C
:10D9B000BC92FFEC2FF0680EF66E540EF76E0BEC77
:10D9C00030F020EC30F07A0EF66E540EF76E0BEC61
:10D9D00030F001018E6B8D6B8E51130818E303E15B
:10D9E0008D51870814E3CBAE05D000016989010190
:10D9F0000ED003D0000169990101010EA56F00014D
:10DA00009CEC2DF001018D2BD8B48E2BE5D70001B5
:10DA1000FDEC2DF003EC2EF00101906B8F6B905319
:10DA200059E18F51630856E3000169A929D0EDC07F
:10DA300091F12DEC30F0D9517F0811E1FFEC2FF07E
:10DA40008C0EF66E540EF76E0BEC30F020EC30F0CE
:10DA50009E0EF66E540EF76E0BEC30F010D0FFEC0D
:10DA60002FF0B00EF66E540EF76E0BEC30F020EC8B
:10DA700030F0C20EF66E540EF76E0BEC30F025D07F
:10DA80006999D9517F0811E1FFEC2FF0D40EF66EA1
:10DA9000540EF76E0BEC30F020EC30F0E60EF66E24
:10DAA000540EF76E0BEC30F010D0FFEC2FF0F80EA8
:10DAB000F66E540EF76E0BEC30F020EC30F00A0EE0
:10DAC000F66E550EF76E0BEC30F001018F2BD8B4CB
:10DAD000902BA5D700016997DF6BE06B956B88856C
:10DAE0008897896B8A6BDC51BA25C06FDD51BB21E9
:10DAF000C16FDA51B65DBC6FDB51B759BD6FDA51FA
:10DB0000B85DBE6FDB51B959BF6F889DD76B8C6B09
:10DB10008D6B8B6BD86B0101126B0001E16BF49381
:10DB2000FC6B699B9551020802E188EC58F00101F9
:10DB300016971699020E916FFA0EA56F00019CECD4
:10DB40002DF00101912FF8D7169716990001F4993D
:10DB5000F49BF49D0101169F0001F49101011787C8
:10DB600017990001889501011B6B179D816B179F09
:10DB700080910001656B6991FDEC2DF06F0048FF0D
:10DB800091F1D29E3901E16B010EE06FE59DE59FB9
:10DB9000E581E351E59DE58F010191BFD28E186FBC
:10DBA0001853D8A408D1C00ED21200016B6B6A6B57
:10DBB0006D6B6C6B6F6B6E6B050E0101916F936BF0
:10DBC000140E926F030E946F966B6A0E956F0001A0
:10DBD00098EC59F0015251E06BC070F06AC071F0DE
:10DBE0006DC072F06CC073F06FC074F06EC075F0F1
:10DBF000FFEC2FF01C0EF66E550EF76E0BEC30F0AE
:10DC000020EC30F02E0EF66E550EF76E040E01016C
:10DC1000956F0001B6EC30F070C091F1370E010144
:10DC2000926F000143EC5BF071C091F1370E01017E
:10DC3000926F000143EC5BF072C091F1370E01016D
:10DC4000926F000143EC5BF073C091F1370E01015C
:10DC5000926F000143EC5BF074C091F1370E01014B
:10DC6000926F000143EC5BF075C091F1370E01013A
:10DC7000926F000143EC5BF010D0FFEC2FF04C0EE4
:10DC8000F66E550EF76E0BEC30F020EC30F05E0EB9
:10DC9000F66E550EF76E0BEC30F0080E0101916F29
:10DCA000FA0EA56F00019CEC2DF00101912FF8D721
:10DCB00000016B6B6A6B6D6B6C6B6F6B6E6B040E44
:10DCC0000101916F936B140E926F030E946F966B1C
:10DCD0006A0E956F000198EC59F0015251E06BC04B
:10DCE00070F06AC071F06DC072F06CC073F06FC0FC
:10DCF00074F06EC075F0FFEC2FF0700EF66E550EDE
:10DD0000F76E0BEC30F020EC30F0820EF66E550E14
:10DD1000F76E040E0101956F0001B6EC30F070C093
:10DD200091F1370E0101926F000143EC5BF071C07D
:10DD300091F1370E0101926F000143EC5BF072C06C
:10DD400091F1370E0101926F000143EC5BF073C05B
:10DD500091F1370E0101926F000143EC5BF074C04A
:10DD600091F1370E0101926F000143EC5BF075C039
:10DD700091F1370E0101926F000143EC5BF010D07E
:10DD8000FFEC2FF0A00EF66E550EF76E0BEC30F098
:10DD900020EC30F0B20EF66E550EF76E0BEC30F054
:10DDA000080E0101916FFA0EA56F00019CEC2DF099
:10DDB0000101912FF8D7BA9C010E0C6FC00ED21240
:10DDC00039019685938F9481988D968DBD9E000123
:10DDD0006991F9EC5BF09EEC5DF03BEC5CF0879FA9
:10DDE0000101065311E00001FB3D03D001010CD0FD
:10DDF0000001F4A502D0010107D0FC2BFC51FB5D12
:10DE000001E2F483F4850101000188A702D0F493B4
:10DE1000FC6B88A501D0F495CBBE75D069A973D0F1
:10DE2000F499F49B6F0048FF91F1D29E3901E16BA8
:10DE3000070EE06FE59DE59FE581E351E59DE58FE8
:10DE4000010191BFD28E926F6F0048FF93F1D29E75
:10DE50003901E16B060EE06FE59DE59FE581E35139
:10DE6000E59DE58F010193BFD28E946F92C1B7F00B
:10DE700094C1B6F06F0048FF91F1D29E3901E16B79
:10DE8000090EE06FE59DE59FE581E351E59DE58F96
:10DE9000010191BFD28E926F6F0048FF93F1D29E25
:10DEA0003901E16B080EE06FE59DE59FE581E351E7
:10DEB000E59DE58F010193BFD28E946F92C1BBF0B7
:10DEC00094C1BAF0926BF7C091F10001B1EC2FF060
:10DED00002C0DBF001C0DAF0DA51B65DBC6FDB5195
:10DEE000B759BD6F0101926BF8C091F10001B1EC1F
:10DEF0002FF002C0DDF001C0DCF0DC51BA25C06FAC
:10DF0000DD51BB21C16FF4AB74D0EF5372E1F49BD0
:10DF10006F0048FF91F1D29E3901E16B070EE06F6F
:10DF2000E59DE59FE581E351E59DE58F010191BF09
:10DF3000D28E926F6F0048FF93F1D29E3901E16B50
:10DF4000060EE06FE59DE59FE581E351E59DE58FD8
:10DF5000010193BFD28E946F92C1B7F094C1B6F015
:10DF60006F0048FF91F1D29E3901E16B090EE06F1D
:10DF7000E59DE59FE581E351E59DE58F010191BFB9
:10DF8000D28E926F6F0048FF93F1D29E3901E16B00
:10DF9000080EE06FE59DE59FE581E351E59DE58F86
:10DFA000010193BFD28E946F92C1BBF094C1BAF0BD
:10DFB000926BF7C091F10001B1EC2FF002C0DBF0E1
:10DFC00001C0DAF0DA51B65DBC6FDB51B759BD6FF5
:10DFD0000101926BF8C091F10001B1EC2FF002C089
:10DFE000DDF001C0DCF0DC51BA25C06FDD51BB2192
:10DFF000C16FF4BD31D0010116A902D000012CD0AF
:10E000000001F4A929D0EF5327E1F499B9C0B7F082
:10E01000B8C0B6F00101926BF7C091F10001B1EC0C
:10E020002FF002C0DBF001C0DAF0DA51B65DBC6F50
:10E03000DB51B759BD6F0101926BF8C091F100013E
:10E04000B1EC2FF002C0DDF001C0DCF0DC51BA25EC
:10E05000C06FDD51BB21C16F88A501D0F49DEF3D9C
:10E0600002D0F499F49B3BEC5CF088A70AD088B509
:10E0700008D0010116A702D0000103D0045315E116
:10E08000000188A7CBEF73F088B5CBEF73F00101E7
:10E0900016A702D000017FD30053D8B402D00001EC
:10E0A0007AD30001F53D77D30101005308E1000167
:10E0B000F53D01D002D0010102D00DD00101025383
:10E0C000D8A402D0000107D0CBBE54D1000169B959
:10E0D00002D001014FD18E6BF53D0DD00101966B41
:10E0E000956B946B936B9A6B996B986B020E976F11
:10E0F000000150EC30F0B2530BE1B35309E1B453DB
:10E1000007E1B55305E139015B5104000001F3D784
:10E1100001010453D8B49FD00001F48F010116917E
:10E120000001F4AF03D0010116810001F15305E1B4
:10E13000F25303E1CBBE01D0698BFD3D01D0FD6BF5
:10E14000FD510A0DF3500101916F966B956B946B25
:10E15000936B9A6B996B986B976F000150EC30F052
:10E16000B2536EE1B3536CE1B4536AE1B55368E165
:10E17000D93D20D0FFEC2FF0C40EF66E550EF76E91
:10E180000BEC30F020EC30F0D60EF66E550EF76E3C
:10E19000070E0101956F0001B6EC30F0090EE96E33
:10E1A000CDC098F1CCC097F1CBC096F1CAC095F123
:10E1B000CFEC5EF0D95320E1FFEC2FF0E20EF66ECB
:10E1C000550EF76E0BEC30F020EC30F0F40EF66EDE
:10E1D000550EF76E070E0101956F0001B6EC30F099
:10E1E000090EE96ECDC098F1CCC097F1CBC096F185
:10E1F000CAC095F1CFEC5EF0D9517F0820E1FFEC69
:10E200002FF0000EF66E560EF76E0BEC30F020EC91
:10E2100030F0120EF66E560EF76E070E0101956F76
:10E220000001B6EC30F0090EE96ECDC098F1CCC01B
:10E2300097F1CBC096F1CAC095F1CFEC5EF090D7C4
:10E24000010116870001F4A703D00101168B00011C
:10E2500069978ED001010001FD3D01D0FD6BFD519C
:10E260000A0DF3500101916F966B956B946B936B54
:10E270009A6B996B986B976F000150EC30F0B2532A
:10E280006EE1B3536CE1B4536AE1B55368E1D93D33
:10E2900020D0FFEC2FF01E0EF66E560EF76E0BEC34
:10E2A00030F020EC30F0300EF66E560EF76E070EA2
:10E2B0000101956F0001B6EC30F0090EE96ECDC09A
:10E2C00098F1CCC097F1CBC096F1CAC095F1CFECD4
:10E2D0005EF0D95320E1FFEC2FF03C0EF66E560EA7
:10E2E000F76E0BEC30F020EC30F04E0EF66E560E62
:10E2F000F76E070E0101956F0001B6EC30F0090EC4
:10E30000E96ECDC098F1CCC097F1CBC096F1CAC0F0
:10E3100095F1CFEC5EF0D9517F0820E1FFEC2FF0B2
:10E320005A0EF66E560EF76E0BEC30F020EC30F015
:10E330006C0EF66E560EF76E070E0101956F00011A
:10E34000B6EC30F0090EE96ECDC098F1CCC097F173
:10E35000CBC096F1CAC095F1CFEC5EF090D7010129
:10E3600016870001F4A703D00101168B00016997FD
:10E370008E6B01010053D8B40FD20001F53D01D0DE
:10E3800002D0010109D2F053D8A405D2F49FE15381
:10E3900010E10101966B956B946B936BE6C09AF15B
:10E3A000E5C099F1E4C098F1E3C097F1000150ECA9
:10E3B00030F0B253D8A4BFD1B353D8A4BCD1B45316
:10E3C000D8A4B9D1B553D8A4B6D160EC5CF0FE5353
:10E3D00009E10101105303E00001F55303E00001DE
:10E3E000952D02D09EEC5DF09551020802E188EC7B
:10E3F00058F095510308D8B4E1EC5FF0952D01D0A9
:10E400003FD1D93D68D0FFEC2FF0AA51AE5D01019C
:10E41000916F0001AB51AF590101926F0001AC51F6
:10E42000B0590101936F0001AD51B1590101946FD1
:10E43000D892196AD2BE198ED29ECA6F93C1C9F101
:10E4400092C1C8F191C1C7F1CE6BCD6B020ECC6FFA
:10E45000580ECB6F0001D7EC24F019BED28E03C04A
:10E4600094F102C093F101C092F100C091F1010E4C
:10E4700001019127000E922393239423780EF66EC8
:10E48000560EF76E0D0E956F0001B6EC30F0030ED0
:10E49000E96E94C198F193C197F192C196F191C13F
:10E4A00095F1CFEC5EF020EC30F08A0EF66E560E51
:10E4B000F76E070E0101956F0001B6EC30F0090E02
:10E4C000E96ECDC098F1CCC097F1CBC096F1CAC02F
:10E4D00095F1CFEC5EF0D95368E1FFEC2FF0AA5133
:10E4E000AE5D0101916F0001AB51AF590101926F17
:10E4F0000001AC51B0590101936F0001AD51B15908
:10E500000101946FD892196AD2BE198ED29ECA6F39
:10E5100093C1C9F192C1C8F191C1C7F1CE6BCD6B66
:10E52000020ECC6F580ECB6F0001D7EC24F019BE51
:10E53000D28E03C094F102C093F101C092F100C0E9
:10E5400091F1010E01019127000E92239323942350
:10E55000960EF66E560EF76E0D0E956F0001B6EC28
:10E5600030F0030EE96E94C198F193C197F192C116
:10E5700096F191C195F1CFEC5EF020EC30F0A80E51
:10E58000F66E560EF76E070E0101956F0001B6ECA0
:10E5900030F0090EE96ECDC098F1CCC097F1CBC038
:10E5A00096F1CAC095F1CFEC5EF0D9517F0868E1D1
:10E5B000FFEC2FF0AA51AE5D0101916F0001AB514C
:10E5C000AF590101926F0001AC51B0590101936F35
:10E5D0000001AD51B1590101946FD892196AD2BEB0
:10E5E000198ED29ECA6F93C1C9F192C1C8F191C16F
:10E5F000C7F1CE6BCD6B020ECC6F580ECB6F000106
:10E60000D7EC24F019BED28E03C094F102C093F16E
:10E6100001C092F100C091F1010E01019127000E9D
:10E62000922393239423B40EF66E560EF76E0D0EBE
:10E63000956F0001B6EC30F0030EE96E94C198F1CD
:10E6400093C197F192C196F191C195F1CFEC5EF033
:10E6500020EC30F0C60EF66E560EF76E070E010176
:10E66000956F0001B6EC30F0090EE96ECDC098F15F
:10E67000CCC097F1CBC096F1CAC095F1CFEC5EF05B
:10E680000101005308E10001F53D01D002D0010174
:10E6900002D00DD001010253D8A402D0000107D04E
:10E6A000CBBE43D0000169B902D001013ED00101C7
:10E6B000178900018E6B0101966B956B946B936BC0
:10E6C0009A6B996B986B020E976F000150EC30F0CB
:10E6D000B2530BE1B35309E1B45307E1B55305E17C
:10E6E00039015B5104000001F3D70101005313E02D
:10E6F0000001F53D01D002D001010DD0010104530C
:10E7000006E016870001F4A703D00101168B000173
:10E71000699709D0010116870001F4A703D0010110
:10E72000168B000169978E6B0101010E0001E16FEC
:10E73000F9EC5BF03ED6E12D2ED0F48F0101966B03
:10E74000956B946B936B9A6B996B986B020E976FAA
:10E75000000150EC30F0B2530BE1B35309E1B45374
:10E7600007E1B55305E139015B5104000001F3D71E
:10E770000101045301E016870001F4A703D0010151
:10E78000168B0001010117B902D0168B01D0179921
:10E79000000169978E6B01010001E7EC63F088B717
:10E7A0005AD088B558D0010116A702D0000153D025
:10E7B00016B902D000014FD0005308E10001F53D29
:10E7C00001D002D0010102D01ED001010253D8A411
:10E7D00002D0000118D0CBBE04D0000169B913D01B
:10E7E00001010853D8B402D000010DD00A53D8B4A7
:10E7F00002D0000108D006532FE00001F03D01D007
:10E8000002D0010129D00101169B169D1697169979
:10E81000966B956B946B936B9A6B996B986B0A0ED6
:10E82000976F000150EC30F0B2530BE1B35309E1A4
:10E83000B45307E1B55305E139015B510400000110
:10E84000F3D78E6B010116870001F4A703D00101F5
:10E85000168B000169970101000188B70ED088B5B9
:10E860000CD0010116A702D0000107D016A902D0D2
:10E87000000103D0045313E1000188B731D088B5FB
:10E880002FD0010116A702D000012AD016A902D06C
:10E89000000126D00053D8B402D0000121D000538B
:10E8A00008E10001F53D01D002D0010102D00DD0F8
:10E8B00001010253D8A402D0000107D0CBBE11D071
:10E8C000000169B902D001010CD0010116870001D5
:10E8D000F4A703D00101168B0001F48F69978E6BAA
:10E8E000010100019EEC5DF08799010116B951D23A
:10E8F0000001E83D6AD188A568D1AD6BAC6BAB6B0C
:10E90000AA6BDE6BB56BB46BB36BB26BD6C093F115
:10E91000D5C092F10101956B0A0E946F000136EC9F
:10E920002EF002C092F101C091F10101966B956B3E
:10E93000946B936B9A6B996B02C098F101C097F13D
:10E94000000150EC30F0F49DB253D8A42AD1B35357
:10E95000D8A427D1B453D8A424D1B553D8A421D155
:10E960009EEC5DF03BEC5CF0F553D8B4E7EC63F063
:10E9700039015B510400010116A903D0000111D136
:10E980000101000160EC5CF09551020829E188EC7E
:10E9900058F0AD6BAC6BAB6BAA6BDE6BB56BB46B4D
:10E9A000B36BB26BD6C093F1D5C092F10101956BF8
:10E9B0000A0E946F000136EC2EF002C092F101C0F5
:10E9C00091F10101966B956B946B936B9A6B996BBC
:10E9D00002C098F101C097F1000150EC30F0D4D79B
:10E9E000952D01D003D09551070841E169A93BD08D
:10E9F00020EC30F0D20EF66E560EF76E030E0101CB
:10EA0000956F0001B6EC30F096C0A1F1C7EC2DF087
:10EA100097C0A1F1C7EC2DF098C0A1F1C7EC2DF083
:10EA200099C0A1F1C7EC2DF09AC0A1F1C7EC2DF06F
:10EA30009BC0A1F1C7EC2DF09CC0A1F1C7EC2DF05B
:10EA40009DC0A1F1C7EC2DF0E50EF66E560EF76EE7
:10EA5000040E0101956F0001B6EC30F09EC0A1F1EB
:10EA6000C7EC2DF002D067EC5DF004EC5CF0010126
:10EA7000005323E00001F53D01D002D001011DD07B
:10EA8000F4B302D0010119D0FFEC2FF0EC0EF66EBA
:10EA9000560EF76E0BEC30F020EC30F0FA0EF66EFE
:10EAA000560EF76E0BEC30F0010116971699169B77
:10EAB000169D0001FC6BDBD701010001F493952D3D
:10EAC00001D007D09551070804E0E9EC64F0E1ECCF
:10EAD0005FF00101005308E10001F53D01D002D0D3
:10EAE000010102D02FD001010253D8A402D00001AD
:10EAF00029D00853D8B402D0000124D00A53D8B486
:10EB000002D000011FD0065307E00001F03D01D004
:10EB100002D0010101D016D00001FE5313E1010122
:10EB2000105303E00001F5530DE0000187B90AD04E
:10EB30009551040807E09551070804E0CBBE25D0A5
:10EB400069A923D0010ECE5D0101226F236BD6C0CF
:10EB500093F1D5C092F1956B0A0E946F000136ECDB
:10EB60002EF002C092F101C091F10101966B956BFC
:10EB7000946B936B9A6B996B02C098F101C097F1FB
:10EB8000000150EC30F0879907D00101005305E1F6
:10EB9000236B226B000105D001010001F9EC5BF051
:10EBA000D3D669978E6B889301011689169B168DB3
:10EBB000966B956B946B936B9A6B996B986B976B49
:10EBC000000150EC30F0878DE16BE853D8A4E0D021
:10EBD00088A5DED0010116B9D2D00001F49DF5530D
:10EBE000D8B4E7EC63F00101005323E00001F53DE8
:10EBF00001D002D001011DD0F4B302D0010119D01F
:10EC0000FFEC2FF00C0EF66E570EF76E0BEC30F09B
:10EC100020EC30F01A0EF66E570EF76E0BEC30F05B
:10EC2000010116971699169B169D0001FC6BDBD708
:10EC300001010001F4939551020803E09551050884
:10EC400055E19551020802E188EC58F0955105080C
:10EC50004CE10101005308E10001F53D01D002D073
:10EC6000010102D02AD001010853D8B402D000011A
:10EC700024D00A53D8B402D000011FD0065307E0B5
:10EC80000001F03D01D002D0010101D016D00001F9
:10EC9000FE5313E10101105303E00001F5530DE0B1
:10ECA000000187B90AD09551040807E0955107087B
:10ECB00004E0CBBE05D069A903D0E9EC64F015D01F
:10ECC00001010253D8B45BD00001FFEC2FF02C0EF1
:10ECD000F66E570EF76E0BEC30F020EC30F03E0E77
:10ECE000F66E570EF76E0BEC30F043D060EC5CF034
:10ECF00069A93BD020EC30F0500EF66E570EF76E3F
:10ED0000030E0101956F0001B6EC30F096C0A1F141
:10ED1000C7EC2DF097C0A1F1C7EC2DF098C0A1F180
:10ED2000C7EC2DF099C0A1F1C7EC2DF09AC0A1F16C
:10ED3000C7EC2DF09BC0A1F1C7EC2DF09CC0A1F158
:10ED4000C7EC2DF09DC0A1F1C7EC2DF0630EF66E5F
:10ED5000570EF76E040E0101956F0001B6EC30F00E
:10ED60009EC0A1F1C7EC2DF002D067EC5DF004EC81
:10ED70005CF09EEC5DF03BEC5CF02CD70101168959
:10ED8000169B168D000169978E6B8893878DE16BBA
:10ED90000101000160EC5CF0010116A702D016AB86
:10EDA00004D016A97CD016BB7AD00001952D3FD097
:10EDB00069A93BD020EC30F06A0EF66E570EF76E64
:10EDC000030E0101956F0001B6EC30F096C0A1F181
:10EDD000C7EC2DF097C0A1F1C7EC2DF098C0A1F1C0
:10EDE000C7EC2DF099C0A1F1C7EC2DF09AC0A1F1AC
:10EDF000C7EC2DF09BC0A1F1C7EC2DF09CC0A1F198
:10EE0000C7EC2DF09DC0A1F1C7EC2DF07D0EF66E84
:10EE1000570EF76E040E0101956F0001B6EC30F04D
:10EE20009EC0A1F1C7EC2DF002D067EC5DF0952DEE
:10EE300001D034D0D9517F0819E120EC30F0840E94
:10EE4000F66E570EF76E070E0101956F0001B6ECD6
:10EE500030F0090EE96ECDC098F1CCC097F1CBC06F
:10EE600096F1CAC095F1CFEC5EF018D020EC30F0EE
:10EE7000900EF66E570EF76E070E0101956F0001AA
:10EE8000B6EC30F0090EE96ECDC098F1CCC097F128
:10EE9000CBC096F1CAC095F1CFEC5EF00101000144
:10EEA00088A7B4D0010116A702D00001AFD000019D
:10EEB000F49F952D41D069A93BD020EC30F09C0EF9
:10EEC000F66E570EF76E030E0101956F0001B6EC5A
:10EED00030F096C0A1F1C7EC2DF097C0A1F1C7ECBE
:10EEE0002DF098C0A1F1C7EC2DF099C0A1F1C7ECAD
:10EEF0002DF09AC0A1F1C7EC2DF09BC0A1F1C7EC99
:10EF00002DF09CC0A1F1C7EC2DF09DC0A1F1C7EC84
:10EF10002DF0AF0EF66E570EF76E040E0101956FD1
:10EF20000001B6EC30F09EC0A1F1C7EC2DF002D08C
:10EF300067EC5DF004EC5CF0952D01D067D0D93D15
:10EF400020D0FFEC2FF0B60EF66E570EF76E0BECDE
:10EF500030F020EC30F0C80EF66E570EF76E070E4C
:10EF60000101956F0001B6EC30F0090EE96ECDC0DD
:10EF700098F1CCC097F1CBC096F1CAC095F1CFEC17
:10EF80005EF0D95320E1FFEC2FF0D40EF66E570E51
:10EF9000F76E0BEC30F020EC30F0E60EF66E570E0C
:10EFA000F76E070E0101956F0001B6EC30F0090E07
:10EFB000E96ECDC098F1CCC097F1CBC096F1CAC034
:10EFC00095F1CFEC5EF0D9517F0820E1FFEC2FF0F6
:10EFD000F20EF66E570EF76E0BEC30F020EC30F0C0
:10EFE000040EF66E580EF76E070E0101956F0001C4
:10EFF000B6EC30F0090EE96ECDC098F1CCC097F1B7
:10F00000CBC096F1CAC095F1CFEC5EF0010116B904
:10F01000B9D016B7B7D0000188A702D00101B2D08D
:10F0200088A502D00101AED0952D41D069A93BD071
:10F0300020EC30F0100EF66E580EF76E030E010144
:10F04000956F0001B6EC30F096C0A1F1C7EC2DF041
:10F0500097C0A1F1C7EC2DF098C0A1F1C7EC2DF03D
:10F0600099C0A1F1C7EC2DF09AC0A1F1C7EC2DF029
:10F070009BC0A1F1C7EC2DF09CC0A1F1C7EC2DF015
:10F080009DC0A1F1C7EC2DF0230EF66E580EF76E61
:10F09000040E0101956F0001B6EC30F09EC0A1F1A5
:10F0A000C7EC2DF002D067EC5DF004EC5CF0952D20
:10F0B00001D067D0D93D20D0FFEC2FF02A0EF66E9C
:10F0C000580EF76E0BEC30F020EC30F03C0EF66E84
:10F0D000580EF76E070E0101956F0001B6EC30F087
:10F0E000090EE96ECDC098F1CCC097F1CBC096F176
:10F0F000CAC095F1CFEC5EF0D95320E1FFEC2FF0C0
:10F10000480EF66E580EF76E0BEC30F020EC30F037
:10F110005A0EF66E580EF76E070E0101956F00013C
:10F12000B6EC30F0090EE96ECDC098F1CCC097F185
:10F13000CBC096F1CAC095F1CFEC5EF0D9517F08F3
:10F1400020E1FFEC2FF0660EF66E580EF76E0BEC1A
:10F1500030F020EC30F0780EF66E580EF76E070E99
:10F160000101956F0001B6EC30F0090EE96ECDC0DB
:10F1700098F1CCC097F1CBC096F1CAC095F1CFEC15
:10F180005EF00101000160EC5CF0010116A79BD06C
:10F190000001952D41D069A93BD020EC30F0840EC0
:10F1A000F66E580EF76E030E0101956F0001B6EC76
:10F1B00030F096C0A1F1C7EC2DF097C0A1F1C7ECDB
:10F1C0002DF098C0A1F1C7EC2DF099C0A1F1C7ECCA
:10F1D0002DF09AC0A1F1C7EC2DF09BC0A1F1C7ECB6
:10F1E0002DF09CC0A1F1C7EC2DF09DC0A1F1C7ECA2
:10F1F0002DF0970EF66E580EF76E040E0101956F06
:10F200000001B6EC30F09EC0A1F1C7EC2DF002D0A9
:10F2100067EC5DF004EC5CF0952D01D01FD0D93D7A
:10F2200008D0FFEC2FF09E0EF66E580EF76E0BEC2A
:10F2300030F0D95308E1FFEC2FF0B00EF66E580E07
:10F24000F76E0BEC30F0D9517F0808E1FFEC2FF09E
:10F25000C20EF66E580EF76E0BEC30F0BDAF03D059
:10F26000C3AF0AD002D0C3BF2DD0BD51C35D2AE3C6
:10F2700003E1C251BC5D26E2952D02D004EC5CF0A6
:10F28000952D01D01FD0D93D08D020EC30F0D40E00
:10F29000F66E580EF76E0BEC30F0D95308E120EC07
:10F2A00030F0E60EF66E580EF76E0BEC30F0D951DA
:10F2B0007F0808E120EC30F0F80EF66E580EF76E7D
:10F2C0000BEC30F0010116A99ED00001952D41D024
:10F2D00069A93BD020EC30F00A0EF66E590EF76E9D
:10F2E000030E0101956F0001B6EC30F096C0A1F15C
:10F2F000C7EC2DF097C0A1F1C7EC2DF098C0A1F19B
:10F30000C7EC2DF099C0A1F1C7EC2DF09AC0A1F186
:10F31000C7EC2DF09BC0A1F1C7EC2DF09CC0A1F172
:10F32000C7EC2DF09DC0A1F1C7EC2DF01D0EF66EBF
:10F33000590EF76E040E0101956F0001B6EC30F026
:10F340009EC0A1F1C7EC2DF002D067EC5DF004EC9B
:10F350005CF0952D01D01FD0D93D08D0FFEC2FF0E7
:10F36000240EF66E590EF76E0BEC30F0D95308E10F
:10F37000FFEC2FF0360EF66E590EF76E0BEC30F0F8
:10F38000D9517F0808E1FFEC2FF0480EF66E590EB8
:10F39000F76E0BEC30F0C3AF03D0C1AF0AD002D090
:10F3A000C1BF32D0C351C15D2FE303E1C051C25D83
:10F3B0002BE2952D02D004EC5CF0952D01D01FD0EE
:10F3C000D93D08D020EC30F05A0EF66E590EF76E8B
:10F3D0000BEC30F0D95308E120EC30F06C0EF66EF7
:10F3E000590EF76E0BEC30F0D9517F0808E120EC94
:10F3F00030F07E0EF66E590EF76E0BEC30F0010118
:10F4000016A701D0169D0001010116B702D016A95A
:10F4100078D0000169A72ED0010116971699169B86
:10F42000169D0001FFEC2FF0900EF66E590EF76E50
:10F430000BEC30F020EC30F0A20EF66E590EF76EA9
:10F440000BEC30F0640E0101A56F00019CEC2DF077
:10F45000CC8C640E0101A56F00019CEC2DF0CC9CBE
:10F46000640E0101A56F00019CEC2DF001011783D2
:10F47000D4D70001E051080845E20101169716991A
:10F48000169B169DCCBC13D00001FFEC2FF0B40EE0
:10F49000F66E590EF76E0BEC30F020EC30F0C60E25
:10F4A000F66E590EF76E0BEC30F012D00101000130
:10F4B000FFEC2FF0D80EF66E590EF76E0BEC30F015
:10F4C00020EC30F0EA0EF66E590EF76E0BEC30F0D1
:10F4D000640E0101A56F00019CEC2DF0CC8C640E34
:10F4E0000101A56F00019CEC2DF0CC9C640E010184
:10F4F000A56F00019CEC2DF0E06BCC9C0101178303
:10F50000BDD70001E1EC5FF0010116A716D00001A4
:10F5100087BD02D0010111D0010ECA27D8B0CB2B74
:10F52000D8B4CC2BD8B4CD2B879D8E6B84EF69F0EB
:10F53000FDEC2DF003EC2EF00101000195510208C5
:10F5400002E188EC58F0DF510A0805E2FDEC2DF0ED
:0EF5500003EC2EF0DF6B0101DEEF6EF0030026
:00000001FF
